:1000000000800010CD0000003D4A00003F4A000083
:10001000414A0000434A0000454A00000000000039
:10002000000000000000000000000000474A00003F
:10003000494A0000000000004B4A0000C9070000C8
:100040004F4A00004F4A00004F4A00004F4A00004C
:100050004F4A00004F4A00004F4A00004F4A00003C
:100060004F4A00004F4A00004F4A00004F4A00002C
:100070004F4A00004F4A00004F4A00004F4A00001C
:100080004F4A00004F4A00004F4A00004F4A00000C
:100090004F4A00004F4A00004F4A00004F4A0000FC
:1000A0004F4A00004F4A00004F4A00004F4A0000EC
:1000B0004F4A00004F4A00004F4A00004F4A0000DC
:1000C0004F4A00004F4A00004F4A00000148804755
:1000D000014800471D8500002509010040F26053DA
:1000E000C1F200031A780AB901201870704700BFE6
:1000F00040F20000C1F2000008B503682BB140F2E5
:100100000003C0F2000303B1984708BD00B583B0F7
:100110004FF000038DF802304FF000038DF80430EB
:100120004FF000038DF803304FF001038DF80030DD
:100130004FF012038DF801306B46184606F058FC5C
:100140004FF000038DF802304FF000038DF80430BB
:100150004FF000038DF803304FF003038DF80030AB
:100160004FF01A038DF801306B46184606F040FC3C
:100170004FF003004FF080614FF0010205F02CFFBB
:100180004FF001004FF480214FF0010205F024FFF1
:100190004FF003004FF0806105F048FF4FF0010081
:1001A0004FF4802105F042FF03B000BD00B583B0DD
:1001B000019045F2A473C1F200031B684CF20000E9
:1001C000C4F2000040F69011C0F20101984745F2D8
:1001D000A473C1F200031B684CF20000C4F20000DB
:1001E0000199984745F2AC73C1F200031B684CF2C9
:1001F0000000C4F2000040F6A411C0F201019847CB
:1002000003B000BD10B58AB004F0E0FF45F2AC7356
:10021000C1F200031B684CF20000C4F2000040F67B
:10022000A811C0F20101984745F2AC73C1F2000376
:100230001B684CF20000C4F2000040F6C411C0F28A
:1002400001019847FFF762FF45F2AC73C1F200036A
:100250001B684CF20000C4F2000040F6DC11C0F252
:100260000101984700F0D2FA05AB18464FF0320171
:1002700000F040FF03AB18464FF47A7100F03AFFEC
:1002800045F2AC73C1F200031B684CF20000C4F2EB
:10029000000040F6E811C0F20101984718E045F26D
:1002A000AC73C1F200031B684CF20000C4F2000002
:1002B00040F6F411C0F2010198474FF480130993FE
:1002C00003E0099B03F1FF330993099B002BF8D14D
:1002D00000F0C2FA0346002BE1D045F2AC73C1F244
:1002E00000031B684CF20000C4F2000040F62C2111
:1002F000C0F20101984701F0D1F840F26453C1F215
:1003000000034FF00C021A7040F26453C1F2000374
:100310004FF000025A7040F26453C1F200034FF0F4
:1003200000029A7040F26453C1F200036FF05C0265
:10033000DA7040F26453C1F200034FF021021A71E7
:1003400040F26453C1F200034FF000025A7140F2D0
:100350006453C1F200031A7840F26453C1F20003FF
:100360001A7040F26453C1F200035A7840F26453A9
:10037000C1F200035A7040F26453C1F200039A784C
:1003800040F26453C1F200039A7040F26453C1F228
:100390000003DA7840F26453C1F20003DA7040F2ED
:1003A0006453C1F200031A7940F26453C1F20003AE
:1003B0001A7140F26453C1F200035A7940F2645357
:1003C000C1F200035A714AF6C003ADF81C3007AB06
:1003D00003F1020346F201321A8007AB1B781A467A
:1003E00007AB03F101031B7807A901F102010978AA
:1003F000084607A901F1030109780090019143F231
:100400009C00C1F2000040F63821C0F2010109F061
:1004100059F945F2A473C1F200031B684CF20000C5
:10042000C4F2000043F29C01C1F200019847BDF8FC
:100430001C2045F29C13C1F200031A80AD4B07AAA1
:1004400002F1020212881A804AF6C003ADF81C308D
:1004500007AB03F1020340F201121A8007AB1B78CD
:100460001A4607AB03F101031B7807A901F102014A
:100470000978084607A901F1030109780090019164
:1004800043F29C00C1F2000040F65C21C0F2010181
:1004900009F018F945F2A473C1F200031B684CF28D
:1004A0000000C4F2000043F29C01C1F20001984731
:1004B000BDF81C2045F26813C1F200031A808E4B70
:1004C00007AA02F1020212881A804FF6FF73ADF8F4
:1004D0001C3007AB03F102034FF0FF021A8007AB99
:1004E0001B781A4607AB03F101031B7807A901F13A
:1004F00002010978084607A901F103010978009073
:10050000019143F29C00C1F2000040F68421C0F248
:10051000010109F0D7F845F2A473C1F200031B688A
:100520004CF20000C4F2000043F29C01C1F2000151
:100530009847BDF81C2045F29813C1F200031A80B9
:100540006E4B07AA02F1020212881A8045F2AC73C0
:10055000C1F200031B684CF20000C4F2000040F638
:10056000A421C0F20101984704F05EFA45F2AC7391
:10057000C1F200031B684CF20000C4F2000040F618
:10058000B021C0F20101984708E000BF06E000BFBB
:1005900004E000BF02E000BF00E000BF45F2A01091
:1005A000C1F2000000F026FA03469AB243F220138B
:1005B000C1F200031A8043F22013C1F200031B882A
:1005C000002B49D045F2A013C1F200039C894FF4DF
:1005D000006002F06FFD03469C421BD102F06AFFEF
:1005E0004FF0010001F06CF943F22013C1F2000357
:1005F0001B88002BC9D003F06FF843F22013C1F21F
:1006000000031B8845F2A010C1F20000194600F05B
:1006100019FAC3E745F2A013C1F200039C8940F622
:10062000060002F047FD03469C42B0D102F08EFF67
:1006300043F22013C1F200031B88002BA9D043F220
:100640002013C1F200031B8845F2A010C1F2000084
:10065000194600F0F7F9A1E705AB184600F06EFD6A
:100660000346002B97D005AB184600F051FD4FF024
:10067000000308932BE0089B4FF0CC0202FB03F22F
:1006800043F23813C1F200031A4443F23413C1F2A7
:1006900000031A604FF0020001F012F943F2201338
:1006A000C1F200031B88002B0DD003F015F843F2B4
:1006B0002013C1F200031B8845F2A010C1F2000014
:1006C000194600F0BFF9089B03F101030893089B4A
:1006D000272BD0D903AB184600F030FD0346002B82
:1006E0003FF45BAF03AB184600F012FD02F056FD7D
:1006F00054E700BF9E5100106A5100109A5100103B
:1007000008B5FFF77FFD0346184608BD82B001908B
:100710000091FEE782B0034600918DF807309DF905
:100720000730002B11DA4EF60053CEF200039DF88D
:10073000072002F00F02A2F10401009AD2B24FEAA0
:10074000C202D2B20B441A760DE04EF20013CEF282
:1007500000039DF90710009AD2B24FEAC202D2B24A
:100760000B4483F8002302B0704700BF00B583B08C
:100770000190019A6FF07F439A4202D94FF0010332
:100780001FE04EF21003CEF20003019A22F07F42E6
:1007900002F1FF325A604FF0FF304FF01F01FFF7B8
:1007A000B9FF4EF21003CEF200034FF000029A6040
:1007B0004EF21003CEF200034FF007021A604FF022
:1007C0000003184603B000BD43F2DC03C1F200038E
:1007D0001B6803F1010243F2DC03C1F200031A605B
:1007E00043F2DC03C1F200031B6803F00703002B94
:1007F0000BD14CF22003C2F209034CF22002C2F2E8
:100800000902526982F480225A61704708B543F2A6
:10081000DC03C1F200034FF000021A6040F23C0317
:10082000C1F200031A6848F21F53C5F2EB13A3FB91
:1008300002134FEA53131846FFF798FF0346002BA5
:1008400000D0FEE708BD00BF43F2DC03C1F20003A5
:100850001B681846704700BF00B58BB040F60832E1
:10086000C0F2010204AB92E80300186003F1040334
:1008700019804FF0000308934FF001038DF81A30F0
:100880004FF000038DF81C304FF000038DF81B3043
:100890004FF001038DF818304FF000038DF8193038
:1008A00006AB184606F0A4F84FF001038DF8193096
:1008B00006AB184606F09CF84FF004038DF819308B
:1008C00006AB184606F094F84FF008038DF819307F
:1008D00006AB184606F08CF84FF009038DF8193076
:1008E00006AB184606F084F84FF00A038DF819306D
:1008F00006AB184606F07CF84FF00E038DF8193061
:1009000006AB184606F074F84FF00F038DF8193057
:1009100006AB184606F06CF84FF010038DF819304E
:1009200006AB184606F064F84FF011038DF8193045
:1009300006AB184606F05CF845F2AC73C1F2000352
:100940001B684CF20000C4F2000040F6C021C0F267
:10095000010198479DF810301A469DF811309DF816
:1009600012108E469DF813108C469DF81410084600
:100970009DF81510CDF800E0CDF804C00290039169
:1009800043F2E000C1F2000040F6D421C0F20101C0
:1009900008F098FE45F2A473C1F200031B684CF204
:1009A0000000C4F2000043F2E001C1F200019847E8
:1009B0004FF00003089304AB099308AB184604F00A
:1009C00083FE0346002B02D14FF000030FE045F2F7
:1009D000AC73C1F200031B684CF20000C4F20000CB
:1009E00040F6F421C0F2010198474FF00103184688
:1009F0000BB000BD00B587B001904FF4C063049305
:100A000005F0B6F90346002B02D14FF0000316E0C3
:100A100005F0F0F9034603F101030593049A059BE1
:100A20009A4238BF13460493019B0393049B02939D
:100A300002AB184605F02CF905F0F0F9049B1846B6
:100A400007B000BD00B585B001900091009B002B60
:100A500002D14FF001031AE005F09CF90346002B88
:100A600002D14FF0000312E0009BB3F5C06F28BF26
:100A70004FF4C0630093009B0293019B039302AB6E
:100A8000184605F0C7F805F0E1F94FF001031846E4
:100A900005B000BD84B0039002911346ADF8063056
:100AA000039B029A1A60039BBDF806209A8004B04B
:100AB000704700BF00B585B00390019200930B46CC
:100AC000ADF80A30009B1A88039B9B889A4228D273
:100AD000039B1968019B1A68009B1B8808461146F6
:100AE0001A4608F01DFC039B1A68009B1B881A44D9
:100AF000039B1A60039B9A88009B1B88C3EB02032D
:100B00009AB2039B9A80019B1A68009B1B881A4427
:100B1000019B1A60009B4FF000021A804FF0000307
:100B200051E0009B1A88039B9B889A4223D1039B28
:100B30001968019B1A68009B1B88084611461A46D3
:100B400008F0EEFB039B1A68009B1B881A44039B6A
:100B50001A60039B4FF000029A80019B1A68009B69
:100B60001B881A44019B1A60009B4FF000021A80F8
:100B70004FF0010327E0039B1968019B1A68039B50
:100B80009B88084611461A4608F0CAFB039B1A6860
:100B9000039B9B881A44039B1A60009B1A88039B43
:100BA0009B88C3EB02039AB2009B1A80019B1A68D0
:100BB000039B9B881A44019B1A60039B4FF0000221
:100BC0009A804FF00103184605B000BD84B08DF83F
:100BD000071024E00168D2F800C09CF800C081F83A
:100BE00000C009788DF80F10116801F10101116042
:100BF000016801F101010160198801F1FF3189B239
:100C00001980818801F1FF3189B281809DF80FC080
:100C10009DF807108C4502D14FF0020327E0818830
:100C2000002902D019880029D4D11988002918D1A7
:100C30004FF000031BE0116809788DF80F10198838
:100C400001F1FF3189B21980116801F101011160D0
:100C50009DF80F009DF80710884203D14FF0030361
:100C600005E000BF19880029E5D14FF001031846BF
:100C700004B0704710B5044694F82030062B08D114
:100C800043F22C13C1F200031B7803F00403002B82
:100C900021D0228A43F23413C1F200031B685B8A1D
:100CA0009A420BD9626843F23413C1F200031B6805
:100CB0005B8A1046194602F013FA05E06268238A3F
:100CC0001046194602F00CFA4FF0060384F8203063
:100CD0004FF0010301E04FF00003184610BD00BFC4
:100CE000034693F82020062A35D143F22C12C1F294
:100CF0000002127802F00102D2B2002A2BD0198A27
:100D000043F23412C1F200021268528A914214D99D
:100D1000198A43F23412C1F200021268528AC2EBFD
:100D2000010292B21A82596843F23412C1F20002EF
:100D30001268528A0A445A6006E059681A8A0A44BC
:100D40005A604FF000021A824FF0010283F820200F
:100D50004FF0010301E04FF000031846704700BF59
:100D600030B585B00446019100924FF001038DF833
:100D70000F306388002B02D0D02B16D02DE0009BC3
:100D8000002B05D14FF0000363804FF001032DE0ED
:100D9000019B6360009B9BB223824FF0000384F8A9
:100DA000203013E04FF0D00363802046FFF798FF18
:100DB00003461D462046FFF75DFF034605EA030391
:100DC000DBB2002B02D14FF000030FE0238A002B8F
:100DD000E8D14FF0000384F820304FF000038DF885
:100DE0000F304FF0000363804FF00203184605B048
:100DF00030BD00BF30B585B00446019100924FF080
:100E000001038DF80F306388002B02D0EF2B27D021
:100E10003EE0019B002B05D14FF0000363804FF0B3
:100E200001033EE0019B009898470346238243F26A
:100E30003013C1F200031B6863604FF0000384F8B5
:100E4000203043F22C13C1F200031B7803F004039B
:100E5000002B02D0019B009898474FF0EF0363806E
:100E60002046FFF73DFF03461D462046FFF702FFE1
:100E7000034605EA0303DBB2002B02D14FF0000367
:100E80000FE0238A002BDCD14FF0000384F82030E0
:100E90004FF000038DF80F304FF0000363804FF0E8
:100EA0000203184605B030BD82B00190019BDB699A
:100EB0009AB2019B1B8BC3EB02039BB2184602B094
:100EC000704700BF82B00190019B5B8A002B02D06B
:100ED0004FF001031AE0019B93F82030022B07D159
:100EE000019B4FF0030283F820204FF000030DE038
:100EF00043F22C13C1F200031B7803F00203002B12
:100F000002D04FF0010301E04FF00003184602B099
:100F1000704700BF10B584B004460B468DF807300B
:100F20004FF001038DF80F306388002B03D0B3F529
:100F30008E7F10D047E004F11401E268E3699BB2B0
:100F4000084611461A46FFF7A5FD638A002B1BD100
:100F50004FF48E7363802046FFF7B4FF0346002BE7
:100F600002D14FF0000337E04FF0020384F8203045
:100F700043F23013C1F200031B68A36043F2201355
:100F8000C1F200031B88638204F1140004F108021B
:100F900004F112039DF80710FFF718FE034603F053
:100FA0000203002BD1D02046FFF77EFF0346002B23
:100FB00009D14FF0000384F820304FF00003638024
:100FC0004FF0000308E04FF000038DF80F304FF0B2
:100FD000000363804FF00203184604B010BD00BF49
:100FE00010B582B004464FF001038DF807306388D6
:100FF000002B04D040F23712934210D04BE004F1A2
:101000001401E268E3699BB2084611461A46FFF7ED
:1010100041FD638A002B21D140F2371363802046C3
:10102000FFF750FF0346002B02D14FF000033BE0D7
:1010300040F61030C0F2010008F0A4FA4FF00203AD
:1010400084F8203043F23013C1F200031B68A36020
:1010500043F22013C1F200031B88638204F11400E1
:10106000E36999B204F1080204F11203FFF722FDCB
:101070000346012BCDD12046FFF716FF0346002B78
:1010800009D14FF0000384F820304FF00003638053
:101090004FF0000308E04FF000038DF807304FF0E9
:1010A000000363804FF00203184602B010BD00BF7A
:1010B00010B582B00446019100924FF0000384F80D
:1010C00020304FF000036382019BE360009BE361EB
:1010D00004F11402009B9BB2104601991A46FFF7D7
:1010E000D9FC4FF0000323804FF00003638002B06F
:1010F00010BD00BF00B583B001900091019B009A24
:101100005A60FFF7A1FB0246019B1A6003B000BDC5
:1011100082B00190019B1A68019B5B681A44019B95
:101120001A6002B0704700BF00B583B00190FFF7AE
:101130008BFB0246019B1A6003B000BD00B583B073
:101140000190FFF781FB0246019B1B68C3EB020283
:10115000019B5B689A4234BF00230123184603B009
:1011600000BD00BF82B00346ADF8063040F26C53BC
:10117000C1F20003BDF806201A8002B0704700BF1C
:1011800082B001900B46ADF80230019B03F10303DE
:101190001A78BDF80230DBB21344DAB243F22813F6
:1011A000C1F20003DA70019B03F102031A78BDF863
:1011B00002304FEA13239BB2DBB21344DAB243F29C
:1011C0002813C1F200039A70019B03F101031A78FE
:1011D00043F22813C1F200035A70019B1A7843F2BC
:1011E0002813C1F200031A7043F22813C1F200035E
:1011F0009B781A46BDF802304FEA13239BB29A42FD
:1012000020D243F22813C1F200035B7803F10103FB
:10121000DAB243F22813C1F200035A7043F22813E2
:10122000C1F200035B78002B0CD143F22813C1F20A
:1012300000031B7803F10103DAB243F22813C1F271
:1012400000031A7043F22813C1F20003DB781A4638
:10125000BDF8023003F0FF039A4234DA43F2281358
:10126000C1F200039B7803F10103DAB243F22813C1
:10127000C1F200039A7043F22813C1F200039B7875
:10128000002B20D143F22813C1F200035B7803F155
:101290000103DAB243F22813C1F200035A7043F299
:1012A0002813C1F200035B78002B0CD143F2281302
:1012B000C1F200031B7803F10103DAB243F22813F1
:1012C000C1F200031A7002B0704700BF88B00291EB
:1012D00013460246ADF80E20ADF80630029B069389
:1012E000BDF8063003F1FF33029A1344079322E05E
:1012F000069B1B784FEA03239AB2069B03F1010376
:101300001B781344ADF81630BDF80E20BDF816302A
:101310001344ADF80E30BDF80E20BDF816309A42D9
:1013200005D2BDF80E3003F10103ADF80E30069B77
:1013300003F102030693069A079B9A42D8D3069AB2
:10134000079B9A4218D1069B1B784FEA0323ADF8FE
:101350001630BDF80E20BDF816301344ADF80E302F
:10136000BDF80E20BDF816309A4205D2BDF80E30F9
:1013700003F10103ADF80E30BDF80E30184608B089
:10138000704700BF00B583B001900B46ADF8023046
:10139000019ABDF802304FF0000011461A46FFF7DF
:1013A00095FF0346184601F085FE0346184603B034
:1013B00000BD00BF00B583B04FF000000B494FF0F7
:1013C0001402FFF783FF0346ADF80630BDF8063080
:1013D000002B06D0BDF80630184601F06BFE034620
:1013E00001E04FF6FF73184603B000BDAE51001088
:1013F00000B585B003468DF807301D4B9B784FEA4A
:1014000003239AB21A4BDB7813449BB2A3F1140363
:10141000ADF80C309DF80720BDF80C301344ADF842
:101420000E30BDF80E30184612494FF00802FFF793
:101430004DFF0346ADF80E30BDF80E20BDF80C3060
:1014400010460D491A46FFF741FF0346ADF80E302E
:10145000BDF80E30002B06D0BDF80E30184601F056
:1014600029FE034601E04FF6FF73184605B000BDA4
:10147000AE510010BA510010C251001008B54FF023
:101480000600FFF7B5FF0346184608BD08B54FF044
:101490001100FFF7ADFF0346184608BD40F2765332
:1014A000C1F200034FF000021A701AE040F27653C6
:1014B000C1F200031B781A4645F21813C1F200036B
:1014C0004FF0000123F8121040F27653C1F20003EE
:1014D0001B7803F10103DAB240F27653C1F2000344
:1014E0001A7040F27653C1F200031B78272BDDD926
:1014F00040F27653C1F200034FF000021A7020E070
:1015000040F27653C1F200031B781A4643F23813B7
:10151000C1F200034FF0CC0101FB02F2134403F1CE
:1015200018034FF000025A7040F27653C1F20003E4
:101530001B7803F10103DAB240F27653C1F20003E3
:101540001A7040F27653C1F200031B78272BD7D9CB
:1015500040F27453C1F200034FF480621A80704766
:1015600030B583B001900B46ADF8023000E000BF0B
:1015700040F27453C1F200031B8803F101039AB2D5
:1015800040F27453C1F200031A8040F27453C1F266
:1015900000031A8847F6FF439A4206D940F2745373
:1015A000C1F200034FF480521A8040F27653C1F228
:1015B00000034FF000021A702AE040F27653C1F2A5
:1015C00000031B784FF0CC0202FB03F243F2381306
:1015D000C1F2000302EB0304637E002B0BD0A4884E
:1015E00040F27453C1F200031B88184601F062FDFB
:1015F00003469C42BBD040F27653C1F200031B78F5
:1016000003F10103DAB240F27653C1F200031A701B
:1016100040F27653C1F200031B78272BCDD94FF04F
:10162000000440F27653C1F200034FF000021A703A
:101630002AE040F27653C1F200031B784FF0CC024F
:1016400002FB03F243F23813C1F2000302EB03057D
:101650006B7E002B01D12C461DE06B7E072B06D143
:10166000002C03D0AA7EA37E9A4200D92C4640F2D9
:101670007653C1F200031B7803F10103DAB240F2A2
:101680007653C1F200031A7040F27653C1F20003A0
:101690001B78272BCDD9002C02D14FF0000349E055
:1016A0004FF00203637640F27053C1F200031B78DF
:1016B000237340F27053C1F200035B78637340F20E
:1016C0007053C1F200039B78A37340F27053C1F2D0
:1016D0000003DB78E37340F2BA536382638AA38228
:1016E0004FF0010323824FF00003E3764FF0010334
:1016F000A3764FF0030323764FF00003A3754FF05A
:101700001003E37540F27453C1F200031B881846BE
:1017100001F0D0FC0346A380BDF80230E380019BBA
:101720001B88238004F10203019A02F1020212884D
:101730001A802346184603B030BD00BF82B003466E
:10174000ADF8063040F27653C1F200034FF00002CC
:101750001A702BE040F27653C1F200031B781A4650
:1017600045F21813C1F2000333F81230BDF8062019
:101770009A420ED140F27653C1F200031B781A460A
:1017800045F21813C1F200034FF0000123F81210C4
:1017900013E040F27653C1F200031B7803F101031A
:1017A000DAB240F27653C1F200031A7040F2765377
:1017B000C1F200031B78272BCCD902B0704700BFC1
:1017C00082B00346ADF8063040F27653C1F2000312
:1017D0004FF000021A7029E040F27653C1F2000384
:1017E0001B781A4645F21813C1F2000333F8123081
:1017F000002B0ED140F27653C1F200031B781A463B
:1018000045F21813C1F20003BDF8061023F81210B8
:1018100013E040F27653C1F200031B7803F1010399
:10182000DAB240F27653C1F200031A7040F27653F6
:10183000C1F200031B78272BCED902B0704700BF3E
:1018400000B583B00346ADF8063043F23413C1F25D
:1018500000031B6803F10802BDF806301046194664
:10186000FFF78EFC43F23413C1F200031A6843F20F
:101870002813C1F200031B78137243F23413C1F230
:1018800000031A6843F22813C1F200035B78537215
:1018900043F23413C1F200031A6843F22813C1F271
:1018A00000039B78937243F23413C1F200031A6869
:1018B00043F22813C1F20003DB78D37203B000BDFA
:1018C00010B584B003468DF8073043F23413C1F2EB
:1018D00000031C6843F23013C1F20003A94A1A60E6
:1018E00043F23013C1F200031A6843F22413C1F229
:1018F00000031A609DF80730032B14D1637E03F0B8
:101900000F03032B41F0A683238A002B41F0A4830D
:1019100043F22C13C1F200034FF008021A7002F0D8
:10192000F9FF01F041B99DF80730022B40F0F78034
:1019300040F27053C1F20003DB7803F10103DAB225
:1019400040F27053C1F20003DA7040F27053C1F2FA
:101950000003DB78002B34D140F27053C1F2000356
:101960009B7803F10103DAB240F27053C1F2000335
:101970009A7040F27053C1F200039B78002B20D183
:1019800040F27053C1F200035B7803F10103DAB255
:1019900040F27053C1F200035A7040F27053C1F22A
:1019A00000035B78002B0CD140F27053C1F20003AE
:1019B0001B7803F10103DAB240F27053C1F2000365
:1019C0001A7043F22013C1F200034FF000021A8094
:1019D00045F29273C1F200034FF000021A80637E59
:1019E000072B02D0637E052B0DD1A37E03F10103EB
:1019F000DBB2A376A37E782B02D14FF0000363768F
:101A000000BF01F044BB637E002B01F02783238AD3
:101A1000002B73D0A37E03F1FF33DBB2A376A37E4A
:101A2000002B41F01D83E37E082B08D0637E022B40
:101A300002D0637E012B15D1E37E052B12D14FF02E
:101A40000003637643F22C13C1F200036FF07F02B0
:101A50001A7002F05FFF4C4B4FF0140283F8212004
:101A600001F006BAE37E042B06D8E37E4FF00302B2
:101A700002FA03F3DBB201E04FF03003A376E37E1A
:101A800003F10103DBB2E37645F26C13C1F200030C
:101A9000DB8C03F101039AB245F26C13C1F200032F
:101AA000DA84637E03F00F0303F1FF33072B01F2A7
:101AB000D98201A252F823F053240000D91A000061
:101AC000E71A0000712A000065300000712A00004A
:101AD00065300000712A00002B4B4FF0000283F8A4
:101AE000212000F0C0BC43F22C13C1F200034FF0E0
:101AF00004021A7002F00EFF01F0C3B8637E03F017
:101B00000F03032B41F0B08243F22C13C1F2000308
:101B10004FF008021A7002F0FDFE01F045B845F2E0
:101B20006C13C1F200035B8803F101039AB245F222
:101B30006C13C1F200035A80134B1B78452B25D040
:101B400045F26C13C1F200031B8803F101039AB242
:101B500045F26C13C1F200031A8045F26C13C1F216
:101B60000003DB8803F101039AB245F26C13C1F262
:101B70000003DA8040F62C30C0F20100FEF716FBBD
:101B800001F085BAD6510010AE510010A14B9B78E0
:101B90004FEA03229F4BDB781A4443F22013C1F231
:101BA00000031B889A4214DC9A4B9B784FEA03236C
:101BB0009AB2984BDB7813449AB243F22013C1F2E5
:101BC00000031A80934B9B7903F03F03002B0CD149
:101BD00007E040F65430C0F20100FEF7E7FA01F0EA
:101BE00056BA8C4BDB79002B21D045F26C13C1F235
:101BF00000031B8803F101039AB245F26C13C1F292
:101C000000031A8045F26C13C1F200039B8903F1B3
:101C100001039AB245F26C13C1F200039A8140F6B7
:101C20008430C0F20100FEF7C1FA01F030BA45F28B
:101C30009C13C1F200031A8840F62833C0F2010356
:101C40001B889A4205D1744B1A88744B1B889A42A0
:101C50001DD0734B1A8845F29C13C1F200031B88F8
:101C60009A4205D16F4B1A886B4B1B889A420ED053
:101C700045F26C13C1F200031B8803F101039AB211
:101C800045F26C13C1F200031A8001F000BAFFF7AD
:101C900091FB03461A464FF6FF739A4221D045F254
:101CA0006C13C1F200031B8803F101039AB245F2E1
:101CB0006C13C1F200031A8045F26C13C1F20003E9
:101CC000DB8903F101039AB245F26C13C1F2000300
:101CD000DA8140F69C30C0F20100FEF767FA01F0AD
:101CE000D6B94C4B5B7A062B00F0A280494B5B7A4D
:101CF000012B21D045F26C13C1F200031B8803F1C4
:101D000001039AB245F26C13C1F200031A8045F246
:101D10006C13C1F200031B8A03F101039AB245F26E
:101D20006C13C1F200031A8240F6B030C0F2010019
:101D3000FEF73CFA01F0ABB945F26C13C1F20003B7
:101D40009B8A03F101039AB245F26C13C1F20003BE
:101D50009A82304B1B7D082B21D045F26C13C1F2C7
:101D600000035B8A03F101039AB245F26C13C1F2DE
:101D700000035A8245F26C13C1F200031B8B03F17E
:101D800001039AB245F26C13C1F200031A8340F6C4
:101D9000CC30C0F20100FEF709FA01F078B91D4B12
:101DA0004FF000021A751B4BDA8A4FF6F6739A420F
:101DB00007D9184B174AD28A02F1090292B2DA8285
:101DC00006E0144B134AD28A02F1080292B2DA8278
:101DD000134B154A12881A80124B144A12881A8023
:101DE000114A45F29C13C1F200031B8813800F4B6C
:101DF000094A12881A8045F26C13C1F20003DB8A8B
:101E000003F101039AB245F26C13C1F20003DA82C6
:101E100001F00BB9AE5100109E5100102A0B0100C9
:101E2000BE510010C0510010BA510010BC5100103A
:101E300000BF45F26C13C1F200039B8B03F1010359
:101E40009AB245F26C13C1F200039A83FFF716FBB6
:101E500003461A464FF6FF739A4221D045F26C139F
:101E6000C1F200035B8B03F101039AB245F26C13DC
:101E7000C1F200035A8345F26C13C1F200031B8CBC
:101E800003F101039AB245F26C13C1F200031A8404
:101E900040F6E430C0F20100FEF788F901F0F7B82F
:101EA00043F23814C1F200041BE0637E002B16D00D
:101EB0008F4BDA8AA3889A4211D18D4B9A8AE38894
:101EC0009A420CD18B4B1A8823889A4207D18A4BAD
:101ED0001A8804F102031B889A4200F0F58204F18B
:101EE000CC04864B9C42E0D9814B93F8213003F01F
:101EF0003F03022B44D17E4BDA8A40F27853C1F281
:101F000000031A8040F27653C1F200034FF0000242
:101F10001A7020E040F27653C1F200031B781A4693
:101F200045F21813C1F2000333F8122040F278533F
:101F3000C1F200031B889A4200F0E88040F2765319
:101F4000C1F200031B7803F10103DAB240F27653C9
:101F5000C1F200031A7040F27653C1F200031B78FD
:101F6000272BD7D945F26C13C1F200035B8D03F127
:101F700001039AB245F26C13C1F200035A8500E0E6
:101F800000BF5B4B93F8213003F00403002B41F0BA
:101F90006D8045F26C13C1F200039B8C03F10103C9
:101FA0009AB245F26C13C1F200039A84504B4FF081
:101FB000140283F8212043F22013C1F200034FF0F2
:101FC00028021A804A4B4FF0500283F82020484BD9
:101FD000DA7E40F27653C1F200031A70444B444A51
:101FE000D27FDA76424A40F27653C1F200031B7880
:101FF000D3773F4B9A7E40F27653C1F200031A70BA
:102000003B4B3B4A927F9A76394A40F27653C1F273
:1020100000031B789377364B5A7E40F27653C1F219
:1020200000031A70324B324A527F5A76304A40F2DD
:102030007653C1F200031B7853772D4B1A7E40F282
:102040007653C1F200031A70294B294A127F1A767F
:10205000274A40F27653C1F200031B781377244BD2
:10206000DA7F02F10102D2B2DA77DB7F002B17D1DF
:102070001F4B9A7F02F10102D2B29A779B7F002B0D
:102080000ED11B4B5A7F02F10102D2B25A775B7F0D
:10209000002B05D1164B1A7F02F10102D2B21A773A
:1020A000134B9A8A40F27853C1F200031A80104B06
:1020B0000F4AD28A9A820E4A40F27853C1F2000344
:1020C0001B88D3820E4B0B4A12881A800D4B0A4A8A
:1020D00012881A80074A45F29C13C1F200031B883C
:1020E0001380054B084A12881A8000F029BF00BFF0
:1020F000AE510010BA510010BC5100104C500010ED
:10210000BE510010C05100109E51001000BF4FF092
:10211000000440F27653C1F200034FF000021A703F
:102120006AE040F27653C1F200031B781A4643F28C
:102130003813C1F200034FF0CC0101FB02F213444B
:1021400003F118035B78002B0FD140F27653C1F2F4
:1021500000031B784FF0CC0202FB03F243F238136A
:10216000C1F2000302EB03044DE040F27653C1F2EA
:1021700000031B781A4643F23813C1F200034FF0F4
:10218000CC0101FB02F2134403F118035B78072B27
:1021900025D1002C14D040F27653C1F200031B78F5
:1021A0001A4643F23813C1F200034FF0CC0101FB91
:1021B00002F2134403F118039A78A37E9A420ED9CF
:1021C00040F27653C1F200031B784FF0CC0202FBC1
:1021D00003F243F23813C1F2000302EB030440F2AE
:1021E0007653C1F200031B7803F10103DAB240F227
:1021F0007653C1F200031A7040F27653C1F2000325
:102200001B78272B8DD9002C14D145F26C13C1F209
:1022100000031B8D03F101039AB245F26C13C1F266
:1022200000031A8540F6F830C0F20100FDF7BEFF4A
:1022300000F02DBF43F23413C1F200031C604FF0D5
:102240000303A376A37E23764FF00003A3754FF01C
:102250000403E3754FF00003E376984BDB8AA38019
:10226000964B9B8AE380964B1B88238004F10203E4
:10227000944A12881A804FF00103637640F270533B
:10228000C1F200031B78237340F27053C1F20003C4
:102290005B78637340F27053C1F200039B78A373C1
:1022A00040F27053C1F20003DB78E3734FF0010397
:1022B0002382824BDB7EE372804B9B7EA3727F4B3B
:1022C0005B7E63727D4B1B7E23724FF00100FFF734
:1022D000B7FA7A4B93F8203003F0F003502B40F319
:1022E000BD8040F27653C1F200034FF000021A7035
:1022F0009BE040F27653C1F200031B7803F13602F3
:1023000045F2A013C1F200039A5C40F27753C1F288
:1023100000031A7040F27753C1F200031B78002BC0
:1023200000F0998040F27753C1F200031B78012B33
:102330000DD140F27653C1F200031B7803F1010383
:10234000DAB240F27653C1F200031A706DE040F247
:102350007753C1F200031B78022B40D140F2765331
:10236000C1F200031B7803F1370245F2A013C1F25A
:1023700000039B5C042B32D140F27653C1F2000380
:102380001B7803F1380245F2A013C1F200039B5CF5
:102390004FEA03239AB240F27653C1F200031B784E
:1023A00003F1390145F2A013C1F200035B5C42EA7C
:1023B00003039BB29AB240F27853C1F200031A8031
:1023C00040F27853C1F200031A8840F2BA539A429D
:1023D00038BF13469BB26382638AA3823EE040F219
:1023E0007653C1F200031B7803F1370245F2A013C4
:1023F000C1F200039B5C002B2FD040F27653C1F258
:1024000000031B7803F1370245F2A013C1F2000369
:102410009A5C40F27653C1F200031B781344DAB29F
:1024200040F27653C1F200031A7040F27653C1F2C3
:1024300000031B781A46214B93F820304FEA131300
:10244000DBB2A3F105034FEA83039A42FFF651AFD3
:1024500004E000BF02E000BF00E000BF174B4FF0F8
:10246000100283F82120154B144A92F8212042F0E3
:102470000202D2B283F82120104B4FF0020283F8FF
:1024800028200E4B4FF0040283F829200B4B4FF00D
:10249000050283F82A20094B6FF0450283F82B20B0
:1024A00043F22013C1F200034FF02C021A80034BB9
:1024B0004FF0600283F8202000F0E6BCAE5100101F
:1024C000BA510010BC51001000BF43F23413C1F2E6
:1024D00000031C6043F22C13C1F200034FF0000212
:1024E0001A70924B93F8213003F00403002B13D0A1
:1024F0004FF00003637640F61C40C0F20100FDF788
:1025000055FE43F22C13C1F200034FF020021A7063
:1025100002F000FA00F0BBBD844B93F820304FEA84
:102520001313DBB24FEA8303DAB240F27653C1F2FF
:1025300000031A7043F22013C1F200031A8840F21C
:102540007653C1F200031B78C3EB02039BB2A3F1E5
:1025500014039AB243F22013C1F200031A80637E7F
:1025600003F00F03022B06D1704B93F8213003F0D8
:102570003F03122B25D043F22013C1F200031B8826
:10258000002B06D1694B93F8213003F00303002B95
:1025900017D0664B1A7E237A9A4240F06484634BCC
:1025A0005A7E637A9A4240F05E84604B9A7EA37AA8
:1025B0009A4240F058845D4BDA7EE37A9A4240F0CA
:1025C00052845A4B93F8213003F01003002B00F093
:1025D0009180238A002B00F08D8004F10C02238A65
:1025E00010461946FEF7CCFD504B1A7F43F22813D4
:1025F000C1F200031B789A427CD14C4B5A7F43F2C4
:102600002813C1F200035B789A4273D1474B9A7F3B
:1026100043F22813C1F200039B789A426AD1434BDC
:10262000DA7F43F22813C1F20003DB789A4261D1CA
:1026300043F22813C1F200031B78237343F22813DB
:10264000C1F200035B78637343F22813C1F2000305
:102650009B78A37343F22813C1F20003DB78E37382
:10266000E37E002B3AD1227EA37EC3EB0203DBB2D2
:102670008DF80F309DF80F20A37D4FEAD303DBB216
:10268000C3EB0203DBB28DF80F30A27D9DF80F3053
:102690001344DBB2A3759DF90F30002B05DA9DF8CA
:1026A0000F30C3F100038DF80F309DF80F20E37D4C
:1026B0004FEA9303DBB2C3EB0203DBB28DF80F30BA
:1026C000E27D9DF80F301344DBB2E375A37D4FEA42
:1026D000D303DAB2E37D1344DBB2237643F22C1347
:1026E000C1F200034FF001021A70237EA3764FF06F
:1026F00000032382637E03F00F0303F1FF33072BF4
:1027000000F2B68401A252F823F000BF3127000086
:10271000AD270000DB2900002D2D0000D92D000081
:10272000412E0000652E0000FD2C0000AE5100106F
:1027300043F22C13C1F200031B7803F00103DBB258
:10274000002B00F097844FF00303637643F22C13C1
:10275000C1F200034FF040021A704FF000032382D1
:1027600043F22013C1F200031B88002B14D043F264
:102770002C13C1F200031B7843F00203DAB243F2D8
:102780002C13C1F200031A7043F22013C1F20003AC
:102790001B881846FFF754F845F29273C1F2000304
:1027A0004FF000021A8002F0B5F8FDE143F22C135D
:1027B000C1F200031B7803F00103DBB2002B00F031
:1027C000F980AA4B93F8213003F03F03122B40F01D
:1027D000F180A64B93F8203003F0F003502B40F328
:1027E000BB8040F27653C1F200034FF000021A7032
:1027F0009BE040F27653C1F200031B7803F13602EE
:1028000045F2A013C1F200039A5C40F27753C1F283
:1028100000031A7040F27753C1F200031B78002BBB
:1028200000F0978040F27753C1F200031B78012B30
:102830000DD140F27653C1F200031B7803F101037E
:10284000DAB240F27653C1F200031A706DE040F242
:102850007753C1F200031B78022B40D140F276532C
:10286000C1F200031B7803F1370245F2A013C1F255
:1028700000039B5C042B32D140F27653C1F200037B
:102880001B7803F1380245F2A013C1F200039B5CF0
:102890004FEA03239AB240F27653C1F200031B7849
:1028A00003F1390145F2A013C1F200035B5C42EA77
:1028B00003039BB29AB240F27853C1F200031A802C
:1028C00040F27853C1F200031A8840F2BA539A4298
:1028D00038BF13469BB26382638AA3823CE040F216
:1028E0007653C1F200031B7803F1370245F2A013BF
:1028F000C1F200039B5C002B2DD040F27653C1F255
:1029000000031B7803F1370245F2A013C1F2000364
:102910009A5C40F27653C1F200031B781344DAB29A
:1029200040F27653C1F200031A7040F27653C1F2BE
:1029300000031B781A464D4B93F820304FEA1313CF
:10294000DBB2A3F105034FEA83039A42FFF651AFCE
:1029500002E000BF00E000BF4FF003036376434B8B
:102960001B7E2372414B5B7E6372404B9B7EA37246
:102970003E4BDB7EE3724FF00100FEF761FF43F256
:102980002C13C1F200034FF042021A704FF0000303
:10299000238243F22013C1F200034FF000021A8099
:1029A00045F29273C1F200034FF000021A8001F069
:1029B000B1FFF9E043F22C13C1F200034FF0200203
:1029C0001A7001F0A7FF43F23413C1F200031B6831
:1029D0004FF000025A76FFF7D4BA244B93F8213017
:1029E00003F00103DBB2002B49D0637E03F0100338
:1029F000002B44D1238A002B40F03E8343F2201366
:102A0000C1F200031B8803F101039BB21846FEF7D5
:102A100017FF43F22C13C1F200031B7843F010039D
:102A2000DAB243F22C13C1F200031A7043F22013FE
:102A3000C1F200031B88002B0CD043F22C13C1F20F
:102A400000031B7843F00203DAB243F22C13C1F205
:102A500000031A7001F05EFF4FF0010323824FF074
:102A6000080363764FF00003E37602E0AE510010F6
:102A700000BFA14B4FF0110283F82120F8E19E4BDB
:102A800093F8213003F02003002B2ED043F23013B3
:102A9000C1F200031A68984B93F826304FEA0321DD
:102AA000954B93F8273041EA03031A4443F230135D
:102AB000C1F200031A6043F22013C1F200031A8826
:102AC0008D4B93F826304FEA032399B28A4B93F843
:102AD000273041EA03039BB29BB2C3EB02039AB2D5
:102AE00043F22013C1F200031A8043F22013C1F213
:102AF00000031B88002B19D0637E03F01003002B0A
:102B000014D143F22C13C1F200031B7843F00203EB
:102B1000DAB243F22C13C1F200031A7043F220130D
:102B2000C1F200031B881846FEF78AFE724B93F829
:102B300022304FEA03239AB26F4B93F823301344A9
:102B40009AB240F27853C1F200031A80A28A40F28E
:102B50007853C1F200031B889A4206D340F278539F
:102B6000C1F200031B88002B05D1A28A40F27853E2
:102B7000C1F200031A8040F27853C1F200031B88AF
:102B8000638243F22C13C1F200031B7803F00303AA
:102B9000002B00F0738245F29273C1F200034FF0F4
:102BA00000021A8001F0B6FE43F22C13C1F20003BA
:102BB0001B7803F02003002B0FD045F29273C1F273
:102BC00000034FF000021A804FF0000363764A4B77
:102BD0004FF0140283F821204AE143F22C13C1F292
:102BE00000031B7803F01003002B15D045F29273FD
:102BF000C1F200034FF000021A804FF0010323825C
:102C00004FF0040363764FF00003E3763A4B4FF046
:102C1000110283F821202BE145F29273C1F20003E7
:102C20001B88002B2AD043F22C13C1F200031B781F
:102C300003F00103DBB2002B02D04FF0000323822C
:102C4000238A002B14D1628A45F29273C1F20003E9
:102C50001B889A4205D2628A45F29273C1F2000340
:102C60001A8045F29273C1F200031B88238205E0AB
:102C7000228A45F29273C1F200031A804FF00003DA
:102C8000E37643F22413C1F200031A6843F23013CF
:102C9000C1F200031A6045F29273C1F200031B886F
:102CA000002B11D0238A002B0ED0238A03F1280396
:102CB0009AB243F22013C1F200031A800E4B4FF078
:102CC000180283F82120DAE043F22C13C1F200034A
:102CD0001B7803F00203002B00F0D28143F2201393
:102CE000C1F200034FF028021A80034B4FF010028C
:102CF00083F82120C3E000BFAE51001043F22C1333
:102D0000C1F200031B7803F00103DBB2002B0BD0F0
:102D10004FF00003637643F22C13C1F200034FF02F
:102D200010021A7001F0F6FD00BFB0E143F220136B
:102D3000C1F200031B88002B07D043F22013C1F21D
:102D400000031B881846FEF77BFD724B93F8213079
:102D500003F00103DBB2002B24D043F22C13C1F2A9
:102D600000031B7803F00103DBB2002B09D04FF006
:102D7000070363764FF00003A3764FF0000323822E
:102D800002E04FF0060363764FF00100FEF758FDB6
:102D900043F22C13C1F200034FF010021A7001F03D
:102DA000B9FD60E043F22C13C1F200031B7803F07D
:102DB0000103DBB2002B06D04FF0050363764FF022
:102DC0000003238263E143F22013C1F200031B8856
:102DD000002B00F0578146E043F22013C1F20003BC
:102DE0001B88002B07D043F22013C1F200031B887D
:102DF0001846FEF725FD474B93F8213003F00103F9
:102E0000DBB2002B13D04FF0070363764FF00003C3
:102E1000A3764FF00100FEF713FD43F22C13C1F22D
:102E200000034FF010021A7001F074FD1BE043F232
:102E30002013C1F200031B88002B00F0258112E053
:102E400043F22C13C1F200031B7803F00103DBB241
:102E5000002B00F01B814FF0070363764FF0000357
:102E6000A37614E100BF2B4B4FF0100283F8212012
:102E700043F22013C1F200034FF028021A80254BC1
:102E80004FF0500283F82020224B227A1A77214BF0
:102E9000627A5A771F4BA27A9A771E4BE27ADA77D8
:102EA0001C4B227B1A761B4B627B5A76194BA27BFA
:102EB0009A76184BE27BDA76164B4FF006025A727E
:102EC000144BA2889A82134BE288DA82124A45F2A6
:102ED0009C13C1F200031B881380104B104A128808
:102EE0001A80104B22881A800F4B04F102021288BC
:102EF0001A80637E03F01003002B17D0054A054BA0
:102F00004FF0000183F8231093F8233082F8223029
:102F100016E000BFAE510010BA510010BC510010B5
:102F20009E510010BE510010C0510010604B4FF078
:102F3000050283F822205E4B6FF0450283F82320C0
:102F40005B4B4FF040021A72594A43F22013C1F210
:102F500000031B884FEA13239BB2DBB29370544AE1
:102F600043F22013C1F200031B88DBB2D370504A36
:102F70004F4B4FF0000183F8271093F8273082F869
:102F800026304B4B4FF000029A84494CFEF776FAFC
:102F900003466FEA03039BB2A384454B4FF04502FF
:102FA0001A70434B4FF000025A70414A404B4FF0A9
:102FB0000001D971DB79937140F26C53C1F20003C7
:102FC0001B8803F101039AB240F26C53C1F2000373
:102FD0001A80374A40F26C53C1F200031B884FEA53
:102FE00013239BB2DBB21371314A40F26C53C1F22E
:102FF00000031B88DBB253712D4B4FF000025A8146
:103000002B4CFEF7D7F903466FEA03039BB26381AB
:1030100045F26C13C1F20003DB8B03F101039AB29A
:1030200045F26C13C1F20003DA8345F26C13C1F26E
:1030300000039B8803F101039AB245F26C13C1F2BD
:1030400000039A8043F22C13C1F200034FF00002F8
:103050001A702BE000BF1AE000BF18E000BF16E0B6
:1030600000BF14E000BF12E000BF10E000BF0EE0A0
:1030700000BF0CE000BF0AE000BF08E000BF06E0B0
:1030800000BF04E000BF02E000BF00E000BF43F269
:103090002013C1F200034FF000021A8043F22C13F8
:1030A000C1F200034FF000021A7000BF04B010BD5F
:1030B000AE51001082B00346ADF80630BDF80630C0
:1030C0004FEA03239AB2BDF806304FEA13239BB2AE
:1030D00042EA03039BB29BB2184602B0704700BF9E
:1030E00000B583B001900091009B002B1DDD009B7B
:1030F0009AB245F29273C1F200031A8043F224138C
:10310000C1F200031B68019A9A420ED043F22413C5
:10311000C1F200031A6845F29273C1F200031B88E2
:10312000104601991A4606F0FBF803B000BD00BF37
:1031300008B540F2E053C1F200034FF000021A70EC
:1031400024E040F2E053C1F200031B781A46134614
:103150004FEA430313444FEA830240F27C53C1F227
:103160000003134418464FF000014FF0040206F02C
:103170009FF940F2E053C1F200031B7803F1010311
:10318000DAB240F2E053C1F200031A7040F2E053A9
:10319000C1F200031B78072BD3D908BD00B583B05B
:1031A00040F2E253C1F200031B7803F10103DAB2EB
:1031B00040F2E253C1F200031A7040F2E053C1F250
:1031C00000034FF000021A703CE040F2E053C1F2FD
:1031D00000031B781A4613464FEA430313444FEA91
:1031E00083031A4640F27C53C1F200031344019357
:1031F000019B1A88019B5B8842EA03039BB2002B68
:1032000013D040F2E253C1F200031B781A46019B2F
:103210009B7AC3EB0203772B07DD019B18464FF027
:1032200000014FF0040206F043F940F2E053C1F20E
:1032300000031B7803F10103DAB240F2E053C1F25C
:1032400000031A7040F2E053C1F200031B78072B11
:10325000BBD903B000BD00BF10B582B00190009192
:1032600040F2E053C1F200034FF000021A7041E057
:1032700040F2E053C1F200031B781A4613464FEAAE
:10328000430313444FEA83031A4640F27C53C1F2CE
:10329000000302EB03042388002B1ED06388002B5D
:1032A0001BD0019B1A8823889A4216D1019B03F1F7
:1032B00002031A8863889A420FD104F10402009B2A
:1032C000104619464FF0060206F02AF840F2E25383
:1032D000C1F200031B78A372EAE040F2E053C1F2AE
:1032E00000031B7803F10103DAB240F2E053C1F2AC
:1032F00000031A7040F2E053C1F200031B78072B61
:10330000B6D940F2E053C1F200034FF000021A7048
:1033100025E040F2E053C1F200031B781A46134641
:103320004FEA430313444FEA83031A4640F27C53A7
:10333000C1F2000302EB03042388002B02D163884F
:10334000002B14D040F2E053C1F200031B7803F1CC
:103350000103DAB240F2E053C1F200031A7040F206
:10336000E053C1F200031B78072BD2D900E000BF65
:1033700040F2E053C1F200031B78082B40F082803A
:1033800040F2E353C1F200034FF000021A7040F222
:10339000E153C1F200034FF000021A7040F2E05313
:1033A000C1F200034FF000021A7047E040F2E05310
:1033B000C1F200031B781A4613464FEA4303134435
:1033C0004FEA83031A4640F27C53C1F2000302EB3A
:1033D000030440F2E253C1F200031B781A46A37AB9
:1033E000C3EB020240F2E353C1F200031B789A429E
:1033F00017DD40F2E253C1F200031A78A37AC3EB5F
:103400000203DAB240F2E353C1F200031A7040F251
:10341000E053C1F200031A7840F2E153C1F2000315
:103420001A7040F2E053C1F200031B7803F101036C
:10343000DAB240F2E053C1F200031A7040F2E053F6
:10344000C1F200031B78072BB0D940F2E153C1F25F
:1034500000031A7840F2E053C1F200031A7040F200
:10346000E053C1F200031B781A4613464FEA4303A8
:1034700013444FEA83031A4640F27C53C1F200031F
:1034800002EB03042346184601994FF0040205F0AD
:1034900047FF04F10402009B104619464FF0060254
:1034A00005F03EFF40F2E253C1F200031B78A37225
:1034B00002B010BD08B543F22013C1F200031B880F
:1034C000A3F10E039AB243F22013C1F200031A8053
:1034D00045F2A013C1F200035A8B45F29C13C1F2CE
:1034E00000031B8882EA03039AB245F29813C1F2E3
:1034F00000031B8802EA03039BB2002B1ED145F296
:10350000A013C1F200039A8B45F29C13C1F2000391
:103510005B8882EA03039AB245F29813C1F2000372
:103520005B8802EA03039BB2002B09D1054A064BD4
:1035300010461946FFF790FE00BF02E000BF00E012
:1035400000BF08BDBA510010A651001008B543F2E3
:103550002013C1F200031B88292B07D843F2201344
:10356000C1F200034FF000021A80A5E043F22013DD
:10357000C1F200034FF000021A8045F2A013C1F21D
:1035800000039B8AB3F5807F03D0B3F5007F75D02D
:1035900092E04A4B1A8845F29C13C1F200031B8843
:1035A0009A4240F08180464B1A88464B1B889A42CB
:1035B0007CD1454A454B10461946FFF74DFE45F272
:1035C000A013C1F200034FF400729A8240483F49B1
:1035D0004FF0060205F0A4FE3C4840F26451C1F2EF
:1035E00000014FF0060205F09BFE3A4840F264519C
:1035F000C1F200014FF0060205F092FE45F2A01064
:10360000C1F2000032494FF0060205F089FE45F292
:10361000A013C1F2000345F2A012C1F20002928B86
:10362000DA8445F2A013C1F2000345F2A012C1F200
:103630000002D28B1A8545F2A013C1F2000345F2B5
:103640009C12C1F2000212889A8345F2A013C1F2C3
:10365000000345F29C12C1F200025288DA8345F25F
:10366000A013C1F200034FF4C1629A8143F2201308
:10367000C1F200034FF02A021A8018E00F4B1A889B
:1036800045F29C13C1F200031B889A4211D10C4BE6
:103690001A880C4B1B889A420DD10B4A0B4B1046D3
:1036A0001946FFF7D9FD07E000BF00E000BF00BFEB
:1036B00002E000BF00E000BF08BD00BFC65100101F
:1036C000C85100109E510010BC510010B65100109E
:1036D000C0510010A651001000B583B09E4B1A884F
:1036E00040F64C43C0F201031B889A4212D19B4B17
:1036F0001A889B4B1B889A420CD145F2A010C1F24C
:10370000000040F64441C0F201014FF0060205F00E
:1037100007FE01E1904B1A8845F29C13C1F20003A9
:103720001B8882EA03039AB245F29813C1F20003A0
:103730001B8802EA03039BB2002B0DD1874B1A882A
:10374000884B1B8882EA03039AB2874B1B8802EAE4
:1037500003039BB2002B0ED045F26813C1F20003A5
:103760001A8840F2DC53C1F200031A807F4B804A72
:1037700012881A800AE0784B1A8840F2DC53C1F2B2
:1037800000031A80794B754A12881A8040F2E05380
:10379000C1F200034FF000021A7030E040F2E05333
:1037A000C1F200031B781A4613464FEA4303134441
:1037B0004FEA83031A4640F27C53C1F200031344DC
:1037C000019340F2DC53C1F200031A88019B1B886D
:1037D0009A4207D1654B1A88019B03F102031B88AB
:1037E0009A4214D040F2E053C1F200031B7803F177
:1037F0000103DAB240F2E053C1F200031A7040F262
:10380000E053C1F200031B78072BC7D900E000BFCB
:1038100040F2E053C1F200031B78082B70D145F24F
:10382000A010C1F200004FF0FF014FF0060205F0BA
:103830003FFE4A484FF000014FF0060205F038FE07
:103840004C4840F26451C1F200014FF0060205F00D
:1038500067FD494840F26451C1F200014FF0060291
:1038600005F05EFD454A40F2DC53C1F200031B88BF
:103870001380434B3D4A12881A80424A45F29C13FA
:10388000C1F200031B881380334B364A12881A801A
:1038900045F2A013C1F200034FF480729A8245F200
:1038A000A013C1F200034FF48072DA8145F2A01335
:1038B000C1F200034FF008021A8245F2A013C1F2D0
:1038C00000034FF006029A7445F2A013C1F2000300
:1038D0004FF00402DA7445F2A013C1F200034FF472
:1038E000C1629A8143F23013C1F20003264A1A6082
:1038F00043F22013C1F200034FF02A021A8028E09D
:10390000019B03F1040345F2A010C1F20000194627
:103910004FF0060205F004FD164840F26451C1F272
:1039200000014FF0060205F0FBFC45F2A013C1F2C6
:1039300000034FF008029A8143F22013C1F2000302
:103940001B8803F10E039AB243F22013C1F2000365
:103950001A8003B000BD00BFBE510010C05100105E
:103960004E0C01009E5100109A510010DE0500100F
:103970006A510010A6510010B6510010C651001037
:10398000C8510010BC510010D651001084B00190F5
:1039900000914FF001038DF80F304FF000038DF8C8
:1039A0000F30019B4FF000021A854FF002031846BA
:1039B00004B0704710B584B0019040F20803C1F222
:1039C0000003039319E0039B1B681C68039B1B689F
:1039D0001B68184605F07EFF0346204601991A46EB
:1039E00005F0A8FF0346002B03D1039B1B685B680F
:1039F0000BE0039B03F104030393039B1B68002B61
:103A0000E1D143F68D13C0F20003184604B010BD97
:103A100010B584B00190019B039343F23013C1F2BF
:103A200000031B681C46039800F034FA0346204646
:103A300040F2BA5140F60072C0F2010205F0D4FD26
:103A400003469BB2184604B010BD00BF10B584B049
:103A5000019000914FF001038DF80F30019B1B8DF9
:103A6000002B02D0612B04D01CE0019B4FF06102BF
:103A70001A85019B03F1280400984FF0200105F0FE
:103A80006BFE034603F10103204643F61121C0F209
:103A900000011A46FDF7AEF90346002B02D14FF0A4
:103AA000000309E04FF000038DF80F30019B4FF049
:103AB00000021A854FF00203184604B010BD00BF83
:103AC0002DE9F0458FB00B900B9B0D930D9BB3F838
:103AD000AC304FF0CC0202FB03F243F23813C1F2D8
:103AE000000313440C9343F23013C1F200031B682C
:103AF0001D460C9B9B881846FFF7DCFA03461C46C4
:103B00000C9B1B881846FFF7D5FA03464FEA132390
:103B10009BB29A460C9B1B881846FFF7CBFA0346CC
:103B200003F0FF080C9B5B881846FFF7C3FA0346B7
:103B30004FEA13239BB21F460C9B5B881846FFF786
:103B4000B9FA034603F0FF060C9BDB881846FFF723
:103B5000B1FA03469E460C9B5B7E03F00F0240F2D7
:103B60001803C1F2000353F822C00C9BDB7E1846F9
:103B70000C9B9B7E19460C9B1B8A002B02D04FF09E
:103B80002A0201E04FF020020C9B5B7E03F0100341
:103B9000002B02D04FF0210301E04FF02003CDF8BD
:103BA00000A0CDF8048002970396CDF810E0CDF880
:103BB00014C00690079108920993284640F2BA5122
:103BC00040F60472C0F20102234605F00DFD0346E3
:103BD0009BB218460FB0BDE8F08500BF00B585B0B8
:103BE000019000914FF001038DF80F30019B1B8D68
:103BF000002B02D0AB2B1ED03CE0019B4FF000020B
:103C0000A3F8AC2031E0019BB3F8AC301A4643F284
:103C10003813C1F200034FF0CC0101FB02F2134450
:103C200003F118035B7803F00F03002B14D0019B02
:103C30004FF0AB021A85019B03F12803184643F6A7
:103C4000C121C0F20001019AFDF7D4F80346002B10
:103C500002D14FF0000317E0019BB3F8AC3003F141
:103C600001039AB2019BA3F8AC20019BB3F8AC30DE
:103C7000272BC8D94FF000038DF80F30019B4FF070
:103C800000021A854FF00203184605B000BD00BFC0
:103C900000B585B00190019B039343F23013C1F24C
:103CA00000031B681A46039BB3F8AC304FEA43018C
:103CB00045F26C13C1F200030B441B88104640F21E
:103CC000BA5140F66472C0F2010205F08DFC034661
:103CD0009BB2184605B000BD00B585B001900091BB
:103CE0004FF001038DF80F30019B1B8D002B02D08C
:103CF000C32B0AD028E0019B4FF00002A3F8AC20B0
:103D00001DE0019B4FF0C3021A85019B03F12803BC
:103D1000184643F69141C0F20001019AFDF76AF896
:103D20000346002B02D14FF0000317E0019BB3F8CC
:103D3000AC3003F101039AB2019BA3F8AC20019BC4
:103D4000B3F8AC30152BDCD94FF000038DF80F30F1
:103D5000019B4FF000021A854FF00203184605B090
:103D600000BD00BF84B0019000914FF000038DF8BA
:103D70000F309DF80F20009B13441B78002B0DD0B3
:103D80009DF80F20019B13441B780D2B06D09DF846
:103D90000F20019B13441B780A2B02D14FF0000324
:103DA00015E09DF80F20019B13441A789DF80F1021
:103DB000009B0B441B789A4202D04FF0010306E0AF
:103DC0009DF80F3003F101038DF80F30D1E718464D
:103DD00004B0704700B585B0019000914FF000032A
:103DE000ADF80A3042F23463C0F2010303932DE0D0
:103DF000039B5B6801981946FFF7B4FF0346002B4D
:103E00001BD1039B9A68009B1A60039BDA68009B96
:103E10005A60BDF80A2040F2E453C1F2000333F8BF
:103E2000123003F1010399B240F2E453C1F20003EE
:103E300023F812104FF001030DE0BDF80A3003F132
:103E40000103ADF80A30039B1B680393039B002B0F
:103E5000CED14FF00003184605B000BD82B04FF040
:103E60000003ADF806300FE0BDF8062040F2E45341
:103E7000C1F200034FF0000123F81210BDF8063024
:103E800003F10103ADF80630BDF80630092BEBD97C
:103E900002B0704700B585B001904FF00003ADF857
:103EA0000E3042F23463C0F2010302931AE0029B27
:103EB0005B6801981946FFF755FF0346002B08D1B0
:103EC000BDF80E2040F2E453C1F2000333F8123083
:103ED0000DE0BDF80E3003F10103ADF80E30029B8A
:103EE0001B680293029B002BE1D14FF000031846A0
:103EF00005B000BD00B585B00190019B0393039B05
:103F0000D3F89C2043F23413C1F200031B685B8A90
:103F10009A420ADD43F23413C1F200031B685B8A44
:103F20001A46039BC3F8A02005E0039BD3F89C200E
:103F3000039BC3F8A02043F23013C1F200031968B9
:103F4000039BD3F89820039BD3F8A0300846114672
:103F50001A4605F0E5F9039BD3F8A0309BB218464A
:103F600005B000BD00B585B001904FF001038DF89C
:103F70000F30019B1B8D002B02D0672B04D02EE04D
:103F8000019B4FF067021A85019B03F12803184635
:103F900043F6F561C0F20001019AFCF72BFF0346DE
:103FA000002B02D14FF0000323E0019BD3F89C20AB
:103FB000019BD3F8A030C3EB0202019BC3F89C2005
:103FC000019BD3F89820019BD3F8A0301A44019BA1
:103FD000C3F89820019BD3F89C30002BD0DC4FF025
:103FE00000038DF80F30019B4FF000021A854FF04F
:103FF0000203184605B000BD00B585B001904FF032
:1040000001038DF80F30019B1B8D002B02D0742B08
:1040100004D017E0019B4FF074021A85019B03F155
:104020002801019BD3F89820019BD3F8A0300846C3
:1040300011461A46FCF794FE0346002B02D14FF0BE
:10404000000309E04FF000038DF80F30019B4FF0A3
:1040500000021A854FF00203184605B000BD00BFEC
:1040600000B585B00190019BD3F8A43018464FF0FD
:104070000A0105F071FB034603F101030393019B61
:10408000D3F8A820039B99B2019BD3F8A4309BB22C
:10409000C3EB01039BB2C3EB0202019BC3F8A82050
:1040A000019B039AC3F8A42005B000BD00B585B0FC
:1040B00001904FF001038DF80F30019BB3F84E30A3
:1040C000932B42D0932B03DC002B00F0F380F8E01D
:1040D000962B48D0B42B00F0CE80F2E0019BD3F8B1
:1040E00098301B78252B61D1019BD3F8983003F1D0
:1040F00001031B78212B59D1019BD3F8983003F190
:104100000302019BC3F8A420019BD3F89C30A3F1C8
:104110000302019BC3F8A820019BD3F8A43003F14C
:10412000FF331B783A2B19D1019BD3F8A43003F14C
:104130000102019B03F1980310461946FFF74AFE5E
:10414000019B4FF09302A3F84E200198FFF70AFF5E
:104150000346002B1AD14FF00003BDE0019B4FF046
:104160009602A3F84E20019BD3F8A4301846FFF71F
:1041700021FC0346019AD2F8A420019811469847E1
:104180000346002B02D14FF00003A5E00198FFF792
:1041900067FF019BD3F8A420019BC3F89820019BE3
:1041A000D3F8A820019BC3F89C2084E0019BD3F89E
:1041B0009C2043F23413C1F200031B685B8A9A42CD
:1041C0000ADD43F23413C1F200031B685B8A1A460E
:1041D000019BC3F8A02005E0019BD3F89C20019B24
:1041E000C3F8A020019BD3F898301B78252B0CD165
:1041F000019BD3F8983003F1010318464FF02501D5
:1042000005F0AAFA0346029309E0019BD3F898301F
:1042100018464FF0250105F09FFA03460293029BD2
:10422000002B23D0019BD3F89820029B9A421DD0EB
:10423000029A019BD3F89830C3EB0202019BC3F8AA
:10424000A020019BD3F8A02043F23413C1F2000355
:104250001B685B8A9A4209DB43F23413C1F2000304
:104260001B685B8A1A46019BC3F8A020019B4FF094
:10427000B402A3F84E200198FFF7BEFE0346002BC0
:1042800002D14FF0000327E0019BD3F89820019B57
:10429000D3F8A0301A44019BC3F89820019BD3F8AF
:1042A0009C20019BD3F8A030C3EB0202019BC3F812
:1042B0009C2000E000BF019BD3F89C30002B3FF70F
:1042C0000DAF4FF000038DF80F30019B4FF000024F
:1042D000A3F84E204FF00203184605B000BD00BF02
:1042E00010B584B0019000914FF001038DF80F30AC
:1042F000019B1B8DCE2B00F0A380CE2B0BDCC52B9E
:104300001DD0C52B02DC002B15D047E1C92B39D0BD
:10431000CC2B6CD042E1D22B00F0E380D22B03DC1B
:10432000D02B00F0B68039E1D42B00F00281D62BDF
:1043300000F01B8132E1019B4FF0C5021A85019B01
:1043400003F12804009805F0C5FA034620460099B9
:104350001A46FCF705FD0346002B02D14FF000037F
:1043600026E1019B03F1820318464FF02E0105F070
:1043700071FB03460293029B002B1CD1019B4FF063
:10438000C9021A85019B03F1280440F66460C0F25B
:10439000010005F09FFA0346204640F66461C0F232
:1043A00001011A46FCF7DCFC0346002B40F0F680C6
:1043B0004FF00003FCE040F69060C0F2010002996B
:1043C0004FF0050205F0B6FA0346002B0BD040F67D
:1043D0009860C0F2010002994FF0060205F0AAFAB7
:1043E0000346002B1CD1019B4FF0CC021A85019B88
:1043F00003F1280440F6B850C0F2010005F06AFA53
:104400000346204640F6B851C0F201011A46FCF7B7
:10441000A7FC0346002B40F0C0804FF00003C7E02C
:1044200040F6A860C0F2010002994FF0040205F0C6
:1044300081FA0346002B1CD1019B4FF0CE021A8556
:10444000019B03F1280440F6D450C0F2010005F0AE
:1044500041FA0346204640F6D451C0F201011A4603
:10446000FCF77EFC0346002B40F098804FF00003E1
:104470009EE040F6B060C0F2010002994FF00402E5
:1044800005F058FA0346002B1BD1019B4FF0D002D8
:104490001A85019B03F1280440F60C60C0F201006C
:1044A00005F018FA0346204640F60C61C0F20101FF
:1044B0001A46FCF755FC0346002B6FD14FF0000362
:1044C00076E040F6B860C0F2010002994FF00402B5
:1044D00005F030FA0346002B1BD1019B4FF0D202AE
:1044E0001A85019B03F1280440F62860C0F2010000
:1044F00005F0F0F90346204640F62861C0F20101BC
:104500001A46FCF72DFC0346002B47D14FF0000361
:104510004EE040F6C060C0F2010002994FF0040284
:1045200005F008FA0346002B1BD1019B4FF0D40283
:104530001A85019B03F1280440F64460C0F2010093
:1045400005F0C8F90346204640F64461C0F2010177
:104550001A46FCF705FC0346002B1FD14FF0000361
:1045600026E0019B4FF0D6021A85019B03F1280437
:1045700040F69850C0F2010005F0ACF90346204621
:1045800040F69851C0F201011A46FCF7E9FB0346D8
:10459000002B03D14FF000030AE000BF4FF00003EF
:1045A0008DF80F30019B4FF000021A854FF0020387
:1045B000184604B010BD00BF00B585B001904FF0A3
:1045C00001038DF80F30019BB3F84C30E92B46D036
:1045D000E92B04DC002B0AD0E72B2ED09CE0F12B3A
:1045E0007BD0F42B00F08780ED2B46D094E0019B2C
:1045F00003F18202019B03F1980310461946FFF76D
:10460000E9FB0346002B33D1019B03F1980340F6ED
:10461000D040C0F201001946FFF7DCFB019B03F11B
:104620008203184640F6D041C0F2010105F0F4F8CB
:10463000019B4FF0E702A3F84C20019840F63C5153
:10464000C0F20101FFF74CFE0346002B02D14FF0F0
:1046500000036CE0019B4FF0E902A3F84C200198A5
:10466000FFF780FC0346002B4FD14FF000035EE0C4
:10467000019B4FF0ED02A3F84C20019840F6E84171
:10468000C0F20101FFF72CFE0346002B02D14FF0D0
:1046900000034CE0019B03F1820318464FF02E010A
:1046A00005F05AF803460293029B002B1ED0029895
:1046B00040F69861C0F201014FF0060205F03AF9A8
:1046C0000346002B12D1019B4FF00002A3F84E20AD
:1046D000019B4FF0F102A3F84C200198FFF7E6FC94
:1046E0000346002B10D14FF0000320E0019B4FF058
:1046F000F402A3F84C200198FFF734FC0346002B8A
:1047000003D14FF0000312E000BF43F22C13C1F2BB
:1047100000034FF010021A704FF000038DF80F30B5
:10472000019B4FF00002A3F84C204FF00203184603
:1047300005B000BD00B585B001904FF001038DF8C4
:104740000F30019B9B88B3F5807F11D0B3F5807F3C
:1047500002DC002B08D0C0E0B3F5837F37D0B3F57F
:104760008C7F00F08D80B8E0019B4FF480729A80BE
:10477000019B03F1040318464FF02001FCF7CAFB2C
:104780000346002B02D14FF00003B0E0019B03F180
:104790005003184640F67041C0F201014FF0040288
:1047A00005F0C8F80346002B0DD043F22C13C1F2DC
:1047B00000034FF010021A70019B4FF000029A8024
:1047C0004FF0010393E0019B4FF483729A80019BA9
:1047D00003F1040318464FF02001FCF79BFB03464E
:1047E000002B02D14FF0000381E0019B93F8503081
:1047F0002F2B0DD043F22C13C1F200034FF0100207
:104800001A70019B4FF000029A804FF001036EE096
:10481000019B93F85130202B0CD1019B03F18203B3
:10482000184640F6C441C0F201014FF0140205F0F1
:10483000D5F81AE0019B03F104031846FCF734FB9A
:10484000034603F1FF32019B13444FF0000283F84B
:104850005020019B03F18202019B03F1500310469B
:1048600019464FF0140205F0B9F8019B4FF0010210
:1048700083F8962000E000BF019B4FF48C729A8071
:10488000019B03F1040318464FF00A01FCF742FBB9
:104890000346002B02D14FF0000328E0019B03F1F7
:1048A0005003184640F6DC41C0F201014FF0080207
:1048B00005F040F80346002BDDD1019B03F1040312
:1048C0001846FCF7F1FA0346A3F10202019B1344D8
:1048D0004FF0000283F85020CEE74FF000038DF830
:1048E0000F30019B4FF000029A804FF002031846F0
:1048F00005B000BD00B583B001900198FFF71AFF25
:10490000019B93F89630012B02D10198FFF754FEDA
:1049100003B000BD00B583B043F23413C1F200030D
:104920001B6803F11C03019343F22C13C1F2000333
:104930001B7803F01003002B73D143F22C13C1F248
:1049400000031B7803F02003002B6AD143F22C13E1
:10495000C1F200031B785BB2002B62DB43F22C1325
:10496000C1F200031B7803F04003002B29D0019B08
:1049700003F10402019B03F15003104619464FF066
:104980003102FCF795FB019B03F12802019B03F127
:104990005003104619464FF03102FCF789FB019B8A
:1049A0004FF00002A3F84C20019B4FF0000283F867
:1049B0009620019B4FF000021A700198FFF79AFFB2
:1049C0002FE0019B002B25D043F22C13C1F20003F2
:1049D0001B7803F00803002B12D0019B1B7803F116
:1049E0000103DAB2019B1A70019B1B78132B0CD9BF
:1049F00043F22C13C1F200034FF020021A7005E0BD
:104A0000019B4FF000021A7000E000BF0198FFF711
:104A100071FF06E043F22C13C1F200034FF02002B5
:104A20001A7003B000BD00BF08B54FF4A040FCF7FA
:104A3000C7FE08BD82B001900091FEE7FEE7FEE7E9
:104A4000FEE7FEE7FEE7FEE7FEE7FEE7FEE7FEE73E
:104A500000B583B001900B468DF803300DF10303D0
:104A6000019819464FF001024FF0010302F006FCD5
:104A700003B000BD00B585B001904FF000038DF884
:104A80000F300DF10F03019819464FF001024FF05E
:104A9000010302F077FC9DF80F30184605B000BD09
:104AA00000B585B001900091009B039309E0039B42
:104AB0001B78039A02F10102039201981946FFF74D
:104AC000C7FF039B1B78002BF1D105B000BD00BFD1
:104AD00000B583B00190009101980099FFF7E0FFC5
:104AE000019842F24861C0F20101FFF7D9FF03B01B
:104AF00000BD00BF00B585B001900B468DF80330B6
:104B00009DF803204CF6CD43CCF6CC43A3FB021317
:104B10004FEAD3010B464FEA83030B444FEA4303AA
:104B2000C3EB02038DF80D309DF803204CF6CD4306
:104B3000CCF6CC43A3FB02134FEAD303DAB24CF614
:104B4000CD43CCF6CC43A3FB02134FEAD3010B4673
:104B50004FEA83030B444FEA4303C3EB02038DF890
:104B60000E309DF8032048F21F53C5F2EB13A3FB50
:104B700002134FEA5313DAB24CF6CD43CCF6CC43D2
:104B8000A3FB02134FEAD3010B464FEA83030B4406
:104B90004FEA4303C3EB02038DF80F309DF80F304B
:104BA00003F13003DBB201981946FFF751FF9DF87E
:104BB0000E3003F13003DBB201981946FFF748FFCE
:104BC0009DF80D3003F13003DBB201981946FFF771
:104BD0003FFF05B000BD00BF00B585B001900B469A
:104BE000ADF80230BDF802204CF6CD43CCF6CC43F4
:104BF000A3FB02134FEAD3010B464FEA83030B4496
:104C00004FEA4303C3EB02039BB28DF80B30BDF8B0
:104C100002204CF6CD43CCF6CC43A3FB02134FEA63
:104C2000D3039AB24CF6CD43CCF6CC43A3FB02138C
:104C30004FEAD3010B464FEA83030B444FEA430389
:104C4000C3EB02039BB28DF80C30BDF8022048F292
:104C50001F53C5F2EB13A3FB02134FEA53139AB28F
:104C60004CF6CD43CCF6CC43A3FB02134FEAD30161
:104C70000B464FEA83030B444FEA4303C3EB0203A3
:104C80009BB28DF80D30BDF8022044F6D353C1F22B
:104C90006203A3FB02134FEA93139AB24CF6CD437F
:104CA000CCF6CC43A3FB02134FEAD3010B464FEAE9
:104CB00083030B444FEA4303C3EB02039BB28DF81B
:104CC0000E30BDF8022041F25973CDF2B713A3FBA9
:104CD00002134FEA53339AB24CF6CD43CCF6CC4391
:104CE000A3FB02134FEAD3010B464FEA83030B44A5
:104CF0004FEA4303C3EB02039BB28DF80F309DF8DC
:104D00000F3003F13003DBB201981946FFF7A0FE24
:104D10009DF80E3003F13003DBB201981946FFF71E
:104D200097FE9DF80D3003F13003DBB20198194670
:104D3000FFF78EFE9DF80C3003F13003DBB20198D3
:104D40001946FFF785FE9DF80B3003F13003DBB207
:104D500001981946FFF77CFE05B000BD00B587B08D
:104D60000190009100994CF6CD43CCF6CC43A3FBC7
:104D700001234FEAD30213464FEA830313444FEA59
:104D80004303C3EB010213468DF80E30009A4CF634
:104D9000CD43CCF6CC43A3FB02134FEAD3014CF630
:104DA000CD43CCF6CC43A3FB01234FEAD3021346F9
:104DB0004FEA830313444FEA4303C3EB0102134654
:104DC0008DF80F30009A48F21F53C5F2EB13A3FB86
:104DD00002134FEA53114CF6CD43CCF6CC43A3FB60
:104DE00001234FEAD30213464FEA830313444FEAE9
:104DF0004303C3EB010213468DF81030009A44F6CA
:104E0000D353C1F26203A3FB02134FEA93114CF692
:104E1000CD43CCF6CC43A3FB01234FEAD302134688
:104E20004FEA830313444FEA4303C3EB01021346E3
:104E30008DF81130009A41F25973CDF2B713A3FBEC
:104E400002134FEA53314CF6CD43CCF6CC43A3FBCF
:104E500001234FEAD30213464FEA830313444FEA78
:104E60004303C3EB010213468DF81230009B4FEA57
:104E7000531245F6C523C0F67C23A3FB02134FEA69
:104E8000D3114CF6CD43CCF6CC43A3FB01234FEA20
:104E9000D30213464FEA830313444FEA4303C3EBA1
:104EA000010213468DF81330009A4DF68363C4F265
:104EB0001B33A3FB02134FEA93414CF6CD43CCF6D0
:104EC000CC43A3FB01234FEAD30213464FEA8303EB
:104ED00013444FEA4303C3EB010213468DF8143029
:104EE000009A4CF66B23C6F65F33A3FB02134FEA1E
:104EF00093514CF6CD43CCF6CC43A3FB01234FEAB0
:104F0000D30213464FEA830313444FEA4303C3EB30
:104F1000010213468DF81530009A43F68933C5F225
:104F2000E653A3FB02134FEA53614CF6CD43CCF694
:104F3000CC43A3FB01234FEAD30213464FEA83037A
:104F400013444FEA4303C3EB010213468DF81630B6
:104F5000009B4FEA532244F68333C0F20403A3FBC1
:104F600002134FEAD3114CF6CD43CCF6CC43A3FB4E
:104F700001234FEAD30213464FEA830313444FEA57
:104F80004303C3EB010213468DF817309DF8173029
:104F900003F13003DBB201981946FFF759FD9DF884
:104FA000163003F13003DBB201981946FFF750FDCC
:104FB0009DF8153003F13003DBB201981946FFF775
:104FC00047FD9DF8143003F13003DBB20198194618
:104FD000FFF73EFD9DF8133003F13003DBB201987B
:104FE0001946FFF735FD9DF8123003F13003DBB2AF
:104FF00001981946FFF72CFD9DF8113003F130039D
:10500000DBB201981946FFF723FD9DF8103003F13C
:105010003003DBB201981946FFF71AFD9DF80F30F7
:1050200003F13003DBB201981946FFF711FD9DF83B
:105030000E3003F13003DBB201981946FFF708FD8B
:1050400007B000BD00B585B001900B468DF8033068
:10505000019842F24C61C0F20101FFF721FD4FF0CF
:1050600001038DF80F309DF803209DF80F304FEAB3
:10507000830342FA03F3DBB203F00F038DF80E3023
:105080009DF80E30092B05D99DF80E3003F137033A
:10509000DBB204E09DF80E3003F13003DBB201987F
:1050A0001946FFF7D5FC9DF80F30002B0CBF0023ED
:1050B0000123DBB29DF80F2002F1FF328DF80F20A3
:1050C000002BD0D105B000BD00B585B001900B46D6
:1050D000ADF80230019842F24C61C0F20101FFF7D5
:1050E000DFFC4FF003038DF80F30BDF802209DF870
:1050F0000F304FEA830342FA03F3DBB203F00F03EE
:105100008DF80E309DF80E30092B05D99DF80E3024
:1051100003F13703DBB204E09DF80E3003F13003F6
:10512000DBB201981946FFF793FC9DF80F30002B76
:105130000CBF00230123DBB29DF80F2002F1FF32E8
:105140008DF80F20002BD0D105B000BD00B585B083
:1051500001900091019842F24C61C0F20101FFF709
:105160009FFC4FF007038DF80F309DF80F304FEA8A
:105170008303009A22FA03F3DBB203F00F038DF8E6
:105180000E309DF80E30092B05D99DF80E3003F135
:105190003703DBB204E09DF80E3003F13003DBB2DD
:1051A00001981946FFF754FC9DF80F30002B0CBFF7
:1051B00000230123DBB29DF80F2002F1FF328DF8AE
:1051C0000F20002BD1D105B000BD00BF00B585B0C8
:1051D0004FF001038DF802304FF000038DF80430DA
:1051E0004FF000038DF803304FF002038DF80130CB
:1051F0004FF000038DF800306B46184601F0F8FBC5
:105200004FF003038DF801306B46184601F0F0FBB8
:1052100002AB184601F0AAFF4FF4E133029302AB50
:105220004CF20000C4F20000194601F091FD4CF26E
:105230000000C4F200004FF0010102F0A5FC45F2AD
:10524000A473C1F2000344F6A122C0F200021A6066
:1052500045F2AC73C1F2000344F6D122C0F2000261
:105260001A6045F2B073C1F2000344F65122C0F255
:1052700000021A6045F2B473C1F2000345F2450220
:10528000C0F200021A6045F2B873C1F2000345F2A1
:10529000C902C0F200021A6045F29C73C1F2000319
:1052A00045F24D12C0F200021A6045F29473C1F249
:1052B000000344F6F522C0F200021A6045F2A07322
:1052C000C1F2000344F6D932C0F200021A6045F27E
:1052D0009873C1F2000344F65D52C0F200021A60F6
:1052E00045F2A873C1F2000344F67522C0F2000231
:1052F0001A6005B000BD00BF82B04FF000030193FB
:1053000039E00199019A13464FEA430313444FEAE7
:1053100043231A4640F25C63C1F2000313441A4669
:1053200040F2F853C1F2000343F83120019B40F2F0
:10533000F852C1F200024FEAC303134440F2FF5295
:10534000C8F200025A60019A40F21863C1F20003E9
:105350004FF0000143F83210019B40F21862C1F295
:1053600000024FEAC30313444FF000025A60019B4E
:1053700003F101030193019B032BC2D94FF0A0421B
:1053800040F2F853C1F20003C2F808314FF0A042D6
:1053900040F21863C1F20003C2F80C314FF0A04391
:1053A0004FF00302C3F810214FF0A0434FF000026A
:1053B000C3F8182102B0704782B04FF00003019388
:1053C0002CE00199019A13464FEA430313444FEA34
:1053D00043231A4641F65C63C1F2000313441A46A4
:1053E00040F23863C1F2000343F83120019B40F2E0
:1053F0003862C1F200024FEAC30313444FF00002C7
:105400005A60019A40F25063C1F200034FF000016C
:1054100043F82210019B03F101030193019B022B2E
:10542000CFD94FF0A04240F23863C1F20003C2F876
:105430001C314FF0A04240F25063C1F20003C2F8A9
:1054400020314FF0A0434FF00202C3F824214FF067
:10545000A0434FF00002C3F8282102B0704700BFFC
:1054600084B001900B46ADF802304FF0A043019A92
:1054700042F480729A624FF0A043BDF80220DA62D3
:105480004FF0000303934FF0000303930DE04FF040
:10549000A0435B6B03F00103002B02D14FF000032C
:1054A0000CE0039B03F101030393039A4FF6FF7390
:1054B000C0F204039A42EAD94FF0FF33184604B011
:1054C000704700BF84B001904FF0A043019A42F4AE
:1054D00080729A624FF0A0434FF001025A624FF07F
:1054E000000303934FF00003039313E04FF0A04336
:1054F0005B6B03F00103002B08D14FF0A0434FF08A
:1055000000025A624FF0A0431B6B0CE0039B03F1B7
:1055100001030393039A4FF6FF73C0F204039A4208
:10552000E4D94FF0FF33184604B0704782B00190C1
:105530004FF0A043019A02F1050212784FEA0221CE
:10554000019A02F10402127841EA02021A644FF051
:10555000A043019A02F1030212784FEA0221019A54
:1055600002F10202127841EA02025A644FF0A043AB
:10557000019A02F1010212784FEA0221019A12788F
:1055800041EA02029A6402B0704700BF8AB00190FB
:1055900000914FF0FF3305934FF00003029389E031
:1055A000019B1B788DF81330019B03F101030193DC
:1055B0004FF00003039376E0059B4FEA23729DF8BA
:1055C00013304FEAD303DBB282EA030303F0010393
:1055D000DBB2002B05D041F6B753C0F2C1430993AB
:1055E00002E04FF000030993059B4FEA63729DF8B8
:1055F00013304FEA9303DBB282EA030303F00103A3
:10560000DBB2002B05D043F66E33C0F6821308934D
:1056100002E04FF000030893059B4FEAA3729DF848
:1056200013304FEA5303DBB282EA030303F00103B2
:10563000DBB2002B05D047F2DC63C1F204330793E1
:1056400002E04FF000030793059B4FEAE3729DF8D9
:10565000133082EA030303F00103DBB2002B05D011
:105660004EF6B853C2F20863069302E04FF000030F
:105670000693059B4FEA0312099B82EA0302089BEB
:1056800082EA0302079B82EA0302069B82EA030383
:1056900005939DF813304FEA13138DF81330039BD5
:1056A00003F101030393039B012B85DD029B03F1AF
:1056B00001030293029A009B9A42FFF671AF059B89
:1056C00018460AB0704700BF00B587B001904FF090
:1056D00080404FF0010103F0F3F84FF0A0434FF486
:1056E0004F421A604FF0A0434FF07802C3F80021F8
:1056F0004FF06403049303E0049B03F1FF3304932E
:10570000049B002BF8D14FF0A0434FF002021A6027
:105710004FF0A0434FF030025A604FF0A0434FF4D7
:10572000C0625A6140F23C03C1F200031A684CF6B1
:105730006B23C6F65F33A3FB02134FEA13530593A3
:105740004FF0000304930DE0049A42F25063C0F25C
:1057500001039B5C1A46059B9A4207DA049B03F1FE
:1057600001030493049B062BEED900E000BF049BC9
:1057700003F1010304934FF0A043049A02F00F02D7
:105780004FEA820242F400421A624FF0A0434FF007
:10579000A042126A22F400421A624FF0A04343F280
:1057A0000F721A614FF0A0434FF01202DA604FF00F
:1057B000A0434FF41072C3F800214FF0A0434FF400
:1057C00000629A614FF06403049303E0049B03F1C9
:1057D000FF330493049B002BF8D14FF0A0434FF00C
:1057E00000029A614FF000004FF40041FFF738FECD
:1057F0004FF48013049314E04FF00000FFF762FEB3
:1058000003460393039B03F40843002B0DD0049B32
:10581000002B02D14FF0000342E0049B03F1FF3361
:105820000493049B002BE7D100E000BF019B1B68A1
:10583000184600F081F80346002B02DA4FF000030F
:105840002EE0019B5B681846FFF770FEFFF754FDE2
:10585000FFF7B2FD4FF0A0434FF02602C3F800223D
:105860004FF0A0434FF08802C3F8E42F4FF0A0435D
:105870004FF6FF72C3F8E82F4FF0A0434FF0A0425D
:10588000D2F8002142F00302C3F800214FF0A043F8
:105890004FF0A042126842F001021A604FF001037B
:1058A000184607B000BD00BF08B54FF0A0434FF049
:1058B0000002C3F8E42F4FF0A04343F2FF02C3F805
:1058C000E82F4FF080404FF0000102F0F9FF08BDD3
:1058D00000B585B001904FF00100FFF7F3FD0346DE
:1058E0000293019B012B0DD0012B02D3022B12D06E
:1058F0001AE0029B03F00403002B0CBF00230123DA
:10590000039314E0029B03F4C043002B0CBF00235D
:10591000012303930BE0029B03F4A043002B0CBF75
:1059200000230123039302E04FF0FF330393039B13
:10593000184605B000BD00BF00B587B001904FF01C
:105940000200FFF7BFFD034602934FF00300FFF78D
:10595000B9FD03460393029B4FEA0342039B42EACD
:10596000030241F21353C0F222039A4260D1019B19
:10597000042B54D801A252F823F000BF9159000023
:10598000E7590000F5590000035A0000115A0000C1
:105990004FF000004FF44051FFF762FD4FF0000060
:1059A0004FF48051FFF75CFD4FF48013049316E031
:1059B0004FF00100FFF786FD03460593059B03F0BA
:1059C0002003002B01D000BF2CE0049B002B02D150
:1059D0004FF0FF3334E0049B03F1FF330493049B47
:1059E000002BE5D11EE04FF000004FF48071FFF76F
:1059F00037FD17E04FF000004FF00001FFF730FDDA
:105A000010E04FF000004FF40451FFF729FD09E0CA
:105A10004FF000004FF40051FFF722FD02E04FF07D
:105A2000FF330DE000F010F80346002B03DB05E028
:105A30004FF0FF3304E04FF0FF3301E04FF000037D
:105A4000184607B000BD00BF00B583B04FF4801307
:105A5000019314E04FF00100FFF734FD034600937B
:105A6000009B03F00403002B0DD1019B002B02D1FE
:105A70004FF0FF333CE0019B03F1FF330193019BA7
:105A8000002BE7D100E000BF009B03F4A043002BF4
:105A900017D04FF0A0434FF0A042526842F00102ED
:105AA0005A604FF0A0434FF0A042D2F8002142F4D8
:105AB0008062C3F800214FF0A0434FF015029A60B6
:105AC00004E04FF0A0434FF012029A60009B03F4F1
:105AD000C043002B05D14FF0A0434FF000029A6164
:105AE00004E04FF0A0434FF480729A614FF000033E
:105AF000184603B000BD00BF00B587B001900B464B
:105B00008DF8033001984FF00601FFF73FFD034683
:105B10000593059B4FEAE35303F03F030593059B71
:105B20001F2B04DD40F21423C5F2000303E040F212
:105B30001023C5F200030393059B1F2B03DD059B78
:105B4000A3F1200300E0059B04939DF80330012B93
:105B50000BD1039B1A68049B4FF0010101FA03F378
:105B600042EA0302039B1A600CE0039B1A68049B41
:105B70004FF0010101FA03F36FEA030302EA0302A3
:105B8000039B1A604FF0A0434FF0A042D2F80021CF
:105B900022F08002C3F8002107B000BD82B001905E
:105BA0000B468DF803309DF80330012B0BD14FF0DD
:105BB000A0434FF0A042D2F80012019A41EA02023B
:105BC000C3F800220CE04FF0A0434FF0A042D2F8FF
:105BD0000012019A6FEA020201EA0202C3F80022EF
:105BE00002B0704782B001904FF0A043D3F8042276
:105BF000019B02EA0303002B07D04FF0A043019A58
:105C0000C3F808224FF0010301E04FF000031846EB
:105C100002B0704786B001904FF0A043D3F828310E
:105C20000293019B5B680493029A40F23863C1F2CD
:105C3000000353F832300593019B1B6803F1030303
:105C40004FEA930303930FE0049B1A68059B1A60C5
:105C5000059B03F104030593049B03F104030493E0
:105C6000039B03F1FF330393039B002BECD1029BB7
:105C7000019A126802F1FF3242F0404140F238626C
:105C8000C1F200024FEAC3031344596006B07047E3
:105C900086B001904FF0A043D3F818310293019BD6
:105CA0005B680493029A40F2F853C1F2000353F880
:105CB00032300593019B5B68002B1AD0019B1B6857
:105CC00003F103034FEA930303930FE0059B1A6864
:105CD000049B1A60049B03F104030493059B03F1E6
:105CE00004030593039B03F1FF330393039B002BF2
:105CF000ECD106B0704700BF82B001900B468DF822
:105D000003309DF80330012B0BD14FF0A0434FF02F
:105D1000A042D2F8E41F019A41EA0202C3F8E42F3C
:105D20000CE04FF0A0434FF0A042D2F8E41F019ADC
:105D30006FEA020201EA0202C3F8E42F02B07047E0
:105D400082B001904FF0A043D3F8E02F019B02EA0C
:105D50000303002B07D04FF0A043019AC3F8E82FAC
:105D60004FF0010301E04FF00003184602B0704706
:105D70004FF0A043D3F818214FF0A043D3F81431CB
:105D80009A4202D04FF0010301E04FF000031846A1
:105D9000704700BF82B04FF0A043D3F82C3103F11D
:105DA000FF3301934FF0A043D3F82821019B9A427F
:105DB00002D14FF0000301E04FF00103184602B09A
:105DC000704700BF84B001904FF0A043D3F8183162
:105DD0000393039A40F21863C1F2000353F8322090
:105DE000019B02EA0303002B0CBF0023012318468A
:105DF00004B0704782B04FF0A043D3F8183101933C
:105E0000019A40F21863C1F2000353F832304FEAAE
:105E100043534FEA5353184602B0704782B04FF0D5
:105E2000A043D3F818310193019B03F101030193BF
:105E3000019B042B02D14FF0000301934FF0A043CC
:105E4000019AC3F8182102B0704700BF82B04FF02A
:105E5000A043D3F828310193019B03F1010301937F
:105E6000019B032B02D14FF0000301934FF0A0439D
:105E7000019AC3F8282102B0704700BF84B00346DE
:105E80008DF807304FF0000303939DF80730042B83
:105E900029D801A252F823F0AD5E0000B95E0000DF
:105EA000C55E0000D15E0000DD5E00004CF2000324
:105EB000C2F20903039316E04CF22003C2F2090375
:105EC000039310E04CF24003C2F2090303930AE08B
:105ED0004CF26003C2F20903039304E04CF2800326
:105EE000C2F209030393039B184604B0704700BF36
:105EF00084B003468DF807304FF0000303939DF8FC
:105F00000730042B29D801A252F823F0215F0000AA
:105F10002D5F0000395F0000455F0000515F000009
:105F20004CF20003C2F20903039316E04CF2200383
:105F3000C2F20903039310E04CF24003C2F20903DA
:105F400003930AE04CF26003C2F20903039304E0F6
:105F50004CF28003C2F209030393039B184604B07A
:105F6000704700BF84B003468DF807304FF0000340
:105F700003939DF80730042B29D801A252F823F08F
:105F8000955F0000A15F0000AD5F0000B95F0000F9
:105F9000C55F00004CF20003C2F20903039316E050
:105FA0004CF22003C2F20903039310E04CF24003C9
:105FB000C2F2090303930AE04CF26003C2F2090340
:105FC000039304E04CF28003C2F209030393039BA2
:105FD000184604B0704700BF00B587B00291134661
:105FE00002468DF80F208DF807309DF80F301846C7
:105FF000FFF744FF03460593059B002B14D09DF843
:106000000730002B07D0059B1A68029B42EA030267
:10601000059B1A6008E0059B1A68029B6FEA030360
:1060200002EA0302059B1A6007B000BD00B585B007
:10603000034600918DF807309DF807301846FFF7AA
:106040001DFF03460393039B002B02D0039B009A82
:106050009A6105B000BD00BF00B585B00346009150
:106060008DF807309DF807301846FFF707FF034605
:106070000393039B002B02D0039B009ADA6105B0C7
:1060800000BD00BF00B585B003468DF807309DF810
:1060900007301846FFF7F2FE03460393039B002BDD
:1060A00002D0039B5B6901E04FF00003184605B086
:1060B00000BD00BF84B00291134602468DF80F2048
:1060C0008DF807309DF80F30002B0AD19DF807306E
:1060D000002B06D148F28003C4F20203029A1A612F
:1060E0002EE09DF80F30022B0AD19DF80730002BCF
:1060F00006D148F28003C4F20203029A1A631FE039
:106100009DF80F30002B0AD19DF80730012B06D1E6
:1061100048F28003C4F20203029A5A6110E09DF82B
:106120000F30022B0BD19DF80730012B07D148F21D
:106130008003C4F20203029A5A6300BF00E0FEE744
:1061400004B0704784B00291134602468DF80F20C8
:106150008DF807309DF80F30002B0FD19DF80730D8
:10616000002B0BD148F28003C4F202035A68029B51
:1061700022FA03F3DBB203F001033CE09DF80F3099
:10618000022B0FD19DF80730002B0BD148F2800372
:10619000C4F202035A6A029B22FA03F3DBB203F051
:1061A000010328E09DF80F30002B0FD19DF8073038
:1061B000012B0BD148F28003C4F202039A68029BC0
:1061C00022FA03F3DBB203F0010314E09DF80F3071
:1061D000022B0FD19DF80730012B0BD148F2800321
:1061E000C4F202039A6A029B22FA03F3DBB203F0C1
:1061F000010300E0FEE7184604B0704782B0034692
:1062000000918DF807309DF80730002B06D148F239
:106210008003C4F20203009ADA600BE09DF80730B5
:10622000022B06D148F28003C4F20203009ADA621C
:1062300000E0FEE702B0704700B585B0029113465A
:1062400002468DF80F208DF807309DF80F209DF83D
:106250000730104602991A46FFF7BEFE05B000BD92
:1062600000B583B0034600918DF807309DF80730E4
:1062700018460099FFF7DAFE03B000BD00B583B001
:10628000034600918DF807309DF8073018460099B5
:10629000FFF7E2FE03B000BD00B583B003468DF802
:1062A00007309DF807301846FFF7ECFE0346184606
:1062B00003B000BD00B585B00291134602468DF8CB
:1062C0000F208DF807309DF80F209DF807301046FD
:1062D00002991A46FFF7EEFE05B000BD00B585B085
:1062E0000291134602468DF80F208DF807309DF875
:1062F0000F209DF80730104602991A46FFF722FF3B
:106300000346184605B000BD00B583B003460091B2
:106310008DF807309DF8073018460099FFF76EFF9B
:1063200003B000BD00B587B00291134602468DF858
:106330000F208DF807309DF80F301846FFF79EFDAF
:1063400003460593059B002B14D09DF80730002BC6
:1063500007D0059B1A69029B42EA0302059B1A615A
:1063600008E0059B1A69029B6FEA030302EA030235
:10637000059B1A6107B000BD00B585B08DF8070018
:106380008DF80610ADF804208DF803309DF8073025
:106390001846FFF7ADFD03460393039B002B40D047
:1063A0009DF80330002B19D09DF80630002B0AD041
:1063B000039B5B889AB2BDF8043042EA03039AB2A9
:1063C000039B5A802DE0039B1B889AB2BDF80430D2
:1063D00042EA03039AB2039B1A8022E09DF806303A
:1063E000002B0FD0039B5B889BB21A46BDF804308C
:1063F0006FEA03039BB202EA03039BB29AB2039BC8
:106400005A800EE0039B1B889BB21A46BDF80430ED
:106410006FEA03039BB202EA03039BB29AB2039BA7
:106420001A8005B000BD00BF00B585B08DF807002B
:106430008DF80610ADF804208DF803309DF8073074
:106440001846FFF755FD03460393039B002B40D0EE
:106450009DF80330002B19D09DF80630002B0AD090
:10646000039B5B8A9AB2BDF8043042EA03039AB2F6
:10647000039B5A822DE0039B1B8A9AB2BDF804301D
:1064800042EA03039AB2039B1A8222E09DF8063087
:10649000002B0FD0039B5B8A9BB21A46BDF80430D9
:1064A0006FEA03039BB202EA03039BB29AB2039B17
:1064B0005A820EE0039B1B8A9BB21A46BDF8043039
:1064C0006FEA03039BB202EA03039BB29AB2039BF7
:1064D0001A8205B000BD00BF00B585B01346024664
:1064E0008DF807200A468DF80620ADF804309DF897
:1064F00007301846FFF7FCFC03460393039B002B71
:106500000CD09DF80630002B04D0039BBDF804206E
:106510005A8303E0039BBDF804201A8305B000BD35
:1065200000B585B0134602468DF807200A468DF85F
:106530000620ADF804309DF807301846FFF7D8FC68
:1065400003460393039B002B0CD09DF80630002BD1
:1065500004D0039BBDF80420DA8303E0039BBDF85D
:1065600004209A8305B000BD00B585B002460B46F5
:106570008DF807208DF806309DF807301846FFF794
:10658000B7FC03460393039B002B0BD09DF806300A
:10659000002B03D0039BDB8A9BB205E0039B9B8A05
:1065A0009BB201E04FF00003184605B000BD00BFEC
:1065B00000B585B08DF807008DF806108DF8052020
:1065C0008DF804309DF807301846FFF7CBFC0346E2
:1065D0000393039B002B2FD09DF80430002B12D087
:1065E0009DF80630032B26D89DF806309DF806202E
:1065F00003998A5CD1B29DF8052041EA0202D1B22A
:10660000039AD15418E09DF80630032B14D89DF856
:1066100006309DF8062003998A5CD2B211469DF897
:1066200005206FEA0202D2B201EA0202D2B2D1B26E
:10663000039AD15400E000BF05B000BD00B585B09D
:106640008DF807008DF806108DF805208DF80430C0
:106650009DF807301846FFF785FC03460393039B1C
:10666000002B33D09DF80430002B14D09DF8063059
:10667000032B2AD89DF806109DF80620039B13448F
:106680001B7CDAB29DF8053042EA0303DAB2039BC1
:106690000B441A741AE09DF80630032B16D89DF8A7
:1066A00006109DF80620039B13441B7CDBB21A46A0
:1066B0009DF805306FEA0303DBB202EA0303DBB2A5
:1066C000DAB2039B0B441A7400E000BF05B000BDB2
:1066D00000B585B0134602468DF807200A468DF8AE
:1066E00006208DF805309DF807301846FFF73AFC74
:1066F00003460393039B002B0AD09DF80630032B1F
:1067000006D89DF80620039B13449DF805201A76B1
:1067100005B000BD00B585B0134602468DF80720D0
:106720000A468DF806208DF805309DF8073018468A
:10673000FFF718FC03460393039B002B0AD09DF838
:106740000630032B06D89DF80620039B13449DF8C2
:1067500005201A7705B000BD00B585B002460B468E
:106760008DF807208DF806309DF807301846FFF7A2
:10677000F9FB03460393039B002B0AD09DF80630D8
:10678000032B06D89DF80620039B13441B7DDBB228
:1067900001E04FF00003184605B000BD86B0134677
:1067A00002468DF807200A468DF806208DF8053040
:1067B0009DF8063003939DF807304FEA4303049396
:1067C0004CF20003C4F202030593039B0F2B07D97D
:1067D000039BA3F110030393049B03F101030493B0
:1067E000049B4FEA8302059B1344049A4FEA8201FB
:1067F000059A0A441168039A4FEA42024FF00300D7
:1068000000FA02F26FEA020201EA02021A60049B35
:106810004FEA8302059B1344049A4FEA8201059ACA
:106820000A4411689DF80500039A4FEA420200FAF3
:1068300002F241EA02021A6006B0704786B01346BF
:1068400002468DF807200A468DF806208DF805309F
:106850009DF8063003939DF807304FEA43030493F5
:106860004CF24003C4F202030593039B0F2B07D99C
:10687000039BA3F110030393049B03F1010304930F
:10688000049B4FEA8302059B1344049A4FEA82015A
:10689000059A0A441168039A4FEA42024FF0030036
:1068A00000FA02F26FEA020201EA02021A60049B95
:1068B0004FEA8302059B1344049A4FEA8201059A2A
:1068C0000A4411689DF80500039A4FEA420200FA53
:1068D00002F241EA02021A6006B0704784B0134621
:1068E00002468DF807200A468DF806208DF80530FF
:1068F0004CF26803C4F2020303939DF80530012BA8
:1069000016D19DF807304FEA8302039B13449DF88C
:1069100007204FEA8201039A0A4411689DF8062075
:106920004FF0010000FA02F241EA02021A6017E099
:106930009DF807304FEA8302039B13449DF807201C
:106940004FEA8201039A0A4411689DF806204FF02D
:10695000010000FA02F26FEA020201EA02021A6082
:1069600004B0704782B003468DF807309DF80730B9
:10697000012B0CD14CF20003C4F202034CF20002D2
:10698000C4F20202926A42F008029A620FE09DF895
:106990000730002B0BD14CF20003C4F202034CF27F
:1069A0000002C4F20202926A22F008029A6202B065
:1069B000704700BF84B002460B468DF807208DF863
:1069C00006309DF80730012B02D14FF005030393E9
:1069D0009DF80630002B02D14FF00A0303934CF2CE
:1069E0000003C4F20203039ADA6704B0704700BFE1
:1069F00000B583B00190019B1978019B5A78019BE7
:106A00009B78084611461A46FFF7C8FE019B197885
:106A1000019B5A78019BDB78084611461A46FFF71E
:106A20000DFF019B1978019B5A78019B1B79084641
:106A300011461A46FFF752FF03B000BD2DE9F04F93
:106A400095B0039002914FF000038DF81730039A30
:106A50004CF20003C4F200039A4206D14FF0060044
:106A600001F0FAFE0346069328E0039A40F2000381
:106A7000C4F201039A4206D14FF0080001F0ECFE87
:106A8000034606931AE0039A48F20003C4F209038E
:106A90009A4206D14FF0300001F0DEFE0346069325
:106AA0000CE0039A4CF20003C4F209039A4205D1A8
:106AB0004FF0320001F0D0FE034606934FF0FF3353
:106AC00012934FF0000309934FF000030A934FF025
:106AD00000024FF00003CDE90C234FF001030893AF
:106AE00074E04FF00003079363E0069B1A464FF0F3
:106AF00000034FEA12114FEA037541EA05054FEA18
:106B00000274089B1A464FF0000302FB05F104FBD8
:106B100003F00144A4FB022319440B46089807998B
:106B20000144029800FB01F18A464FF0000BCDE9C9
:106B300000AB10461946DDE9002301F03DFF024697
:106B40000B46CDE90E230E9B11930F9B9A464FF0F7
:106B5000000B53460B93119BB3F1004F07D9119BC8
:106B6000C3F1000311930B9B03F101030B930B9BE8
:106B7000002B17D00B9BB3F5803F15D8119A129BB1
:106B80009A4212D2119B12930B9B1A464FF00003AC
:106B9000CDE90C23079B0993089B0A93129B002BBA
:106BA0000CD002E000BF00E000BF079B03F101032F
:106BB0000793079A089B9A4297D300E000BF129B65
:106BC000002B07D0089B03F101030893089B0F2BB0
:106BD00087D900E000BFDDE90C2352EA030B02D1A4
:106BE0004FF00003AFE0069B4FEA13130A9A02FB33
:106BF00003F31C464FF000050A9A099B13441A46FA
:106C00004FF000030C9903FB01F10D9802FB00F01B
:106C100001440C98A0FB022319440B462046294648
:106C200001F0CAFE02460B4613461393029A139BC9
:106C30009A4205D9029A139BC3EB0203129304E014
:106C4000139A029BC3EB02031293129B4FF0640250
:106C500002FB03F2029BB2FBF3F31293129B022B93
:106C60006FD8039A40F20003C4F201039A4232D172
:106C7000039A039B1B7BDBB26FEA43636FEA5363A8
:106C8000DBB21373039B0D9A4FEA02620C994FEA31
:106C9000112842EA08080D9A4FEA12295FFA88F291
:106CA0001A71039B9DF830201A70039A039B1B7B7B
:106CB000DBB203F07F031373039B0A9A4FEA0212BD
:106CC00002F0FF01099A02F00F0241EA020202F00B
:106CD000FF029A6231E0039B1B7BDBB26FEA4363E6
:106CE0006FEA5363DAB2039B1A730D9B4FEA036397
:106CF0000C9A4FEA122643EA06060D9B4FEA132729
:106D0000F2B2039B1A719DF83020039B1A70039B0B
:106D10001B7BDBB203F07F03039A13730A9BDBB286
:106D20004FEA0313DAB2099BDBB203F00F0342EA26
:106D30000303DAB2039B83F828204FF001038DF898
:106D400017309DF81730184615B0BDE8F08F00BF1A
:106D500000B585B001900091019A4CF20003C4F295
:106D600000039A421CD0019A40F20003C4F20103CE
:106D70009A4215D0019A48F20003C4F209039A42DC
:106D80000ED0019A4CF20003C4F209039A4207D0D4
:106D900042F25860C0F201004FF0CA01F9F7B6FCA8
:106DA000009B5B79002B13D0009B5B79012B0FD0EC
:106DB000009B5B79022B0BD0009B5B79032B07D0E8
:106DC00042F25860C0F201004FF0CB01F9F79EFC8F
:106DD000009B9B79002B0BD0009B9B79012B07D04C
:106DE00042F25860C0F201004FF0CC01F9F78EFC7E
:106DF000009B1B79002B17D0009B1B79012B13D014
:106E0000009B1B79022B0FD0009B1B79032B0BD00F
:106E1000009B1B79042B07D042F25860C0F201009E
:106E20004FF0CD01F9F772FC019A4CF20003C4F265
:106E300000039A4205D14FF008004FF0010101F024
:106E40003FFD019A40F20003C4F201039A4205D1CA
:106E50004FF010004FF0010101F032FD019A48F2AD
:106E60000003C4F209039A4205D14FF080704FF03D
:106E7000010101F025FD019A4CF20003C4F209035F
:106E80009A4205D14FF000704FF0010101F018FD5A
:106E9000019A40F20003C4F201039A424DD1019BD2
:106EA0004FF007021A72019B4FF000021A7203E0C2
:106EB000019B1B78DBB20393019B1B7DDBB203F0CC
:106EC0000103DBB2002BF3D1019B6FF07F0283F84B
:106ED0003020019B1B7DDBB203F02003002BF8D098
:106EE000019B4FF0000283F83020019B4FF000021D
:106EF0005A60019B4FF000021A73019B4FF0000291
:106F00001A62019B4FF000021A74019B4FF00002BD
:106F100083F84C20019B4FF0000283F85420019B22
:106F20004FF0000283F85020019B1B7EDBB20393DD
:106F3000019B1B7DDBB2039335E0019B4FF0070201
:106F40001A72019B4FF000021A7203E0019B1B783A
:106F5000DBB20393019B1B7DDBB203F00103DBB2C9
:106F6000002BF3D1019B6FF07F0283F83020019B4F
:106F70001B7DDBB203F02003002BF8D0019B4FF008
:106F8000000283F83020019B4FF000025A60019B01
:106F90004FF000021A73019B4FF000021A62019B2E
:106FA0001B7DDBB20393019A4CF20003C4F2090388
:106FB0009A4204D1019B4FF0000283F82420009BE9
:106FC0001B6801981946FFF739FD019A40F200034A
:106FD000C4F201039A4206D1019B1B7BDBB203F092
:106FE000C003039305E0019B1B7BDBB203F0C003EE
:106FF0000393009B5B79012B04D0022B07D0002B5D
:107000000FD009E0039B43F0010303930AE0039BC5
:1070100043F00203039305E0039B43F00303039350
:1070200000E000BF009B1B79002B23D0039B43F0A3
:1070300008030393009B1B7903F1FF33032B19D83B
:1070400001A252F823F000BF7570000059700000D3
:10705000637000006D700000039B43F01003039306
:1070600008E0039B43F02003039303E0039B43F0FA
:1070700030030393009B9B79012B03D1039B43F0C7
:1070800004030393019A40F20003C4F201039A42FD
:1070900004D1019B039AD2B21A7303E0039BDAB2C4
:1070A000019B1A7305B000BD00B583B00190019A31
:1070B0004CF20003C4F200039A421CD0019A40F241
:1070C0000003C4F201039A4215D0019A48F200036A
:1070D000C4F209039A420ED0019A4CF20003C4F2A2
:1070E00009039A4207D042F25860C0F201004FF4FF
:1070F000CB71F9F70BFB01984FF0000100F044FD54
:10710000019A4CF20003C4F200039A4205D14FF0F9
:1071100008004FF0000101F0D3FB019A40F2000398
:10712000C4F201039A4205D14FF010004FF0000164
:1071300001F0C6FB019A48F20003C4F209039A4227
:1071400005D14FF080704FF0000101F0B9FB019ABA
:107150004CF20003C4F209039A4205D14FF00070CB
:107160004FF0000101F0ACFB03B000BD82B0019014
:10717000019B4FF416521A60019B4FF003025A71A3
:10718000019B4FF000021A71019B4FF000029A71AF
:1071900002B0704700B583B001900B468DF8033004
:1071A000019A4CF20003C4F200039A421CD0019AE7
:1071B00040F20003C4F201039A4215D0019A48F24A
:1071C0000003C4F209039A420ED0019A4CF2000364
:1071D000C4F209039A4207D042F25860C0F201009B
:1071E0004FF4ED71F9F792FA019A40F20003C4F2FC
:1071F00001039A4204D1019B9DF803201A7003E019
:10720000019B9DF803201A7003B000BD00B583B048
:107210000190019A4CF20003C4F200039A421CD080
:10722000019A40F20003C4F201039A4215D0019A78
:1072300048F20003C4F209039A420ED0019A4CF2BC
:107240000003C4F209039A4207D042F25860C0F228
:10725000010040F2F311F9F759FA019A40F20003E4
:10726000C4F201039A4203D1019B1B78DBB202E016
:10727000019B1B78DBB2184603B000BD00B58BB094
:107280000390029101928DF80330029B0993019BB8
:1072900005939DF80330012B3ED14FF00003069378
:1072A00036E04FF0FF33079306E0079B002B0BD02F
:1072B000079B03F1FF330793039B1B7DDBB203F0B6
:1072C0002003002BF1D000E000BF079B002B52D021
:1072D0004FF01003089315E0099B1B78099A02F1FF
:1072E0000102099203981946FFF754FF089B03F126
:1072F000FF330893059B03F1FF330593069B03F1CE
:1073000001030693089B002B02D0059B002BE3D1C1
:10731000059B002BC5D131E04FF00003069326E01A
:10732000039B1B7DDBB203F02003002B25D04FF025
:107330001003089315E0099B1B78099A02F10102DA
:10734000099203981946FFF725FF059B03F1FF33C8
:107350000593089B03F1FF330893069B03F1010398
:107360000693089B002B02D0059B002BE3D1059BC5
:10737000002BD5D102E000BF00E000BF069B1846FD
:107380000BB000BD00B589B00390029101928DF859
:107390000330029B0793019B04939DF80330012B5C
:1073A00031D14FF00003059329E04FF0FF330693EE
:1073B00006E0069B002B0BD0069B03F1FF330693E0
:1073C000039B1B7DDBB203F00103002BF1D000E037
:1073D00000BF069B002B38D00398FFF717FF03462A
:1073E0001A46079B1A70079B03F101030793049B3E
:1073F00003F1FF330493059B03F101030593049B01
:10740000002BD2D124E04FF00003059319E0039B39
:107410001B7DDBB203F00103002B18D00398FFF7AC
:10742000F5FE03461A46079B1A70079B03F10103FA
:107430000793059B03F101030593049B03F1FF33BD
:107440000493049B002BE2D102E000BF00E000BFE8
:10745000059B184609B000BD00B583B00190019AA4
:107460004CF20003C4F200039A421CD0019A40F28D
:107470000003C4F201039A4215D0019A48F20003B6
:10748000C4F209039A420ED0019A4CF20003C4F2EE
:1074900009039A4207D042F25860C0F2010040F25C
:1074A0008521F9F733F9019A40F20003C4F2010390
:1074B0009A4208D1019B019A127BD2B242F040025B
:1074C000D2B21A7307E0019B1B7BDBB243F040038F
:1074D000DAB2019B1A7303B000BD00BF00B585B0DE
:1074E000019013460A468DF803208DF80230019A68
:1074F0004CF20003C4F200039A421CD0019A40F2FD
:107500000003C4F201039A4215D0019A48F2000325
:10751000C4F209039A420ED0019A4CF20003C4F25D
:1075200009039A4207D042F25860C0F201004FF4BA
:107530002B71F9F7EBF89DF80230002B0BD09DF87A
:107540000230012B07D042F25860C0F2010040F235
:10755000AD21F9F7DBF89DF80330062B2BD801A2FB
:1075600052F823F0817500008975000091750000C4
:1075700099750000A1750000A9750000B1750000A3
:107580004FF00103039316E04FF00203039312E060
:107590004FF0040303930EE04FF0080303930AE057
:1075A0004FF08003039306E04FF48073039302E0EF
:1075B0004FF400730393019A40F20003C4F20103F5
:1075C0009A4224D19DF80330002B3CD09DF8033023
:1075D000012B38D09DF80330022B34D09DF80330B6
:1075E000052B30D09DF80330062B2CD09DF80330AE
:1075F000032B28D09DF80330042B24D042F258608E
:10760000C0F2010040F2C921F9F780F81BE09DF8B3
:107610000330002B17D09DF80330012B13D09DF8B9
:107620000330022B0FD09DF80330052B0BD09DF8B3
:107630000330062B07D042F25860C0F2010040F23E
:10764000CD21F9F763F89DF80230012B16D1019A8C
:1076500040F20003C4F201039A4207D1019B019A50
:107660005168039A41EA02025A602DE0019B5A6870
:10767000039B42EA0302019B5A6025E0019A40F213
:107680000003C4F201039A420FD1019A019B596889
:10769000039B6FEA030301EA030140F28F33C0F258
:1076A000000301EA030353600EE0019B5A68039B49
:1076B0006FEA030302EA030240F20733C0F2000359
:1076C00002EA0303019A536005B000BD00B583B020
:1076D0000190019A4CF20003C4F200039A421CD0BC
:1076E000019A40F20003C4F201039A4215D0019AB4
:1076F00048F20003C4F209039A420ED0019A4CF2F8
:107700000003C4F209039A4207D042F25860C0F263
:10771000010040F2FB21F8F7F9FF019A40F2000363
:10772000C4F201039A4206D140F20003C4F20103FD
:107730001B7DDBB202E0019B1B7DDBB2184603B070
:1077400000BD00BF00B583B00190019A4CF2000368
:10775000C4F200039A421CD0019A40F20003C4F222
:1077600001039A4215D0019A48F20003C4F20903BA
:107770009A420ED0019A4CF20003C4F209039A42D5
:1077800007D042F25860C0F2010040F21231F8F71F
:10779000BDFF019B9A6840F2CF33C0F2000302EABA
:1077A0000303184603B000BD82B00190019B1B7D0E
:1077B000DBB203F04003002B02D04FF0000301E0E6
:1077C0004FF00103184602B0704700BF00B585B006
:1077D000019000914FF000038DF80F30019A4CF2A8
:1077E0000003C4F200039A421CD0019A40F2000345
:1077F000C4F201039A4215D0019A48F20003C4F280
:1078000009039A420ED0019A4CF20003C4F2090314
:107810009A4207D042F25860C0F201004FF44E7114
:10782000F8F774FF009BDB78002B13D0009BDB780C
:10783000012B0FD0009BDB78022B0BD0009BDB7859
:10784000032B07D042F25860C0F2010040F23931F8
:10785000F8F75CFF009B9B78002B0BD0009B9B787C
:10786000012B07D042F25860C0F2010040F23A31D9
:10787000F8F74CFF009B1B78002B0BD0009B1B786C
:10788000012B07D042F25860C0F2010040F23B31B8
:10789000F8F73CFF009B5B78002B0BD0009B5B78DC
:1078A000012B07D042F25860C0F201004FF44F7133
:1078B000F8F72CFF9DF80F3043F001038DF80F30DF
:1078C000009BDB78012B04D0022B09D0002B19D0B0
:1078D0000FE09DF80F3043F040038DF80F3012E0B9
:1078E0009DF80F306FEA43636FEA53638DF80F30F2
:1078F00009E09DF80F306FEA83636FEA93638DF8B8
:107900000F3000E000BF009B5B78012B05D19DF894
:107910000F3043F004038DF80F30009B1B78012BD0
:1079200005D19DF80F3043F002038DF80F30009B16
:107930009B78012B05D19DF80F3043F008038DF89B
:107940000F30019A40F20003C4F201039A4206D1BB
:10795000019A9DF80F3003F0CF03137205E09DF8F4
:107960000F3003F0CF03019A137205B000BD00BFC2
:1079700082B00190019B4FF000029A70019B4FF082
:107980000002DA70019B4FF001021A70019B4FF068
:1079900001025A7002B0704700B587B0039002919F
:1079A00013468DF80730039A4CF20003C4F200032B
:1079B0009A421CD0039A40F20003C4F201039A4297
:1079C00015D0039A48F20003C4F209039A420ED07C
:1079D000039A4CF20003C4F209039A4207D042F220
:1079E0005860C0F2010040F29331F8F78FFE9DF825
:1079F0000730002B0BD09DF80730012B07D042F247
:107A00005860C0F201004FF46571F8F77FFE4FF047
:107A1000000305939DF80730012B0FD1029B1B78C3
:107A2000012B03D1059B43F002030593029B5B7876
:107A3000012B03D1059B43F004030593039A40F205
:107A40000003C4F201039A422BD19DF80730012BA9
:107A500022D1039A039B1B7BDBB26FEA43636FEA7D
:107A60005363DBB21373039B4FF000021A70039B46
:107A70004FF000021A71039A039B1B7BDBB203F0E9
:107A80007F031373039B4FF010029A62039B059AC6
:107A900042F001021A6230E0039B4FF000021A62CA
:107AA0002BE09DF80730012B23D1039B1B7BDBB21E
:107AB0006FEA43636FEA5363DAB2039B1A73039B63
:107AC0004FF000021A70039B4FF000021A71039BE3
:107AD0001B7BDBB203F07F03039A1373039B4FF00E
:107AE000100283F82820059B43F00102039B1A62D1
:107AF00003E0039B4FF000021A6207B000BD00BF15
:107B000000B583B001900B46ADF80230019A4CF2FB
:107B10000003C4F200039A421CD0019A40F2000311
:107B2000C4F201039A4215D0019A48F20003C4F24C
:107B300009039A420ED0019A4CF20003C4F20903E1
:107B40009A4207D042F25860C0F201004FF47571BA
:107B5000F8F7DCFD019A40F20003C4F201039A42F7
:107B600008D1019B1A6ABDF8023042EA0302019B68
:107B70001A6207E0019B1A6ABDF8023042EA03026A
:107B8000019B1A6203B000BD00B583B001900B46A3
:107B90008DF80330019A4CF20003C4F200039A42BC
:107BA0001CD0019A40F20003C4F201039A4215D09E
:107BB000019A48F20003C4F209039A420ED0019AD6
:107BC0004CF20003C4F209039A4207D042F2586013
:107BD000C0F2010040F2EB31F8F798FD9DF8033058
:107BE000002B0BD09DF80330012B07D042F25860D8
:107BF000C0F201004FF47B71F8F788FD9DF8033067
:107C0000012B20D1019A40F20003C4F201039A42F1
:107C10000CD1019A019B93F83030DBB26FEA4363D9
:107C20006FEA5363DBB282F8303024E0019B93F8B3
:107C30003030DBB26FEA43636FEA5363DAB2019B21
:107C400083F8302017E0019A40F20003C4F20103E8
:107C50009A4208D1019B93F83030019B4FF000020B
:107C600083F8302007E0019B93F83030019B4FF000
:107C7000000283F8302003B000BD00BF00B583B020
:107C800001900B468DF80330019A4CF20003C4F2C8
:107C900009039A4207D042F25860C0F2010040F254
:107CA0001541F8F733FD9DF80330002B0BD09DF8FC
:107CB0000330012B07D042F25860C0F2010040F2BD
:107CC0001641F8F723FD9DF80330012B0AD1019BE3
:107CD00093F82430DBB243F00203DAB2019B83F85D
:107CE00024200CE09DF80330002B08D1019B93F871
:107CF0002430DBB203F03D03019A82F8243003B054
:107D000000BD00BF00B583B001900B468DF8033075
:107D1000019A4CF20003C4F209039A4207D042F2DE
:107D20005860C0F2010040F22D41F8F7EFFC9DF8D9
:107D30000330002B0BD09DF80330012B07D042F20B
:107D40005860C0F2010040F22E41F8F7DFFC9DF8C8
:107D50000330012B0AD1019B93F82430DBB243F0AE
:107D60000103DAB2019B83F8242008E0019B93F819
:107D70002430DBB203F03E03019A82F8243003B0D2
:107D800000BD00BF00B585B001900B468DF80330F3
:107D9000019A4CF20003C4F209039A4207D042F25E
:107DA0005860C0F2010040F24E41F8F7AFFC9DF878
:107DB0000330002B23D09DF80330012B1FD09DF8FA
:107DC0000330022B1BD09DF80330032B17D09DF8F6
:107DD0000330042B13D09DF80330052B0FD09DF8F2
:107DE0000330062B0BD09DF80330072B07D042F24F
:107DF0005860C0F2010040F24F41F8F787FC9DF84F
:107E0000033003F007034FEAC3030393019B93F886
:107E10002430DBB223F038030293039A029B42EA38
:107E2000030343F004030293029BDBB203F03F031E
:107E3000019A82F8243005B000BD00BF00B585B0BE
:107E4000019013460A468DF803208DF802304FF05A
:107E500000038DF80F30019A40F20003C4F20103D1
:107E60009A4207D042F25860C0F2010040F26E41DF
:107E7000F8F74CFC9DF80330002B0BD09DF8033035
:107E8000012B07D042F25860C0F2010040F26F416E
:107E9000F8F73CFC9DF80230002B0BD09DF8023027
:107EA000012B07D042F25860C0F201004FF48E61FE
:107EB000F8F72CFC9DF80330002B02D0012B05D0E5
:107EC00008E04FF001038DF80F3003E04FF002039C
:107ED0008DF80F309DF80230012B0AD1019B1B7CDD
:107EE000DAB29DF80F3042EA0303DAB2019B1A744A
:107EF00011E0019B1B7CDBB21A469DF80F306FEA44
:107F00000303DBB2DBB203F0F30302EA0303DBB2E9
:107F1000DAB2019B1A7405B000BD00BF00B585B090
:107F2000019013460A468DF803208DF80230019A1D
:107F300040F20003C4F201039A4207D042F25860B3
:107F4000C0F2010040F29641F8F7E0FB9DF80330E3
:107F5000002B0FD09DF80330012B0BD09DF8033080
:107F6000022B07D042F25860C0F2010040F2974164
:107F7000F8F7CCFB9DF80230002B0BD09DF80230B7
:107F8000012B07D042F25860C0F201004FF4936118
:107F9000F8F7BCFB9DF80330012B08D0022B0BD067
:107FA000002B0DD14FF010038DF80F3008E04FF08B
:107FB00040038DF80F3003E06FF07F038DF80F3032
:107FC0009DF80230012B0AD1019B1B7CDAB29DF88F
:107FD0000F3042EA0303DAB2019B1A7411E0019BED
:107FE0001B7CDBB21A469DF80F306FEA0303DBB24D
:107FF000DBB203F0F30302EA0303DBB2DAB2019B64
:108000001A7405B000BD00BF00B583B00190019A9D
:1080100040F20003C4F201039A4207D042F25860D2
:10802000C0F2010040F2C141F8F770FB019B1B7EDA
:10803000DBB2184603B000BD00B585B001900091D9
:10804000019A40F20003C4F201039A4207D042F2BF
:108050005860C0F2010040F2D541F8F757FB009B91
:108060009B78002B0BD0009B9B78012B07D042F212
:108070005860C0F2010040F2D641F8F747FB009B80
:10808000DB78002B0BD0009BDB78012B07D042F272
:108090005860C0F2010040F2D741F8F737FB009B6F
:1080A000DB79FF2B07D142F25860C0F201004FF498
:1080B0009B61F8F72BFB009B5B79002B0BD0009B9F
:1080C0005B79012B07D042F25860C0F2010040F208
:1080D000D941F8F71BFB009B1B79002B0BD0009BB1
:1080E0001B79012B07D042F25860C0F2010040F228
:1080F000DA41F8F70BFB009B9B79FF2B07D142F28B
:108100005860C0F2010040F2DB41F8F7FFFA009B33
:108110001B78002B0BD0009B1B78012B07D042F261
:108120005860C0F2010040F2DC41F8F7EFFA009B22
:108130005B78002B0BD0009B5B78012B07D042F2C1
:108140005860C0F2010040F2DD41F8F7DFFA4FF06D
:1081500000030393009BDB78012B18D1039B43F0B2
:1081600010030393009B5B79012B03D1039B43F026
:1081700020030393009B1B79012B03D1039B43F046
:1081800008030393009BDA79019B83F85420009B3A
:108190001B78012B03D1039B43F001030393009B46
:1081A0009B78012B08D1039B43F004030393009BAE
:1081B0009A79019B83F85020009B5B78002B03D1B8
:1081C000039B43F002030393039BDBB203F03F03E3
:1081D000019A82F84C30019B1B7BDBB243F03803E1
:1081E000DAB2019B1A7305B000BD00BF82B00190E6
:1081F0000B468DF803309DF80330012B09D1019B0C
:1082000093F84C30DBB203F0FD03019A82F84C3056
:1082100009E0019B93F84C30DBB243F00203DAB281
:10822000019B83F84C2002B0704700BF00B587B0B7
:108230000390029101928DF803309DF80330002BDA
:1082400027D0039B1B7B8DF812309DF812308DF8E0
:1082500013309DF8123023F010038DF81230039B79
:108260009DF812201A73039B18460299019A4FF049
:108270000103FFF703F803460593039B1B7DDBB265
:1082800003F04003002BF8D0039B9DF813201A73D2
:1082900010E0039B18460299019A4FF00103FEF784
:1082A000EDFF03460593039B1B7DDBB203F0400308
:1082B000002BF8D0059B184607B000BD00B583B071
:1082C00001900B468DF803300DF103030198194618
:1082D0004FF001024FF00103FFF7A8FF03B000BD0C
:1082E00000B585B003900291019203980299019A1A
:1082F0004FF00003FFF79AFF0346184605B000BD94
:108300004CF20003C4F20F03D3F888304FEA136332
:1083100003F00303032B40F0AA804CF20003C4F2E5
:108320000F03D3F80C3103F00303032B00F2F480A6
:1083300001A252F823F000BF49830000AD83000082
:1083400013840000498300004CF20003C4F20F03C1
:10835000D3F888304FEA43434FEA534303F1010215
:1083600041F20023C0F27A0303FB02F24CF2000355
:10837000C4F20F03D3F888304FEA134303F0FF032E
:1083800003F10103B2FBF3F24CF20003C4F20F035A
:10839000D3F8043103F0FF0303F10103B2FBF3F25E
:1083A00040F23C03C1F200031A60B6E04CF2000355
:1083B000C4F20F03D3F888304FEA43434FEA5343E4
:1083C00003F1010243F20063C0F26E1303FB02F2F9
:1083D0004CF20003C4F20F03D3F888304FEA134382
:1083E00003F0FF0303F10103B2FBF3F24CF20003CD
:1083F000C4F20F03D3F8043103F0FF0303F10103C8
:10840000B2FBF3F240F23C03C1F200031A6000BF7A
:1084100083E04CF20003C4F20F03D3F888304FEA34
:1084200043434FEA534303F101034FEA03424CF243
:108430000003C4F20F03D3F888304FEA134303F06C
:10844000FF0303F10103B2FBF3F24CF20003C4F2A9
:108450000F03D3F8043103F0FF0303F10103B2FB70
:10846000F3F240F23C03C1F200031A6055E04CF213
:108470000003C4F20F03D3F80C3103F00303032B02
:108480004BD801A252F823F099840000C584000063
:10849000F1840000998400004CF20003C4F20F0341
:1084A000D3F8043103F0FF0303F1010240F6001397
:1084B000C0F23D03B3FBF2F240F23C03C1F2000311
:1084C0001A602AE04CF20003C4F20F03D3F804311F
:1084D00003F0FF0303F1010241F60033C0F2B703DA
:1084E000B3FBF2F240F23C03C1F200031A6014E065
:1084F0004CF20003C4F20F03D3F8043103F0FF037E
:1085000003F101034FF40042B2FBF3F240F23C03EB
:10851000C1F200031A6000E000BF70474CF2000394
:10852000C4F20F034FF02002C3F8A0214CF2000365
:10853000C4F20F03D3F8A03103F02003002B09D0BD
:108540004CF20003C4F20F03D3F8A03103F0400350
:10855000002BF5D04CF20003C4F20F034FF00302DE
:10856000C3F804214CF20003C4F20F034FF00002E1
:10857000C3F8A8214CF20003C4F20F034FF000022D
:10858000C3F8AC214CF20003C4F20F034FF0010218
:10859000C3F80C214CF20003C4F20F0340F2630253
:1085A000C0F20502C3F884204CF20003C4F20F03AA
:1085B0004FF0AA02C3F88C204CF20003C4F20F0360
:1085C0004FF05502C3F88C204CF20003C4F20F03A5
:1085D0004FF00102C3F880204CF20003C4F20F03F5
:1085E0004FF0AA02C3F88C204CF20003C4F20F0330
:1085F0004FF05502C3F88C204CF20003C4F20F0375
:10860000D3F8883003F08063002BF5D04CF20003E0
:10861000C4F20F034FF00302C3F880204CF20003B2
:10862000C4F20F034FF0AA02C3F88C204CF20003EF
:10863000C4F20F034FF05502C3F88C204CF2000334
:10864000C4F20F03D3F8883003F04073002BF5D049
:108650004CF20003C4F20F034FF02302C3F8A4202E
:108660004CF20003C4F20F034FF0AA02C3F8AC208F
:108670004CF20003C4F20F034FF05502C3F8AC20D4
:108680004CF20003C4F20F034FF00102C3F8A02024
:108690004CF20003C4F20F034FF0AA02C3F8AC205F
:1086A0004CF20003C4F20F034FF05502C3F8AC20A4
:1086B0004CF20003C4F20F03D3F8A83003F4806334
:1086C000002BF5D04CF20003C4F20F034FF003026D
:1086D000C3F8A0204CF20003C4F20F034FF0AA022B
:1086E000C3F8AC204CF20003C4F20F034FF0550264
:1086F000C3F8AC204CF20003C4F20F03D3F8A83047
:1087000003F44073002BF5D04CF20003C4F20F03C6
:1087100048F2DE72C0F22842C3F8C4204CF20003D3
:10872000C4F20F034FF00002C3F8C8214CF200035B
:10873000C4F20F0343F23A021A604EF60053CEF22F
:1087400000034FF000029A60704700BF84B00190B0
:108750000091019B1F2B03D9019BA3F1200300E093
:10876000019B0393019B1F2B27D84CF20003C4F2FB
:108770000F034CF20002C4F20F02D2F8A811039AC0
:108780004FF0030000FA02F26FEA020201EA02026D
:10879000C3F8A8214CF20003C4F20F034CF200020C
:1087A000C4F20F02D2F8A811039A009800FA02F25C
:1087B00041EA0202C3F8A82126E04CF20003C4F209
:1087C0000F034CF20002C4F20F02D2F8AC11039A6C
:1087D0004FF0030000FA02F26FEA020201EA02021D
:1087E000C3F8AC214CF20003C4F20F034CF20002B8
:1087F000C4F20F02D2F8AC11039A009800FA02F208
:1088000041EA0202C3F8AC2104B0704784B0019081
:10881000019B1F2B09D8019B02934CF20003C4F269
:108820000F03D3F8A83103930AE0019BA3F12003BF
:1088300002934CF20003C4F20F03D3F8AC3103935C
:10884000029B039A22FA03F303F003030393039BAF
:10885000184604B0704700BF00B585B0019040F2E3
:108860003C03C1F200031B6802930198FFF7CEFF9F
:1088700003460393039B032B19D801A252F823F05C
:108880009188000099880000A1880000A988000054
:108890004FF0040303930AE04FF00103039306E053
:1088A0004FF00203039302E04FF008030393029A90
:1088B000039BB2FBF3F30293029B184605B000BD85
:1088C00082B001900B468DF803309DF80330012BE8
:1088D00015D14CF20002C4F20F024CF20003C4F2B4
:1088E0000F03D3F8C41001984FF2DE73CEF6EF7386
:1088F00000EA030341EA0303C2F8C4301AE09DF81A
:108900000330002B16D14CF20002C4F20F024CF2DD
:108910000003C4F20F03D3F8C410019B6FEA0303F2
:1089200001EA03014FF2DE73CEF6EF7301EA0303AF
:10893000C2F8C43002B070474CF20003C4F20F0317
:108940004FF00002C3F8C02030BF70474EF600530E
:10895000CEF200034FF004021A614CF20003C4F29D
:108960000F034FF00802C3F8C02030BF704700BFAC
:108970004EF60053CEF200034FF004021A614CF29F
:108980000003C4F20F034FF00902C3F8C02030BF48
:10899000704700BF4EF60053CEF200034FF00402C2
:1089A0001A614CF20003C4F20F034FF00302C3F844
:1089B000C02030BF704700BF4BB942B9002908BF83
:1089C000002802D04FF0FF31084600F037B882B0DF
:1089D000EC462DE9005000F005F8DDF804E002B0A7
:1089E0000CBC7047F8B514461D4606460F4600F00D
:1089F000D9F900FB05F5A0FB042304FB0154E3189F
:108A0000B61A67EB0307069BC3E90067F8BD00BF12
:108A1000F8B514461D4606460F4600F011F800FB57
:108A200005F5A0FB042304FB0154E318B61A67EB19
:108A30000307069BC3E90067F8BD00BF704700BF8E
:108A400000292DE9F04F85B0C0F2C8800026002B28
:108A5000C0F2BF808946144605469B46002B4AD18A
:108A60008A4257D9B2FA82F353B1C3F1200001FA16
:108A700003F925FA00F812FA03F49D4048EA0909BF
:108A8000270C484639461FFA84FB00F00DFB394697
:108A90008246484600F036FC2A0C0BFB0AF342EAF9
:108AA00001494B4509D919EB04090AF1FF3A04D2EF
:108AB0004B4584BF0AF1FF3AA144C3EB090939468B
:108AC0004846ADB200F0F0FA39468046484600F01C
:108AD00019FC0BFB08FB45EA0145AB4507D92D19ED
:108AE00008F1FF3803D2AB4588BF08F1FF3848EAE8
:108AF0000A48002703E08B4257D90027B846424670
:108B00003B4616B1524263EB43031946104605B08B
:108B1000BDE8F08F22B91146012000F0C5FA0446E5
:108B2000B4FA84F8B8F1000F5ED1C4EB0908270C41
:108B30001FFA84F9012102913946404600F0B4FA47
:108B400039468246404600F0DDFB4FEA154809FBF6
:108B50000AF348EA014B5B4509D91BEB040B0AF108
:108B6000FF3A04D25B4584BF0AF1FF3AA344C3EB4A
:108B70000B0B39465846ADB200F096FA394680469E
:108B8000584600F0BFFB09FB08F945EA0145A94535
:108B900007D92D1908F1FF3803D2A94588BF08F17C
:108BA000FF3848EA0A48029FA9E7B3FA83F7002F83
:108BB00068D18B422CBF4FF000094FF0010982426F
:108BC0008CBF4C4649F00104002C96D04FF00108B0
:108BD00095E7524263EB4303F6433BE7404261EBC8
:108BE00041014FF0FF3632E704FA08F4C8F12007DC
:108BF00035FA07F329FA07FA270C09FA08FB394670
:108C0000504643EA0B02029200F04EFA39461FFA30
:108C100084F98346504600F075FB029809FB0BF27D
:108C2000030C43EA01439A4204D91B190BF1FF3BA1
:108C3000C0F0B1809B1A39461846019300F034FA0F
:108C4000019982460846394600F05CFBDDF808C011
:108C500009FB0AF31FFA8CF040EA0142934208D95B
:108C600012190AF1FF3A04D2934284BF0AF1FF3A83
:108C7000121905FA08F54AEA0B4EC3EB0208CDF8C3
:108C800008E059E7C7F1200003FA07FAC24035FAB5
:108C900000F342EA0A0B21FA00F801FA07F940460C
:108CA0004FEA1B4A43EA0901029151461FFA8BF22F
:108CB000039200F0F9F951468146404600F022FB4C
:108CC000039BDDF808C003FB09F24FEA1C4014FACD
:108CD00007F340EA0144A24204D914EB0B0409F162
:108CE000FF3952D3A41A51462046019300F0DCF913
:108CF00051468046204600F005FB0398DDF808C089
:108D000000FB08F21FFA8CF343EA0140019B824208
:108D100004D910EB0B0008F1FF3830D348EA0948BA
:108D20001FFA83FC1B0C801A1FFA88FE4FEA184AB0
:108D30000CFB0EF90CFB0AFC03FB0EC103FB0AF251
:108D400001EB19418C4588BF02F5803202EB114ED0
:108D5000704510D31FFA89F905FA07F709EB0140AE
:108D600014BF0022012287422CBF002702F0010716
:108D7000002F3FF4C4AE08F1FF380027BFE682425F
:108D800084BF584408F1FF38C8E7A24284BF09F104
:108D9000FF395C44A6E79A4284BF0BF1FF3B1B19E5
:108DA00048E700BF2DE9F04F0C4683B080461646D9
:108DB00089461F4615468A46002B4BD18A425CD90C
:108DC000B2FA82F35BB1C3F1200001FA03FA28FA88
:108DD00000F216FA03F508FA03F842EA0A0A2E0C22
:108DE00050463146AFB200F05FF931464FEA1844C1
:108DF0008146504600F086FA07FB09F344EA014A2F
:108E0000534509D91AEB050A09F1FF3904D2534534
:108E100084BF09F1FF39AA44C3EB0A0A3146504620
:108E20001FFA88F800F040F931460446504600F039
:108E300069FA07FB04F748EA0148474506D9013CAF
:108E400018EB050802D2474588BF013C44EA0944B3
:108E500000265CE08B4258D8B3FA83F6002E5BD133
:108E60008B422CBF0022012285428CBF154642F066
:108E70000105002D49D0012449E022B91146012005
:108E800000F012F90546B5FA85F6002E40F0BA80DA
:108E9000641B2F0C1FFA85FA01263946204600F084
:108EA00003F939464FEA184B8146204600F02AFA6A
:108EB0000AFB09F34BEA014B5B4509D91BEB050B98
:108EC00009F1FF3904D25B4584BF09F1FF39AB4496
:108ED000C3EB0B0B394658461FFA88F800F0E4F84C
:108EE00039460446584600F00DFA0AFB04FA48EAEF
:108EF0000148C24506D9013C18EB050802D2C2451B
:108F000088BF013C44EA094401E00026344631466A
:108F1000204603B0BDE8F08FC6F12000B34032FA1E
:108F200000F721FA00FB1F4314FA06F228FA00F1B9
:108F300058464FEA174A114300915146BBB201937C
:108F400000F0B2F85146B5408146584600F0DAF9D3
:108F5000019C009804FB09F34FEA104C4CEA014BCA
:108F60005B4505D91BEB070B09F1FF39C0F08E807B
:108F7000C3EB0B0B5146584600F096F85146044699
:108F8000584600F0BFF90198009A00FB04F31FFA5D
:108F900082FC4CEA0142934206D9013CD21903D229
:108FA000934201D9D219013C44EA0944A8B2D21A29
:108FB0002D0C1FFA84FC230C00FB0CF700FB03FEB6
:108FC00005FB0CE105FB03F501EB17418E4588BF5E
:108FD00005F5803505EB1145AA4210D3BFB208FA5A
:108FE00006F607EB014214BF4FF0000E4FF0010EE2
:108FF00096422CBF00260EF00106002E87D0013CC1
:10900000002684E7B540C6F1200124FA01F928FAC8
:1090100001F22F0CB440394648462243009200F03A
:1090200043F839461FFA85FA8346484600F06AF944
:10903000009B1A0C0AFB0BF342EA0144A34203D93A
:1090400064190BF1FF3B27D3E41A3946204600F0A0
:109050002BF839468146204600F054F900980AFB67
:1090600009F31FFA80FC4CEA0144A34208D96419B1
:1090700009F1FF3904D2A34284BF09F1FF39641911
:1090800008FA06F8E41A49EA0B4606E75B4584BF8E
:1090900009F1FF39BB446BE7A34284BF0BF1FF3BEF
:1090A0006419D1E7000000004A1E08BF7047C0F0F5
:1090B0002481884240F21681114200F01781B0FAF3
:1090C00080F3B1FA81F2A2EB0303C3F11F0304A200
:1090D00002EB03134FF000029F4600BFAFF3008086
:1090E000B0EBC17F00BF42EB020228BFA0EBC17012
:1090F000B0EB817F00BF42EB020228BFA0EB817082
:10910000B0EB417F00BF42EB020228BFA0EB4170F1
:10911000B0EB017F00BF42EB020228BFA0EB017061
:10912000B0EBC16F00BF42EB020228BFA0EBC160F1
:10913000B0EB816F00BF42EB020228BFA0EB816061
:10914000B0EB416F00BF42EB020228BFA0EB4160D1
:10915000B0EB016F00BF42EB020228BFA0EB016041
:10916000B0EBC15F00BF42EB020228BFA0EBC150D1
:10917000B0EB815F00BF42EB020228BFA0EB815041
:10918000B0EB415F00BF42EB020228BFA0EB4150B1
:10919000B0EB015F00BF42EB020228BFA0EB015021
:1091A000B0EBC14F00BF42EB020228BFA0EBC140B1
:1091B000B0EB814F00BF42EB020228BFA0EB814021
:1091C000B0EB414F00BF42EB020228BFA0EB414091
:1091D000B0EB014F00BF42EB020228BFA0EB014001
:1091E000B0EBC13F00BF42EB020228BFA0EBC13091
:1091F000B0EB813F00BF42EB020228BFA0EB813001
:10920000B0EB413F00BF42EB020228BFA0EB413070
:10921000B0EB013F00BF42EB020228BFA0EB0130E0
:10922000B0EBC12F00BF42EB020228BFA0EBC12070
:10923000B0EB812F00BF42EB020228BFA0EB8120E0
:10924000B0EB412F00BF42EB020228BFA0EB412050
:10925000B0EB012F00BF42EB020228BFA0EB0120C0
:10926000B0EBC11F00BF42EB020228BFA0EBC11050
:10927000B0EB811F00BF42EB020228BFA0EB8110C0
:10928000B0EB411F00BF42EB020228BFA0EB411030
:10929000B0EB011F00BF42EB020228BFA0EB0110A0
:1092A000B0EBC10F00BF42EB020228BFA0EBC10030
:1092B000B0EB810F00BF42EB020228BFA0EB8100A0
:1092C000B0EB410F00BF42EB020228BFA0EB410010
:1092D000B0EB010F00BF42EB020228BFA0EB010080
:1092E000104670470CBF012000207047B1FA81F290
:1092F000C2F11F0220FA02F0704708B14FF0FF30B0
:10930000FFF79CBB0029F8D02DE90340FFF7CCFE06
:10931000BDE8064002FB00F3A1EB0301704700BF6C
:10932000032A2DE9F0070BD83AB1002311F803C046
:1093300000F803C001339342F8D1BDE8F00770474D
:1093400082180C46034603E014F8011C03F8011CC4
:1093500003F003061946A44601330134002EF3D16D
:109360001CF00304634608BFC1EB020C68D06542E1
:10937000C4F1040A0CEB050733464FEACA0A5CF84D
:1093800005604FEAC408551A08E057F8044F26460E
:1093900004FA0AF449EA0404CC5004335C18032D9F
:1093A00026FA08F9A5F104050CEB0306EDDC002311
:1093B00002E0F15CE154013319199142F9D3BCE7A1
:1093C00053F8404C41F8404C53F83C4C41F83C4C6D
:1093D00053F8384C41F8384C53F8344C41F8344C7D
:1093E00053F8304C41F8304C53F82C4C41F82C4C8D
:1093F00053F8284C41F8284C53F8244C41F8244C9D
:1094000053F8204C41F8204C53F81C4C41F81C4CAC
:1094100053F8184C41F8184C53F8144C41F8144CBC
:1094200053F8104C41F8104C53F80C4C41F80C4CCC
:1094300053F8084C41F8084C53F8044C41F8044CDC
:109440001C460D4640334031BCF13F0FACF1400C9F
:10945000B6DC21462B46541B0FE051F8105C43F854
:10946000105C51F80C5C43F80C5C51F8085C43F854
:10947000085C51F8045C43F8045C0F2C0D469C46D4
:1094800001F1100103F11003A4F11004E5DCCCEBB1
:109490000201002303E0EC584CF8034004335E194A
:1094A000032903EB0C04A1F10401F4DC7FE700BF06
:1094B000032AC9B230B407D822B10023C154013302
:1094C0009342FBD130BC704700EB020C034601E035
:1094D00003F8011C03F003041A460133002CF7D1F2
:1094E0004FF00133C2EB0C0403FB01F31FE042F821
:1094F000403C42F83C3C42F8383C42F8343C42F8AC
:10950000303C42F82C3C42F8283C42F8243C42F8DB
:10951000203C42F81C3C42F8183C42F8143C42F80B
:10952000103C42F80C3C42F8083C42F8043C15461A
:1095300040323F2CA4F14004D9DC2A46C5EB0C0490
:1095400007E042F8103C42F80C3C42F8083C42F874
:10955000043C154610320F2CA4F11004F1DC2A460D
:10956000C5EB0C0501E042F8043C14460432032D1F
:10957000A5F10405F7DC01E004F8011B6445FBD309
:10958000A0E700BF0FB440F24003C1F2000310B5E2
:109590001C6882B024B1A36913B9204604F0B4FB5F
:1095A000204605AC049A23468168019401F04AFDE7
:1095B00002B0BDE8104004B0704700BF0EB410B553
:1095C000044683B018B183690BB904F09DFB2046B3
:1095D00006AC059A23468168019401F033FD03B07F
:1095E000BDE8104003B070470CB440F24003F0B542
:1095F000C1F200030C1E9DB005461E6828DB23AF98
:10960000229A3B46304601A90CBFA44604F1FF3C18
:109610004FF4027E0595ADF810E04FF0FF3ECDF817
:1096200018C00195ADF812E0CDF80CC01B9700F002
:10963000B5FAB0F1FF3F08DB14B1019B00221A70AC
:109640001DB0BDE8F04002B070478B233360F3E7F4
:109650008B234FF0FF303360F2E700BF08B4F0B562
:10966000141E9CB006460D4627DB22AF219A3B46CE
:1096700001A90CBFA44604F1FF3C4FF4027E0595FE
:10968000ADF810E04FF0FF3ECDF818C00195ADF8F1
:1096900012E0CDF80CC01B9700F080FAB0F1FF3F4C
:1096A00008DB14B1019B00221A701CB0BDE8F04029
:1096B00001B070478B233360F3E78B2303604FF0D7
:1096C000FF30F2E70EB440F2400330B59CB01FAC5F
:1096D000C1F20003054601A954F8042B4FF0FF3CEA
:1096E00018684FF40273ADF81030234605950195C4
:1096F0006FF00045ADF812C0069503951B9400F07D
:109700004DFA019B00221A701CB0BDE8304003B036
:10971000704700BF0CB40B4610B59CB01EAC01A93D
:1097200005934FF4027C54F8042B01934FF0FF3360
:10973000ADF8123023461B946FF00044ADF810C012
:109740000694039400F02AFA019B00221A701CB0C0
:10975000BDE8104002B07047C9B230B419B124E07E
:109760000378D3B1013010F0030FF9D10368A3F1EE
:10977000013222EA030313F0803F08D150F8043F7E
:10978000A3F1013222EA030313F0803FF6D00378FD
:109790001BB110F8013F002BFBD130BC70470378A0
:1097A000002B36D09942F8D0013010F0030FF6D1DB
:1097B000036841EA0125A3F1013245EA054522EAA1
:1097C000030212F0803F1BD185EA0303A3F10132AB
:1097D00022EA030313F0803F03D011E012F0803F30
:1097E0000ED150F8043FA3F1013485EA030224EAC4
:1097F0000303A2F1013C13F0803F2CEA0202EDD0FA
:1098000003781BB905E010F8013F13B19942FAD172
:10981000C3E70020C1E700BF80EA0102844612F0DE
:10982000030F4FD111F0030F32D14DF8044D11F059
:10983000040F51F8043B0BD0A3F101329A4312F00C
:10984000803F04BF4CF8043B51F8043B16D100BFE5
:1098500051F8044BA3F101329A4312F0803FA4F176
:1098600001320BD14CF8043BA24312F0803F04BFFD
:1098700051F8043B4CF8044BEAD023460CF8013B6A
:1098800013F0FF0F4FEA3323F8D15DF8044B704714
:1098900011F0010F06D011F8012B0CF8012B002A52
:1098A00008BF704711F0020FBFD031F8022B12F041
:1098B000FF0F16BF2CF8022B8CF8002012F47F4FFC
:1098C000B3D1704711F8012B0CF8012B002AF9D104
:1098D000704700BF20F0030110F00300C0F100004A
:1098E00051F8043B00F1040C4FEACC0C6FF000027D
:1098F0001CBF22FA0CF213434FF0010C4CEA0C2C63
:109900004CEA0C4CA3EB0C0222EA030212EACC1242
:1099100004BF51F8043B0430F4D013F0FF0F1FBF15
:10992000013013F47F4F013013F47F0F18BF013063
:10993000704700BF30B41346002A43D041EA00020A
:1099400012F0030F25D1032B04460D463DD90268C2
:1099500009688A4239D1043B34D0A2F1013121EAAD
:10996000020212F0803F0DD02CE022682968A2F19B
:1099700001308A4220EA020027D1043B22D010F0B5
:10998000803F1FD104340435032BEED820462946EE
:10999000F3B10478013B91F800C064450FD18BB15D
:1099A00084B1013B002202E063B15CB1013B841849
:1099B0008D180132647895F801C06445F4D0CCEB81
:1099C000040000E0002030BC704720462946E0E754
:1099D000247895F800C0CCEB0400F4E741EA0003DA
:1099E00013F0030F14BF00230123032A94BF0023A5
:1099F00003F0010330B4002B2AD004460B68A3F116
:109A0000013C2CEA030C1CF0803F05D1043A0431E0
:109A1000032A44F8043BF1D82346BAB10D781C461A
:109A2000013A04F8015B55B102337AB111F8015FD4
:109A30001C46013A03F8015C0133002DF5D12AB12F
:109A400000231946E15401339342FBD130BC7047E7
:109A50000346E2E770B503460C4661B1002500E01D
:109A6000154618462146FFF777FE0246431C00289C
:109A7000F6D1284670BDBDE87040FFF76DBE00BF4F
:109A80002DE9F04F85B092460C4603909068176818
:109A9000002800F081804FF000090B684D46002D32
:109AA00054D0A668B542B0463EBF18462E46A846DA
:109AB0003CD3A08910F4906F08BF184636D0626975
:109AC000216902EB420B5B1A03F1010C0BEBDB7B10
:109AD000AC444FEA6B0BE3455A463CBFE3465A465B
:109AE00010F4806F37D011460398019304F012FDF3
:109AF000019B00283BD01A46216901930290FFF791
:109B00000FFCA289019BDDF808C022F4906242F0AC
:109B10008002A2812E46A846C3EB0B020CEB030089
:109B2000A260C4F810C02060C4F814B04246494690
:109B300004F0FCFFA2682368961BA660DAF80820F0
:109B400043442360551BCAF80850FDB1D7F8009074
:109B50007D680837A3E70398019305F0F3FC019BA8
:109B600084460028D6D10398216904F051F9039A5C
:109B70000C234FF0FF3013600023A289CAF8043091
:109B800042F04002CAF80830A28102E02846CAF832
:109B9000045005B0BDE8F08F5060FAE72DE9F04FB2
:109BA000C5B00E469A461546099004F001FCB389EB
:109BB00013F0800F00681B9003D03369002B01F075
:109BC0008C800DF17409B3464C460022109200239C
:109BD000189217921A920D922DAA199328320DF10C
:109BE000F703169207930023CDF8DC90389339934E
:109BF0002B78B3F1250218BF0122002B0CBF0022E5
:109C000002F0010202B32E4616F8013F1A1E18BFD9
:109C10000122252B0CBF002202F00102002AF3D101
:109C2000771B08BF35460FD06760389B399A0133E0
:109C30002560D219072B3992389379DC08340D98B6
:109C40003546C0190D903378002B00F0378700217E
:109C50004FF00002CDF828A06B1C0C914FF0FF389C
:109C60008DF80F218A466A782B204FF0200C5D1C5E
:109C7000A2F12003582B00F21982DFE813F0290229
:109C800017021702350217021702170217021702EE
:109C900017023C0248021702C802CF021702EF0265
:109CA000F602F602F602F602F602F602F602F602F4
:109CB000F6021702170217021702170217021702FD
:109CC0001702170217024F028802170288021702B2
:109CD000170217021702C10217021702EE0317023A
:109CE0001702170217021702930317021702AD0398
:109CF000170217021702170217021702170217029C
:109D000017021702C703D8038802880288020B03D0
:109D1000D803170217020F031702190329033E0382
:109D20008C03170259031702840317021702EA0073
:109D30000998594637AAFFF7A3FE00287CD14C4664
:109D40007DE71899012940F35284119A0123636039
:109D5000389B2260399A013338930132072B3992AC
:109D600000F39685083401236360389B399A0133E8
:109D70001B980132072B39922060389300F37D85C0
:109D80000834109800220023199906F0D9FC002805
:109D900040F003851899119B4A1E6260591C389B3C
:109DA00021603999013338938A18072B399200F3CF
:109DB0002F8408341A9A1A9862603EAA389B22604F
:109DC000399A013338931218072B399200F34F81D7
:109DD00004F108031AF0040F00F056810C990B9A55
:109DE0008E1A002E40F35081102E42F26867D8BFC1
:109DF000C0F2010740F3DE831024C0F201070DF129
:109E0000DC08DDF824A003E0103E102E40F3D283DE
:109E10005C60389A399901321F601031072A3991F4
:109E200003F108033892EFDD504659464246FFF7EA
:109E300027FE4B460028E7D05E46B3890D9813F005
:109E4000400F18BF4FF0FF300D900D9845B0BDE8A2
:109E5000F08F1AF0200F42F2AC60C0F201001492B1
:109E6000179000F0C3820A99CB1D23F0070303F17A
:109E700008020A92D3E9006756EA07010CBF0022E4
:109E800001221AEA020F40F0BC8402234FF00001C5
:109E90008DF80F11B8F1000FA8BF2AF0800AB8F1B1
:109EA000000F18BF42F00102002A00F06081012B70
:109EB00000F03484022B00F017841699CDF82C8022
:109EC00011914FEAD6084FEAD70C48EA477806F0D6
:109ED000070067464646303056EA070201F8010D92
:109EE000EFD11AF0010FDDF82C80119140F0DB84E6
:109EF000169B5B1A0E930E9BCDF854804345B8BF5A
:109F000043460B939DF80F3113B10B9901310B911F
:109F10001AF00202139202D00B9B02330B931AF039
:109F20008400129038D10C990B9A8E1A002E33DDD2
:109F3000102E42F26867D8BFC0F2010720DD4FF053
:109F40001008C0F2010702E0103E102E18DDC4F820
:109F50000480389B399A013327601032072B3992DD
:109F600004F108043893EFDD0998594637AA4C46A6
:109F7000FFF786FD00287FF45FAF103E102EE6DC71
:109F80006660389B27605A1C399B38929B19072AB8
:109F9000399300F3F78308349DF80F3173B101232F
:109FA0006360389B43AA03322260399A01333893A5
:109FB0000132072B399200F340830834139B6BB1B5
:109FC00002236360389B43AA2260399A0133389395
:109FD0000232072B399200F33A8308341298802812
:109FE00000F0B28215980E9BC61A002E2EDD102EA0
:109FF000A74FC8BF4FF0100803DC1BE0103E102E27
:10A0000018DDC4F80480389B399A01332760103278
:10A01000072B399204F108043893EFDD099859466B
:10A0200037AA4C46FFF72CFD00287FF405AF103E01
:10A03000102EE6DC6660389B27605A1C399B3892EC
:10A040009B19072A399300F3EE8208341AF4807FB3
:10A0500040F019820E99119A6160389B2260399AFA
:10A06000013338935218072B39927FF7B1AE099814
:10A07000594637AAFFF704FD00287FF4DDAE1AF039
:10A08000040F4B467FF4AAAE399B0D980B9A0C999E
:10A090008A42ACBF801840180D90002B40F09E8281
:10A0A0000023DDF828A038934C46A1E51492002A3D
:10A0B00000F0048501208DF8B4204FF000012DAA96
:10A0C0000B908DF80F1111920E90002115911FE742
:10A0D0009DF80F31002B40F00C840A992B468DF827
:10A0E0000FC12A780A91C2E50A994AF0010A2A7832
:10A0F0002B460A91BBE50A9B0A9A1B68111D002B8F
:10A100000C93C0F2B2852A782B460A91AFE50A99E2
:10A110002B468DF80F012A780A91A8E54AF0100A1B
:10A1200014921AF0200F00F087810A98C31D23F0C3
:10A13000070303F108010A91D3E90067002E77F1C4
:10A140000000C0F2768356EA07014FF001030CBF0E
:10A1500000220122B8F1000FA8BF2AF0800AB8F14E
:10A16000000F18BF42F00102002A7FF4A0AE002BBE
:10A1700040F0E5811AF0010F00F0E18130238DF805
:10A18000DB302DAB012027330E901193B3E61AF08C
:10A19000080F149200F0BF830A98C31D23F0070331
:10A1A00003F108010A915E681F68199610973846F6
:10A1B000314605F0A1FB0346002800F093843846A1
:10A1C00000220023314606F0C5FA002840F015842D
:10A1D0009DF80F31032042F2A06242F29C610B9085
:10A1E0001498C0F20101C0F201022AF0800A472847
:10A1F000D8BF0A460321119200220E91159283E6E0
:10A200000A994AF0080A2A782B460A912FE50A99FA
:10A210002A784AF0040A2B460A9128E52B4613F8BF
:10A22000012B2A2A00F0CF86A2F13001092988BF2C
:10A230004FF0000810D802354FF0000815F8012C37
:10A2400008EB88082B46013501EB4808A2F13001E4
:10A250000929F3D948EAE8781D4609E50A994AF040
:10A26000800A2A782B460A9101E5A2F130010026E6
:10A270002B4606EB860613F8012B01EB4606A2F1EE
:10A2800030011D460929F3D90C961D46F0E400BFA4
:10A29000782601004AF0400A0A9934E72A786C2AA5
:10A2A00000F018840A994AF0100A2B460A91DEE45D
:10A2B0001AF0200F00F023830A990D9A0B681046BC
:10A2C0004FEAE0710A9AC3E9000102F1040A8FE43F
:10A2D0001AF02003149200F0C7800A9BDA1D0023B5
:10A2E00022F0070202F108000A90D2E9006756EA5C
:10A2F00007010CBF00220122C8E50A9A42F2AC60B5
:10A300000A997823C0F201001493166804318DF87D
:10A310000D314AF0020A3023321E18BF01228DF897
:10A320000C3136464FF00007179002230A91ADE535
:10A330000A9B14924FF00002181D8DF80F211B6824
:10A340000A901193002B00F04D85B8F1000F119881
:10A35000C0F22A850021424604F0AEFB03460028E5
:10A3600000F06E8511981B1A0E93434540F38284CA
:10A37000CDF83880002128EAE8789DF80F31CDF833
:10A380002C801591C0E51AF0200F149210D00A9B72
:10A39000DA1D0123A4E70A994AF0200A2A782B46FD
:10A3A0000A9164E44AF0100A14921AF0200FEED1D8
:10A3B0001AF0100F40F054821AF0400F00F0508253
:10A3C0000A980123011D0A910688321E18BF012236
:10A3D00036464FF0000759E51AF0200F149242F26A
:10A3E0008862C0F2010217927FF43DAD1AF0100F9F
:10A3F00040F02D821AF0400F00F029820A990A1DC0
:10A400000A920E8836464FF0000735E51492012077
:10A410000A9A4FF000010B900E90136804328DF8E9
:10A420000F110A922DAA8DF8B43011924DE61AF050
:10A43000200F14927FF479AE1AF0100F40F0ED81E6
:10A440001AF0400F00F0E9810A98011D0A91B0F955
:10A45000006036464FEAE67770E64AF0100A14923A
:10A460001AF020037FF439AF1AF0100200F05F8277
:10A470000A9A101D0A901668321E18BF012236462D
:10A480004FF0000702E5149B652B7FF75AAC10983C
:10A4900000220023199906F053F9002800F0E1800A
:10A4A00001236360389A42F2C863C0F2010323605B
:10A4B000399B013238920133072A3993D8BF04F10E
:10A4C000080300F39F82429A1898824203DB1AF035
:10A4D000010F3FF47FAC1B9901225A60389A196032
:10A4E0003999013238920131072A399100F3EB830F
:10A4F0000833189A561E002E7FF76CAC102EA04F12
:10A5000040F3E98110240DF1DC0803E0103E102E29
:10A5100040F3E1815C60389A399901321F60103153
:10A52000072A399103F108033892EFDD099859465B
:10A530004246FFF7A5FA4B460028E7D07CE416997F
:10A5400000220E921191D6E40C990B9A8E1A002ECD
:10A550007FF748AD102E8A4FC8BF4FF0100803DCBC
:10A560001BE0103E102E18DDC4F80480389B399A89
:10A57000013327601032072B399204F10804389315
:10A58000EFDD0998594637AA4C46FFF779FA0028BB
:10A590007FF452AC103E102EE6DC6660389B2760DC
:10A5A0005A1C399B38929B19072A399300F38881EA
:10A5B000083417E55E60389A1F60399B0132389283
:10A5C000F318072A39937FF760AD0998594637AADF
:10A5D000FFF756FA00283FF457AD2DE40998594685
:10A5E00037AAFFF74DFA00283FF45AAD24E41AF0D9
:10A5F000010F7FF4AAAB01236360389B399A0133C2
:10A6000011990132072B3992216038937FF7D1AB32
:10A610000998594637AAFFF733FA00287FF40CACA3
:10A620004C46FFF7C7BB0998594637AAFFF728FAE7
:10A6300000287FF401AC4C4608E50998594637AA32
:10A64000FFF71EFA00287FF4F7AB4C46B6E40998F2
:10A65000594637AAFFF714FA00287FF4EDAB4C46B1
:10A66000BCE4429B002B40F3D98118998B42C0F285
:10A670006F81119A6160389B2260399A0133389357
:10A680005218072B3992D8BF04F1080300F3BA839C
:10A69000429C1898241A002C40F39B81102C384FB0
:10A6A00040F38B81CDF838A01026AA460DF1DC08C6
:10A6B000099D03E0103C102C40F37C815E60389AC9
:10A6C000399901321F601031072A399103F10803CB
:10A6D0003892EFDD284659464246FFF7D1F94B46FE
:10A6E0000028E7D0FFF7A8BB1698DDF85CC003464A
:10A6F0001190310906F00F0241EA077138091CF880
:10A7000002200E46074656EA070103F8012DF0D154
:10A71000169A1193D21A0E92FFF7EDBB002309226D
:10A72000B24273EB0700169B3EBFCDF82C80A046CB
:10A730001C461AD2304639460A220023FEF73CF95D
:10A7400030463946002302F1300C0A2204F801CDCC
:10A75000FEF732F906460F4609200021B042B94102
:10A76000E8D323464446DDF82C805A1E3036119239
:10A7700003F8016C169B9B1A0E93FFF7BCBB00BF3E
:10A78000782601000998594637AAFFF779F9002879
:10A790007FF452AB4C46FFF7FFBB1898461E002EC5
:10A7A0007FF708AB102E9C4FC8BF4FF0100803DC9A
:10A7B0001BE0103E102E18DDC4F80480389B399A37
:10A7C000013327601032072B399204F108043893C3
:10A7D000EFDD0998594637AA4C46FFF751F9002892
:10A7E0007FF42AAB103E102EE6DC6660389B399A67
:10A7F000013327609219072B399238937FF7D9AA32
:10A8000006E7149830214AF0020A012202238DF84B
:10A810000C118DF80D01FFF739BB0A9A131D16684C
:10A820000A9336464FEAE677002E77F10000BFF62E
:10A830008AAC764267EB47072D2356EA07028DF86C
:10A840000F310CBF002201220123FFF723BB0A9B1B
:10A85000181D1E680A9036464FF00007FFF70CBB24
:10A860000A9A131D16680A930123321E18BF01228B
:10A8700036464FF00007FFF709BB0998594637AA3B
:10A88000FFF7FEF800287FF4D7AA4C46FFF779BA05
:10A890000998594637AAFFF7F3F800287FF4CCAAA5
:10A8A0004C46FFF760BA302800F09682119A3023A8
:10A8B00002F8013D169B11929B1A0E93FFF71BBBEA
:10A8C0000998594637AAFFF7DBF800287FF4B4AAA5
:10A8D0004C46FFF787BB5E60389A399901321F609A
:10A8E0008919072A399138923FF7C1AB0833FFF72E
:10A8F00071BA0A992B462A780A91FFF7B8B91AF06B
:10A90000100F00F0CD810A980D9900F1040A036838
:10A910001960FFF76DB90A9AD31D23F0070303F1FD
:10A9200008000A905E681F68199610973FE41AF0B5
:10A93000400300F0A9810A9913460A1D0A920E8865
:10A94000321E18BF012236464FF00007FFF79EBAAD
:10A95000119A636038992260399A01313891D3187D
:10A960000729399300F3628208340123429E636011
:10A97000389B399A01331B980132072B3893D8BF83
:10A9800004F108032060399200F34682429A11993B
:10A9900018988E191E60811A596039998A1A389947
:10A9A000121839920131389107293FF760AB08330B
:10A9B000FFF710BA5546DDF838A05C60389A39992F
:10A9C00001321F600919072A3991389200F37F82FA
:10A9D00008331AF0010F3FF4FDA91B9901225A60B8
:10A9E000389A19603999013238920131072A399120
:10A9F0003FF73DAB0833FFF7EDB92D238DF80F314D
:10AA0000FFF7E8BB0998594637AAFFF739F800283D
:10AA10007FF412AA4B4656E57826010001236360B5
:10AA2000389A42F2C863C0F201032360399B0132B5
:10AA300038920133072A3993D8BF04F1080300F391
:10AA40007381429A2AB9189818B91AF0010F3FF485
:10AA5000C1A91B9901225A60389A196039990132AB
:10AA600038920131072A399100F368810833429CFA
:10AA70006442002C40F38781102C9E4F40F3A0814C
:10AA800010260DF1DC0803E0103C102C40F39881F7
:10AA90005E60389A399901321F601031072A399166
:10AAA00003F108033892EFDD099859464246FEF754
:10AAB000E7FF4B460028E7D0FFF7BEB9399B5E465B
:10AAC000002B3FF4BAA90998594637AAFEF7D8FFD8
:10AAD000FFF7B3B90A994AF0200A6A786B1C0A9109
:10AAE000FFF7C5B838463146089304F017FF089BB6
:10AAF000002840F00181B8F1FF3F08BF08F10708C6
:10AB00000ED0149A672A14BF00230123472A08BFD6
:10AB100043F0010323B1B8F1000F08BF4FF0010863
:10AB200033463A46CDE93A234AF4807A3B9B002BE0
:10AB3000C0F20A82002315931499662914BF0023DA
:10AB40000123462908BF43F001031293002B00F0B4
:10AB50008A810323CDF82C800B990E970F960093D2
:10AB60000998DDE90E23019142A9029141A90391BF
:10AB700040A9049102F00CF8149AB2F1670318BFCF
:10AB80000123472A0CBF002303F0010311902BB9C6
:10AB90001AF0010F08BFDDF800C11AD0119B0B9805
:10ABA000129903EB000C29B11B78302B00F0D080F8
:10ABB000429B9C443846002200233146CDF820C0F9
:10ABC00005F0BEFDDDF820C0002800F07381CDF84F
:10ABD00000C114981199672814BF00230123472846
:10ABE00008BF43F00103C1EB0C011891002B00F0EA
:10ABF0004A81429A12F1030F0E9202DB904580F2D5
:10AC00004B81149B023B14930E9A1498531E42934B
:10AC1000002B8DF8F800C0F2D1812B228DF8F9209D
:10AC2000092B00F362813FA930338DF8FB303023CC
:10AC30008DF8FA303EAB189ACB1A18991A93591816
:10AC4000012A0E9140F3CC810E9801300E9020EA3B
:10AC5000E0710B91159B002B00F0FD802D2300204F
:10AC60008DF80F311590FFF750B90C9B5B420C9398
:10AC7000FFF7CEBA0E9A00209DF80F3122EAE27259
:10AC800015900B92FFF740B90A98011D0A910668CA
:10AC9000321E18BF012236464FF00007FFF7F6B804
:10ACA0001AF0400F17BF0A9A0A990D9802F1040A88
:10ACB00011BF136801F1040A0B680D9A14BF1880C4
:10ACC0001A60FEF795BF0998594637AAFEF7D8FED5
:10ACD00000287FF4B1A84B460BE40998402103F00B
:10ACE00019FC30603061002800F08D8140237361D1
:10ACF000FEF767BF78260100032042F2A86242F205
:10AD0000A4610B901498C0F20101C0F201021593E6
:10AD10004728D8BF0A462AF0800A032111929DF8DD
:10AD20000F310E91FFF7F0B80998594637AAFEF790
:10AD3000A7FE00287FF480A84B4682E60998594672
:10AD400037AAFEF79DFE00287FF476A84B468EE6D4
:10AD50003846002200233146CDF820C005F0F0FC33
:10AD6000DDF820C000287FF423AF0B9AC2F1010365
:10AD700042931EE70998594637AAFEF781FE00283C
:10AD80007FF45AA84B46189A11985A60389A399904
:10AD900018600132189838920918072A39913FF73C
:10ADA00066A90833FFF716B800211591FEF792FD4A
:10ADB0009DF80F3120EAE0720E900B92FFF7A4B8D5
:10ADC0005C60389A1F60511C399A38911219072912
:10ADD0003992CFDC0833D6E716991198081A0E90ED
:10ADE000FFF789B8B8F1060F34BF4146062142F299
:10ADF000C062C0F2010221EAE1730E9111920B933D
:10AE0000FFF763B90998594637AAFEF739FE0028BB
:10AE10007FF412A84B463BE40998594637AAFEF73F
:10AE20002FFE00287FF408A84B46AFE50998594645
:10AE300037AAFEF725FE00287EF4FEAF4C4694E5C7
:10AE4000CDF8388028EAE8781590CDF82C809DF868
:10AE50000F31FFF759B80E989DF80F3120EAE070D6
:10AE60000B90FFF751B8149A652A14BF00230123F1
:10AE7000452A08BF43F00103002B32D008F101033B
:10AE80000B93022368E61498652862DD149A662AFB
:10AE90001CBF429B0E936FD0189A0E9B9A425BDCAC
:10AEA0001AF0010F40F0818023EAE37067210B90D4
:10AEB0001491CFE6409B9C4598BF9C467FF689AE97
:10AEC000302203F8012B9C454093FAD881E609987B
:10AED000594637AAFEF7D4FD00287EF4ADAF4B46A5
:10AEE00077E5CDF82C80023336E646F2676C0DF13B
:10AEF000F700C6F2666C8CFB0321DA17C2EBA102E5
:10AF000002EB8201A3EB410113463031092A00F81C
:10AF1000011DF0DC3033421ED9B200F8011C079B42
:10AF2000934298BF0DF1FA017FF684AE02460DF10F
:10AF3000FB0301E012F8011B03F8011C19460798F6
:10AF400001339042F6D875E62D2006F100461590A3
:10AF5000F2E542990E9157E60E9918980029DABF4A
:10AF60000E9AC2F1020301231B18672123EAE37240
:10AF70000E9314910B926DE6429800280E9038DDE6
:10AF8000B8F1000F07D11AF0010F04BF20EAE071F9
:10AF90000B913FF45FAE0E9A66201490531C43440D
:10AFA0000E9323EAE3710B9154E60E9A67231493F0
:10AFB00001320E9222EAE2700B904BE62D225B42A8
:10AFC0008DF8F9202CE60A991A78D1F8008004311E
:10AFD0000A91B8F1000FB8BF4FF0FF38FEF747BE37
:10AFE0001AF0010F04BF21EAE1730B933FF432AE74
:10AFF0002AE6B8F1000F0ED11AF0010F0BD1012291
:10B000000B920E9226E609980C234FF0FF310D911A
:10B010000360FEF71ABF08F10203662023EAE3711A
:10B020000E9314900B9115E6936810B5144613B95E
:10B030005360184610BD02F0CBFF00236360A3608D
:10B0400010BD00BF2DE9F04FADF5AE6D83B00E46DB
:10B0500015469A46814603F0ABF900681D90B9F198
:10B06000000F04D0D9F81830002B00F05A8142F2BA
:10B07000FC63C0F201039E4208BFD9F8046010D0FF
:10B0800042F21C73C0F201039E4208BFD9F8086067
:10B0900007D042F23C73C0F201039E4208BFD9F8C8
:10B0A0000C60B6F80CC01FFA8CF313F4005F09D1E2
:10B0B0004CF4005C726EA6F80CC01FFA8CF322F4FC
:10B0C0000052726613F0080F01F001833269002A02
:10B0D00001F0FD8203F01A030A2B00F0E080002249
:10B0E00012921A9200231C920DF59C641192043462
:10B0F00019920DF5A4621B9304320DF5906328326A
:10B100000333189207930023CDF84C45CDF8503502
:10B11000CDF854352B781A1E18BF0122252B0CBFF1
:10B12000002202F0010232B32F4617F8013F1A1E27
:10B1300018BF0122252B0CBF002202F00102002AB9
:10B14000F3D1B7EB050808BF3D4614D0C4F804801E
:10B15000DDF85035DDF8542501332560072B4244D6
:10B16000CDF85035CDF8542578DC083411983D469B
:10B17000404411903B78002B7CD06B1C4FF0FF3784
:10B180002B204FF0200C00214FF000020F918DF882
:10B190007725CDF82CA06A780A915D1CA2F12003D6
:10B1A000582B00F28682DFE813F0980284028402B2
:10B1B000A402840284028402840284028402AD0216
:10B1C000BA028402C102CA028402E702F002F0025B
:10B1D000F002F002F002F002F002F002F00284024B
:10B1E000840284028402840284028402840284022F
:10B1F0008402040326038402260384028402840258
:10B2000084026A0384028402810484028402840228
:10B21000840284021404840284022F0484028402BF
:10B2200084028402840284028402840284028402EE
:10B230004F04650426032603260373036504840272
:10B2400084027903840285039603AD030A04840211
:10B25000CC038402F40384028402C0000DF5A862CA
:10B26000484631460C32FFF7DFFE58B90DF59C64B5
:10B2700004347BE7DDF85435002B41F09281002344
:10B28000CDF85035B38913F0400F02D04FF0FF30A6
:10B29000119011985FB00DF5806DBDE8F08FB6F993
:10B2A0000E30002BFFF61BAF376A2CF0020CD6F8DD
:10B2B00028E00DF58E64ADF888C40C34B6F80EC0E5
:10B2C0002A465346484621461FADCDF89C740027B8
:10B2D000CDF88C54CDF87C544FF48065CDF8A4E4BF
:10B2E000ADF88AC4CDF89054CDF89474CDF8845458
:10B2F000FFF7A8FE0028119009DB2146484602F01E
:10B3000093FB1199B84218BF4FF0FF311191BDF86E
:10B31000883413F0400FBCD0B38943F04003B381AD
:10B32000B7E7484602F0F0FCA1E60A9842F2AC6C9E
:10B33000C0F2010C169210F0200FCDF864C000F09E
:10B340006E830B99CB1D23F0070303F108020B92C8
:10B35000D3E900AB5AEA0B020A9B0CBF0022012280
:10B36000134240F06B8602234FF000018DF87715F1
:10B37000002FA2BFDDF828C02CF0800CCDF828C02B
:10B38000002F18BF42F00102002A00F01E84012B9A
:10B3900000F0DE85022B00F0C185189913914FEA69
:10B3A000DA084FEADB0C48EA4B780AF00700E3467C
:10B3B000C24630305AEA0B0201F8010DEFD1DDF838
:10B3C00028C013911CF0010F40F08C861898401A89
:10B3D00010909DF87735109A1797BA42B8BF3A4641
:10B3E0000C9213B10C9A01320C920A9B0A9813F03A
:10B3F000020315931EBFDDF830C00CF1020CCDF82E
:10B4000030C010F0840014904DD10F990C9A8F1A0F
:10B41000002F48DD102F42F2CC68D8BFC0F20108DF
:10B4200030DDC0F201080DF5A86B43464FF0100A5D
:10B43000A8460BF10C0B1D4602E0103F102F1EDD3D
:10B44000C4F804A0DDF85035DDF85425013325603B
:10B450001032072BCDF8542504F10804CDF85035EF
:10B46000EBDD0DF59C64484631465A460434FFF73F
:10B47000DBFD00287FF406AF103F102FE0DC2B46E9
:10B48000454698466760DDF85035C4F800805A1C80
:10B49000DDF85435CDF85025DB19072ACDF85435A1
:10B4A00000F38A8508349DF877359BB101236360EA
:10B4B000DDF850350DF5AE6207322260DDF8542517
:10B4C0000133CDF850350132072BCDF8542500F368
:10B4D000B6840834159B9BB102236360DDF85035B8
:10B4E0000DF5AE6204322260DDF854250133CDF84B
:10B4F00050350232072BCDF8542500F3AF840834C1
:10B50000DDF850C0BCF1800F00F07683179B109AD5
:10B510009F1A002F43DD102FDFF88C8B2EDD434662
:10B520000DF5A86BA8464FF0100A0BF10C0B1D4649
:10B5300002E0103F102F1EDDC4F804A0DDF85035E6
:10B54000DDF85425013325601032072BCDF8542542
:10B5500004F10804CDF85035EBDD0DF59C64484648
:10B5600031465A460434FFF75FFD00287FF48AAE67
:10B57000103F102FE0DC2B46454698466760DDF80B
:10B580005035DDF854250133C4F80080D219072B5B
:10B59000CDF85425CDF8503500F342840834DDF859
:10B5A00028C01CF4807F40F09D8210981399606041
:10B5B000DDF85035DDF85425013321601218072BD2
:10B5C000CDF85035D8BF04F10803CDF8542500F369
:10B5D0009B830A9911F0040F55D00F9ADDF830C003
:10B5E000CCEB0207002F4EDD102F42F2CC68D8BF03
:10B5F000C0F201082EDDC0F201080DF5A86A42462E
:10B600001024A8460AF10C0A154602E0103F102F3C
:10B610001DDD5C60DDF85025DDF8541501321D603C
:10B620001031072ACDF8541503F10803CDF8502541
:10B63000ECDD484631465246FFF7F6FC0DF59C63BB
:10B64000043300287FF41EAE103F102FE1DC2A46A1
:10B65000454690465F60DDF85025C3F80080DDF870
:10B6600054350132CDF85025FB18072ACDF8543552
:10B670000BDD0DF5A862484631460C32FFF7D4FCCD
:10B6800000287FF4FFADDDF8543511980C9A0F991E
:10B690008A42ACBF801840181190002B40F04283C2
:10B6A0000DF59C640023DDF82CA00434CDF8503552
:10B6B00030E51692002A3FF4DDAD0DF5A4600123BC
:10B6C0004FF0000C04300C938DF824258DF877C5CD
:10B6D000139010930021179187E69DF87735002B82
:10B6E00040F02B850B992B468DF877C52A780B9166
:10B6F00053E50B990A9B43F001030A932B462A78E2
:10B700000B914AE50B990B9A09680F91111D0F9B3C
:10B71000002BC0F280872A782B460B913DE50B99D0
:10B720002B468DF877052A780B9136E50B990A9B05
:10B7300043F004030A932B462A780B912DE52B4600
:10B7400013F8012B2A2A01F0CD80A2F1300109293A
:10B7500001F237800235002715F8012C07EB870727
:10B760002B46013501EB4707A2F130010929F3D936
:10B7700047EAE7771D4611E50B992B460A9A42F0F6
:10B7800080020A922A780B9107E5A2F130014FF06E
:10B7900000082B4608EB880813F8012B01EB48083A
:10B7A000A2F130011D460929F3D9CDF83C801D4690
:10B7B000F4E40A9B169243F010030A93DDF828C0C4
:10B7C0001CF0200F00F05D810B98C31D23F00703D0
:10B7D00003F108010B91D3E900ABBAF1000F7BF143
:10B7E0000002C0F29B845AEA0B034FF001030CBF26
:10B7F00000220122BCE50A98169210F0080F00F012
:10B80000ED840B99CB1D23F0070303F108020B9283
:10B81000D3F80480D3F800A0CDF86C80CDF848A010
:10B820005046414604F068F88346002800F09985A8
:10B83000504600220023414604F08CFF002840F0CF
:10B840000B859DF8773542F2A06142F29C62169812
:10B85000C0F20101C0F201024FF0030C4728D8BF2B
:10B86000114613910A99CDF830C021F08001CDF82E
:10B8700040C00A914FF0000CCDF85CC0B1E50B99C7
:10B880000A9B43F008030A932B462A780B9184E421
:10B890000A9941F040010A910B993CE72A786C2AF9
:10B8A00000F055850B990A9B0B9143F010030A9306
:10B8B0002B4672E40A9A12F0200F00F082840B9853
:10B8C000119A036810464FEAE0710B9AC3E9000130
:10B8D00002F1040A1EE416920A9A12F0200300F004
:10B8E000EF800B9BDA1D002322F0070202F1080C07
:10B8F000CDF82CC0D2E900AB5AEA0B000CBF0022F5
:10B90000012231E50B987821DDF828C016910368F3
:10B9100042F2AC608DF8751530218DF874154CF03D
:10B92000020C0B991A1E18BF0122C0F201009A46A0
:10B930004FF0000B0431CDF828C0199002230B9171
:10B9400012E50B9B16924FF00002181D8DF877251B
:10B950001B680B901393002B00F0C686002F1398E2
:10B96000C0F28F8600213A4603F0A6F8034600286D
:10B9700000F0F58613981B1A1093BB4240F3BE8566
:10B980001097002127EAE7779DF877350C971791F4
:10B9900027E5DDF828C016921CF0200F23D00B9865
:10B9A0000123C21D22F0070202F108010B91D2E926
:10B9B00000AB5AEA0B020CBF00220122D4E40A9920
:10B9C0002B4641F020010A910B992A780B91FFF741
:10B9D000E4BB0A9B169243F010030A93DDF828C0DB
:10B9E0001CF0200FDBD10A9B13F0100F00F0D58361
:10B9F0000B980123021D0B9201680A1E18BF012239
:10BA00008A464FF0000BAFE40A98169242F2886221
:10BA100010F0200FC0F2010219927FF492AC0A9B41
:10BA200013F0100F40F01A830A9A12F0400F00F042
:10BA300015830B9B03F1040CCDF82CC0B3F800A0C8
:10BA4000D2464FF0000B85E416920DF5A4610B9AD7
:10BA50004FF0010C4FF000000431CDF830C01368F6
:10BA600004328DF877050B921391CDF840C08DF814
:10BA700024352FE6DDF828C016921CF0200F7FF445
:10BA8000A3AE0A9A12F0100F40F0F1820A9A12F057
:10BA9000400F00F0EC820B9B03F1040CCDF82CC09E
:10BAA000B3F900A0D2464FEAEA7B96E60A991692CD
:10BAB00041F010010A910A9A12F020037FF411AFAD
:10BAC0000A9911F0100200F054830B9A02F1040C51
:10BAD000CDF82CC011680A1E18BF01228A464FF00B
:10BAE000000B41E4169A652A40F32881129800223F
:10BAF00000231B9904F024FE002800F0BE810123DE
:10BB00006360DDF8502542F2C863C0F20103236090
:10BB1000DDF854350132CDF850250133072ACDF830
:10BB20005435D8BF04F1080300F39B83DDF870257A
:10BB30001A98824204DB0A9911F0010F3FF449ADD3
:10BB400001225A60DDF85025DDF8541501321D98A8
:10BB50000131072ACDF854151860CDF8502500F3AF
:10BB60005F8508331A994F1E002F7FF732AD102FD3
:10BB7000DFF8348540F3EA8242460DF5A86AA8460C
:10BB800010240AF10C0A154603E0103F102F40F371
:10BB9000DA825C60DDF85025DDF8541501321D6055
:10BBA0001031072ACDF8541503F10803CDF85025BC
:10BBB000EBDD484631465246FFF736FA0DF59C63F9
:10BBC00004330028E1D0FFF75DBB7BB90A9911F07F
:10BBD000010F0BD00DF5A462302304328DF84B35E4
:10BBE0002732012313921093FFF7F3BB189800211B
:10BBF00010911390FFF7EDBB0F980C99471A002F87
:10BC00007FF784AC102FDFF8A0842EDD43460DF5BE
:10BC1000A86BA8464FF0100A0BF10C0B1D4602E072
:10BC2000103F102F1EDDC4F804A0DDF85035DDF8FC
:10BC30005425013325601032072BCDF8542504F12B
:10BC40000804CDF85035EBDD0DF59C6448463146CF
:10BC50005A460434FFF7E8F900287FF413AB103F8D
:10BC6000102FE0DC2B46454698466760DDF85035DE
:10BC7000C4F800805A1CDDF85435CDF85025DB1986
:10BC8000072ACDF8543500F33A8208343EE413997C
:10BC90006360DDF850252160DDF854150132CDF8E0
:10BCA0005025CB18072ACDF8543500F349850834C0
:10BCB0001D9A0123DDF870756360DDF85035226050
:10BCC000DDF854250133CDF850350132072BCDF87E
:10BCD0005425D8BF04F1080300F323851398DDF839
:10BCE0007025C7191A981F60811A5960DDF854151C
:10BCF0008A1ADDF850151218CDF854250131CDF807
:10BD00005015072940F332820DF5A86248463146A6
:10BD10000C32FFF789F900287FF4B4AA0DF59C6373
:10BD2000043356E40DF5A862484631460C32FFF75D
:10BD30007BF900283FF4B4ACFFF7A4BA1A990129A3
:10BD40004CDD01236360DDF85035DDF85425013307
:10BD500013980132072BCDF854252060CDF85035CB
:10BD600000F3B281083401236360DDF85035DDF85B
:10BD7000542501331D990132072BCDF8542521603C
:10BD8000CDF8503500F39281083412980022002338
:10BD90001B9904F0D5FC002840F01D811A9B1398D4
:10BDA0005A1E6260DDF85035411C2160DDF85415E3
:10BDB0000133CDF850358A18072BCDF8542521DCF6
:10BDC00008341C9B0DF5AC621C9822606360DDF8A2
:10BDD0005035DDF854250133FFF7F0BB0A9A12F015
:10BDE000010FAED1139A01236360DDF85035226054
:10BDF000DDF854250133CDF850350132072BCDF84D
:10BE00005425DDDD0DF5A862484631460C32FFF7BA
:10BE10000BF900287FF436AA0DF59C640434D0E7B2
:10BE20000DF5A862484631460C32FFF7FDF80028B0
:10BE30007FF428AA0DF59C640434FFF7B0BB0DF520
:10BE4000A862484631460C32FFF7EEF800287FF42E
:10BE500019AA0DF59C640434FFF73CBB0DF5A862EC
:10BE6000484631460C32FFF7DFF800287FF40AAA73
:10BE70000DF59C640434FFF743BBDDF87035002BEF
:10BE800040F3FD811A998B42FFF601AF139A61606E
:10BE9000DDF850352260DDF854250133CDF85035FA
:10BEA0005218072BCDF85425D8BF04F1080300F32E
:10BEB0002984DDF870451A98241A002C40F3B381C8
:10BEC000102CDFF8E48140F39D8142460DF5A86A0D
:10BED000A84610270AF10C0A154603E0103C102C66
:10BEE00040F38D815F60DDF85025DDF85415013297
:10BEF0001D601031072ACDF8541503F10803CDF861
:10BF00005025EBDD484631465246FFF78DF80DF5DA
:10BF10009C6304330028E1D0FFF7B4B9189A19984C
:10BF2000134613920AF00F024FEA1A1141EA0B71FD
:10BF30004FEA1B1C825C8A46E3465AEA0B0C03F864
:10BF4000012DEFD118981393C01A1090FFF741BA42
:10BF500009220023524573EB0B00DDF860801FD2ED
:10BF600023464446B8461F46504659460A220023F7
:10BF7000FCF722FD00235046594602F1300C0A22FC
:10BF800004F801CDFCF718FD0922002382468B46F8
:10BF9000524573EB0B03E7D33B464746A0461C468E
:10BFA00008F1FF300AF1300A139008F801AC189933
:10BFB000091A1091FFF70DBA0DF5A86248463146EF
:10BFC0000C32FFF731F800287FF45CA90DF59C6472
:10BFD0000434FFF768BA1A994F1E002F7FF7F1AEAD
:10BFE000102FDFF8C4804EDD43460DF5A86BA84640
:10BFF0004FF0100A0BF10C0B1D4602E0103F102F02
:10C000003EDDC4F804A0DDF85035DDF854250133D9
:10C0100025601032072BCDF8542504F10804CDF823
:10C020005035EBDD0DF59C64484631465A460434E4
:10C03000FEF7FAFF0028E1D0FFF724B91698302167
:10C04000DDF828C0012202238DF874154CF0020C93
:10C050008DF87505CDF828C0FFF786B90B98011D3E
:10C0600003680B919A464FF0000BFFF773B90B98DA
:10C07000011D03680B919A464FEAEA7BFFF7ADBBBF
:10C080002B46454698466760DDF85035DDF8542567
:10C090000133C4F80080D219072BCDF85425CDF810
:10C0A00050357FF78DAEADE6DC2601000DF5A862B8
:10C0B000484631460C32FEF7B7FF00287FF4E2A86D
:10C0C0000DF59C64043460E60DF5A86248463146DF
:10C0D0000C32FEF7A9FF00287FF4D4A80DF59C646C
:10C0E000043440E6302800F0EC821398302300F846
:10C0F000013D18991390091A1091FFF76AB90DF5CF
:10C10000A862484631460C32FEF78EFF00287FF4C5
:10C11000B9A80DF59C640434FFF7F8B9DAF1000A08
:10C120006BEB4B0B2D235AEA0B0C8DF877350CBFBC
:10C13000002201220123FFF71BB90B992B462A7815
:10C140000B91FFF72AB82A46454690465F60DDF816
:10C150005025DDF854150132C3F80080C919072AAB
:10C16000CDF85415CDF850253FF7CEAD0833FFF785
:10C1700030BA0A9810F0400300F0ED810B99134695
:10C180000A1D0B92B1F800A0BAF1000218BF0122FB
:10C19000D2464FF0000BFFF7E7B80A9B13F0400FB1
:10C1A00000F0CC810B980123011D0B91B0F800A089
:10C1B000BAF1000218BF0122D2464FF0000BFFF780
:10C1C000D3B80A9B13F0100F00F0A4810B981199BB
:10C1D00000F1040A03681960FEF79CBF0B98C31DA9
:10C1E00023F0070303F108010B91D3F80480D3F87F
:10C1F00000A0CDF86C80CDF848A0FFF711BB2A460F
:10C20000454690465C60DDF85025DDF85415013256
:10C21000C3F800800919072ACDF85415CDF8502528
:10C2200000F3EA8208330A9911F0010F3FF4D1A913
:10C2300001225A60DDF85025DDF8541501321D98B1
:10C240000131072ACDF854151860CDF850253FF775
:10C250005BAD0833FFF7BDB92D238DF87735FFF7B8
:10C26000F2BA0DF5A862484631460C32FEF7DCFE04
:10C2700000287FF407A80DF59C63043356E40123DE
:10C280006360DDF8502542F2C863C0F20103236009
:10C29000DDF854350132CDF850250133072ACDF8A9
:10C2A0005435D8BF04F1080300F38781DDF8702509
:10C2B0003AB91A9A2AB9DDF828C01CF0010F3FF4E8
:10C2C00088A901225A60DDF85025DDF854150132A5
:10C2D0001D980131072ACDF854151860CDF8502566
:10C2E00000F379810833DDF870757F42002F40F349
:10C2F000B381102FDFF8508640F3D28142460DF50E
:10C30000A86AA84610240AF10C0A154603E0103F5B
:10C31000102F40F3C2815C60DDF85025DDF8541524
:10C3200001321D601031072ACDF8541503F10803BE
:10C33000CDF85025EBDD484631465246FEF774FEF7
:10C340000DF59C6304330028E1D0FEF79BBF0B99E9
:10C350006B1C0A9A42F020020A926A780B91FEF74F
:10C360001CBF5046414603F0D9FA002840F0FF8038
:10C37000B7F1FF3F00F051821698672814BF0023E1
:10C380000123472808BF43F0010313B1002F08BF62
:10C3900001270DF5AB60434652460A99C0E90023D8
:10C3A000DDF85C3541F480710A91002BC0F26482A3
:10C3B000002117911698662814BF002301234628F0
:10C3C00008BF43F001031093002B00F0D181BC465D
:10C3D0000323CDF830A00DF5AE61CDF8348048468A
:10C3E000009302910DF5AC61DDE90C230C31CDF821
:10C3F00004C003910DF5AD61CDF824C0049100F0A7
:10C40000C7FB169ADDF824C0B2F1670318BF0123F9
:10C41000472A0CBF002303F00103139033B90A9B92
:10C4200013F0010F08BFDDF868B516D01398109906
:10C4300000EB0C0B31B10378302B00F0DA80DDF823
:10C4400070359B44504600220023414604F078F9A1
:10C45000002800F0C281CDF868B5169A1398672AB3
:10C4600014BF00230123472A08BF43F00103C0EB98
:10C470000B001A90002B00F08A81DDF8701511F185
:10C48000030F109102DB8F4280F28C81169A023AE0
:10C4900016921099169A4B1ECDF87035002B8DF818
:10C4A0006025C0F234822B228DF86125092B00F320
:10C4B000B6810DF5AC62303304328DF8633530232C
:10C4C0008DF862350DF5AC631A981A99D31A1818BD
:10C4D0001C930129109040F31082109801301090A5
:10C4E00020EAE0710C911798002800F06E812D234E
:10C4F00000218DF877351791FEF774BF109A4FF031
:10C50000000C9DF8773522EAE272CDF85CC00C92FF
:10C51000FEF767BF0A9A12F0400F17BF0B980B9AED
:10C52000119900F1040A11BF036802F1040A1368AB
:10C53000119814BF19801860FEF7ECBD0B9A131DFB
:10C540000B93116801230A1E18BF01228A464FF07F
:10C55000000BFEF709BF0B98021D0B9201680A1E23
:10C5600018BF01228A464FF0000BFEF7FDBE42F2D3
:10C57000A86242F2A4631699C0F20103C0F201025C
:10C5800003204729D8BF1A4613920A9A0C9022F02A
:10C590008002CDF85CB00A929DF877351090FEF7D6
:10C5A00020BF0DF5A862484631460C32FEF73CFD2F
:10C5B00000287EF467AEFEF762BE0DF5A86248461D
:10C5C00031460C32FEF730FD00287EF45BAE0DF5EF
:10C5D0009C6304336AE60DF5A862484631460C3286
:10C5E000FEF722FD00287EF44DAE0DF59C6304336A
:10C5F00079E65046002200234146CDF824C004F0DD
:10C600009FF8DDF824C000287FF419AFCCF10103B6
:10C61000CDF8703515E70F9A52420F92FFF787B8A1
:10C620000DF5A862484631460C32FEF7FDFC0028A5
:10C630007EF428AE0DF59C630433FFF793BA0DF535
:10C64000A862484631460C32FEF7EEFC00287EF424
:10C6500019AE0DF59C6304331A9913985960DDF8EF
:10C660005025DDF85415186001321A98CDF8502580
:10C670000918072ACDF854153FF746AB0833FEF7E3
:10C68000A8BF00211791FDF725F99DF8773520EA1D
:10C69000E07210900C92FEF7A4BE2A4645469046E2
:10C6A0005F60DDF85025DDF854150132C3F80080D5
:10C6B000C919072ACDF85415CDF85025BFDC083329
:10C6C000CAE7189A1399511A1091FEF782BE48468C
:10C6D000314600F049F900287EF4D8ADB6F80CC018
:10C6E0001FFA8CF3FEF7F6BC062F28BF062742F28E
:10C6F000C061C0F2010127EAE772109713910C9212
:10C70000FEF7E8BF0DF5A862484631460C32FEF749
:10C710008BFC00287EF4B6AD0DF59C630433FFF767
:10C72000C8BB0DF5A862484631460C32FEF77CFCCA
:10C7300000287EF4A7AD0DF59C630433FFF7CEBA55
:10C740000DF5A862484631460C32FEF76DFC002814
:10C750007EF498AD0DF59C640434FFF7A9BA1097E8
:10C7600027EAE77717900C979DF87735FEF739BEE3
:10C770001699652914BF00230123452908BF43F0FA
:10C780000103002B46D007F1010C022321E6169B82
:10C79000652B76DD169A662A1CBFDDF8703510937E
:10C7A00000F083801A9B109883426EDC0A9911F086
:10C7B000010F40F08E8020EAE07267230C921693FE
:10C7C00091E600271D46FEF7E9BC10999DF87735E4
:10C7D00021EAE1710C91FEF704BEDDF868359B4556
:10C7E00098BF9B467FF639AE302203F8012B9B455C
:10C7F000CDF86835F9D830E60DF5A86248463146DF
:10C800000C32FEF711FC00287EF43CAD0DF59C6364
:10C81000043308E5BC460233DBE50737B9E546F2E9
:10C82000676C0DF590610331C6F2666C8CFB0320DA
:10C83000DA17C2EBA00202EB8200A3EB4000134622
:10C840003030092A01F8010DF0DC3033481EDAB22D
:10C8500001F8012C079B83426AD90DF5AC630333C1
:10C8600001E011F8012B03F8012C1A46DDF81CC079
:10C8700001338C45F5D825E62D2208F100481792A2
:10C8800098E5DDF87005109003E6109B1A99002BCF
:10C89000DABF1098C0F1020301235B1867221093DE
:10C8A00023EAE37316920C931DE6DDF87005002869
:10C8B000109031DD1FB90A9911F0010F0ED01098B8
:10C8C00066211691431CDB19109323EAE3720C9244
:10C8D00009E61098672116910130109020EAE07265
:10C8E0000C9200E60B991A780F6804310B91002F17
:10C8F000B8BF4FF0FF37FEF750BC0A9A12F0010F95
:10C9000004BF20EAE0730C933FF4EDADE5E52D2282
:10C910005B428DF86125C9E577B90A9B13F0010FD9
:10C920000AD14FF0010CCDF830C0CDF840C0DAE5A7
:10C930000DF5AC620232C5E50237662127EAE772DF
:10C94000109716910C92CEE5DC26010010B440F24F
:10C950004004C1F200048C4613460146624620683A
:10C9600010BCFEF76FBB00BF70B540F24005C1F2CE
:10C97000000506460C46286810B18369002B36D0A6
:10C9800042F2FC63C0F201039C4238D042F21C73B5
:10C99000C0F201039C4241D042F23C73C0F2010359
:10C9A0009C4204BF2B68DC68A289114693B213F045
:10C9B000080F184618BF226933D01AB313F00101CB
:10C9C00007D063690021A1605B42A36142B10020EE
:10C9D00070BD13F0020F08BF6169A160002AF6D193
:10C9E000A38913F0800FF2D04FF0FF3070BD01F03B
:10C9F0008BF942F2FC63C0F201039C42C6D12B6862
:10CA00005C68D1E703F42071B1F5007FD6D03046E1
:10CA1000214601F001FDA3892269CFE72B689C68BC
:10CA2000C2E713F0100FDFD013F0040F08BF226924
:10CA300017D0616B51B104F14403994203D03046E1
:10CA400001F0E6F9A28990B20023636322694FF6F0
:10CA5000DB71C0F20001002300EA01016360A181E3
:10CA6000226041F00803A3819BB2A6E7000000000A
:10CA70002DE9F84F03690E69824689469E4200F30C
:10CA80008380F21C01F1140500F11404013E9200B0
:10CA90008B18121803F10408596850680131FCF72B
:10CAA00003FB0746002839D000239C461A46E95864
:10CAB000E0581FFA81FE4FEA114B81B20EFB07CE00
:10CAC00051180BFB07FC0CEB1E4C1FFA8EFECEEB35
:10CAD00001011FFA8CF24FEA1C4CC2EB10421FFA04
:10CAE00081FE02EB21424EEA0241E150043312146E
:10CAF00059198845DBD2321D0AEB8203596869B99E
:10CB00009C4209D25AF8222012B105E01A681AB9DB
:10CB1000043B013E9C42F9D3CAF810604946504696
:10CB200002F0B6F800282CDB002301379C46EA58B7
:10CB3000E05891B2120C1FFA80F9C2EB1042C1EB1F
:10CB40000901614402EB214289B241EA0241E1500C
:10CB500004334FEA224C5A199045E8D2321D0AEBB1
:10CB60008203596869B99C4209D25AF8222012B14D
:10CB700005E01A681AB9043B013E9C42F9D3CAF891
:10CB800010603846BDE8F88F0020BDE8F88F00BF80
:10CB90002DE9F04F466AA1B00446904699462D9D76
:10CBA000002E00F02384326882B1616A4FF0010CDC
:10CBB000766820460B6856604A6819460CFA02F2FD
:10CBC0009A6002F09FF9636A00221A60B9F10006C8
:10CBD00038DB00232B6040F20003C7F6F0731A46DF
:10CBE00006EA0303934217D0002200234046494639
:10CBF000CDE9068903F0A4FD002829D02C98012353
:10CC00002E990360002900F0D080794B581E2E9A8F
:10CC1000136021B0BDE8F08F2C9842F20F730360CF
:10CC2000B8F1000F00F0958042F2F860C0F2010008
:10CC30002E990029EDD0C278C31C002AE7D000F15C
:10CC40000803E4E726F000460123B1462B60C2E763
:10CC50002046DDE906231EA900911FA9019102F0DB
:10CC6000A3F9C6F30A558346002D7ED0DDE90601FF
:10CC7000A5F57E751F9F073D21F07F4323F47003C8
:10CC800043F07E51002341F4E001199340F2000388
:10CC90000022C3F6F87303F037F94FA3D3E900235A
:10CCA00003F0E6FA4EA3D3E9002303F02FF9CDE910
:10CCB0000801284603F076FA4BA3D3E9002303F0DA
:10CCC000D7FA02460B46DDE9080103F01FF9CDE96A
:10CCD000080103F067FD002200230646DDE9080194
:10CCE00003F038FD40B1304603F05CFADDE908237B
:10CCF00003F026FD00B9013E162E5BD901231893DF
:10CD0000013FB7EB050A42BFCAF1000ACDF83CA0CB
:10CD10004FF0000A01D400220F92002EC0F271835E
:10CD2000B2440023179615932A9B092B62D8052B32
:10CD300040F377862A98002704382A902A998B1E78
:10CD4000032B00F2DD83DFE813F0A503D803D5033E
:10CD5000C40326F07F4626F47006002E7FF464AFED
:10CD600042F2EC60C0F2010062E71F9F1E9BFB18BD
:10CD700003F586639D1C202DDCBFC5F1200008FA59
:10CD800000F008DD1E3BC5F1400216FA02F228FA57
:10CD900003F342EA030003F0F5F9A5F586650122E5
:10CDA000033D1992A1F1F87170E742F2C860C0F238
:10CDB00001002EE742F2A873DDE90601C0F201038B
:10CDC00003EBC603D3E9002303F0C4FC002840F0C2
:10CDD0002083189094E700BF61436F63A787D23F19
:10CDE000B3C8608B288AC63FFB799F501344D33F5A
:10CDF000C926010000234FF0FF301F4601212A936E
:10CE00001190169108902B93656A00236B60204661
:10CE1000696802F093F8636A28601B681093002F1A
:10CE200000F05B81002E40F32A8442F2A87306F0E2
:10CE30000F02C0F20103351103EBC20315F0100F0E
:10CE4000D3E90001CDE90C0100F0E78242F680034E
:10CE5000DDE90601C0F2010305F00F054FF00308FC
:10CE6000D3E9082303F02EFBCDE91201BDB142F650
:10CE70008007DDE90C23C0F2010715F0010F104611
:10CE8000194607D0D7E9002308F1010803F0F0F9AB
:10CE900002460B4608376D10EFD1CDE90C23DDE9D2
:10CEA0000C23DDE9120103F00DFBCDE90C0118990B
:10CEB000002900F0DE8040F20003DDE90C010022D1
:10CEC000C3F6F0734FF0000503F044FC08B14FF0D7
:10CED0000105089A002AD4BF002505F00105002DA0
:10CEE00000F0C780119B002B40F3F58040F2000357
:10CEF0000022C4F22403DDE90C0103F0B9F9CDE905
:10CF00000C0108F10100711E129103F04BF9024669
:10CF10000B46DDE90C0103F0ABF940F200030022FF
:10CF2000C4F21C0302F0F2FFDDF844C08046A1F118
:10CF30005079169B002B00F0AD8342F2A87340F2AB
:10CF40000001C0F20103002003EBCC03C3F6E07143
:10CF5000CDF80CC053E9022303F0B4FA42464B4625
:10CF6000109D02F0D1FF80468946DDE90C0103F0F7
:10CF700019FC074603F016F902460B46DDE90C01E1
:10CF800002F0C2FF07F13003CDE90C01404605F87D
:10CF9000013B4946DDE90C2303F0FAFB002840F091
:10CFA000138240F20001DDE90C230020C3F6F0718A
:10CFB00002F0AAFF02460B464046494603F0E8FB52
:10CFC000DDF80CC0002840F0E783BCF1010F40F30E
:10CFD0008280CDF868B00127CDF870A01D96664616
:10CFE000DDE90CAB0C9410E040F200010020C3F628
:10CFF000F07102F089FF42464B4603F0ABFB00287C
:10D0000040F0C783B74280F28B8440F20003404671
:10D0100049460022C4F22403013503F029F940F205
:10D0200000030022C4F22403804689465046594634
:10D0300003F01EF98B46824603F0B4FB044603F06E
:10D04000B1F8303402460B465046594602F05CFFB8
:10D05000109A4B46D4554246013782468B4603F020
:10D0600079FB52465B460028BED0DDF868B00C9CC8
:10D07000AAE1404603F096F8DDE90C2303F0F8F846
:10D0800040F200030022C4F21C0302F03FFF089AA2
:10D09000A1F150758046A946002A40F0EC8240F28A
:10D0A0000003DDE90C010022C4F2140302F02CFF9E
:10D0B00042462B46CDE90C0103F06AFB002840F004
:10D0C0004A824246DDE90C0105F1004303F042FBD0
:10D0D000002840F0D581DDE906891E9B6FEA030731
:10D0E0004FEAD7770E2ECCBF002707F00107002F9D
:10D0F00000F0B7802B9842F2A873C0F201030899A0
:10D1000003EBC603C20F0029CCBF002202F00102CC
:10D11000D3E90001CDE90401002A40F0A0810246D4
:10D120000B464046494603F0CDF9109D03F03AFB0B
:10D13000824603F037F8DDE9042303F099F802464C
:10D140000B464046494602F0DFFE0AF1300305F87F
:10D15000013B089A012A8046894652D040F20003DA
:10D160000022C4F2240303F083F800220023CDE957
:10D17000060103F0E5FA002840F0EB8110984FF02B
:10D180000108CDF82CB0A346871C0F96DDF820903F
:10D19000DDE906450AE003F06BF8002200230446AF
:10D1A0000D4603F0CDFA002840F0CE81DDE90423DE
:10D1B0002046294608F1010803F084F93E4603F0B1
:10D1C000F1FA824602F0EEFFDDE9042303F050F8A5
:10D1D00002460B462046294602F096FE00220AF13E
:10D1E000300C07F801CC0137C14540F20003C4F20E
:10D1F0002403D0D135465C460F9E8046DDF82CB026
:10D20000894642464B464046494602F07FFE8046EC
:10D2100089464246DDE904014B4603F09BFA60B9BA
:10D22000DDE9040142464B4603F08AFA002800F08B
:10D2300090811AF0010F00F08C81109900E01D46DA
:10D2400015F8012C6B1E392A40F067838B42F6D10A
:10D2500010993023013631220B70109B1A701296F0
:10D26000B2E0169A002A40F0DF80159F0F9D0C92C5
:10D27000002DD4BF00230123BAF1000FD4BF002337
:10D2800003F001034BB1AA45B4BF53462B460F9898
:10D29000C3EB0A0AED1AC01A0F90159900291CDD7C
:10D2A000169A002A00F0E982002F12DD0C993A4606
:10D2B000204602F0A3F85A460C9020460C9901F043
:10D2C000B5FF594603462046039301F01BFE039B1E
:10D2D0009B46159BDA1B40F011830121204602F08A
:10D2E0003FF806901798002805DD06992046179A02
:10D2F00002F084F806902A99012940F30A81002758
:10D30000179B002B40F061820123534413F01F034D
:10D3100040F02A811C230F9A9A44ED18D2180F92DC
:10D320000F9B002B05DD59461A46204601F020FFD1
:10D330008346BAF1000F05DD06995246204601F0FA
:10D3400017FF06901898002840F029822A9808991B
:10D350000228D4BF002301230029CCBF002303F0FF
:10D360000103002B00F00C81002940F08C80052285
:10D370000699089B204601F0FDFF06905846069945
:10D3800001F086FC00287EDD109D01360027DDF8C7
:10D3900030A0312305F8013B0699204601F0B2FD8B
:10D3A000BAF1000F00F0D5803B1E18BF012357458E
:10D3B0000CBF002303F00103002B40F0D080514646
:10D3C000204601F09FFD12962046594601F09AFD35
:10D3D000129A531C00222A702C982E99036000295F
:10D3E00000F0D4812E9A1098156012E4102001F0FC
:10D3F00089F8C66046608660066006466062FFF790
:10D40000D2BB0F98714200221591801B17920F908A
:10D410008AE40021013E189172E4DDE906234FF011
:10D420000208CDE9122321E52A98012840F36C82F5
:10D43000089A1598531E9842C0F25882C71A089B42
:10D44000002BA8BF0F9DC0F273820F9A20460121C6
:10D450009A44D2180F9201F083FF0C9008E7089BC2
:10D4600073B940F200030022C4F21403DDE90401A1
:10D4700002F0FEFE42464B4603F080F900286AD0D7
:10D48000002206920C922B9B0027DDF830A0DE4391
:10D49000109D81E7002116912B98002840F39F8171
:10D4A0002B98014611900890656A002217296A603E
:10D4B00040F2AB8204235B00013203F11400884286
:10D4C000F9D9089B6A600E2B8CBF002707F0010773
:10D4D0009DE4012216922B9BF3181193591C0029ED
:10D4E000C8BF0891E0DC0E298CBF002707F00107B8
:10D4F000089189E401231693CEE700221692EAE709
:10D500004FF0FF33002701201193169008932B97BB
:10D510007AE4B8F1000F7FF4F2AE29F07F4323F4F0
:10D520007003002B7FF4EBAE40F20003C7F6F073FC
:10D5300009EA0303002B3FF4E2AE0F9A0AF1010A55
:10D54000012701320F92DBE635465C460F9EDDF87F
:10D550002CB0129638E7002006900C9014E739465C
:10D56000204601F0CFFC2AE7C3F12003042B40F34F
:10D5700054820F99043B9A44ED18C9180F91CFE6D5
:10D580001699002900F03181002D05DD0C992A46FD
:10D59000204601F0EDFD0C90002F40F0EA81DDF80F
:10D5A00030A0109D012308F001000C9F11900F95F1
:10D5B0001D460C9606995846FFF75AFA3946303000
:10D5C0000B90584601F064FB0699524606462046E9
:10D5D00001F052FDC3688046002B3DD04FF0010999
:10D5E0004146204601F08EFC2A9959EA010103D1F7
:10D5F000119A002A00F0EB81002EC0F29E812A9A37
:10D60000324303D1119B002B00F09781B9F1000F39
:10D6100000F3CE810F990B9A01F8012B089B0F9113
:10D620009D4200F0C28159460A220023204601F0A3
:10D63000A1FE57453946834614D00A2200232046CE
:10D64000013501F097FE51460A2200230746204685
:10D6500001F090FE8246ADE75846414601F018FBC6
:10D660008146BDE720460A220023013501F082FEF3
:10D67000074682469EE71296DDF820C059E47542BF
:10D68000002D40F00181DDE906014FF00208CDE9EF
:10D690000C010CE442F2A8714246C0F201014B4673
:10D6A00001EBCC01CDF80CC0109D51E9020102F054
:10D6B000DFFDCDE91A01DDE90C0103F073F807463F
:10D6C00002F070FD0B460246DDE90C0102F01CFC85
:10D6D00007F13003CDE90C0105F8013BDDF80CC082
:10D6E000BCF1010F29D0D146DDE90C01B246109EF4
:10D6F0001C9501276546A04640F200030022C4F2B3
:10D70000240302F0B5FDCDE90C0103F04BF804460B
:10D7100002F048FD303402460B46DDE90C0102F010
:10D72000F3FBF4550137AF42E6D11C9D013F56464D
:10D730004446CA46ED19CDE90C0140F2000300222F
:10D74000C3F6E073DDE91A0102F0E0FB02460B4686
:10D75000DDE90C0103F01CF8F0B940F20001DDE94D
:10D760001A230020C3F6E07102F0CEFB02460B46FE
:10D77000DDE90C0102F0EEFF00283FF4ACAC2B46D3
:10D780001D4613F8012D302AFAD01DE61098FFF738
:10D7900040BADDF868B00C9C129E109950E55846CE
:10D7A000069901F075FA0028BFF6D0AD594620461B
:10D7B0000A22002301F0DEFD1699013E834600296E
:10D7C00040F01981119A0892C0E50698036900EBB0
:10D7D0008303186901F00AFAC0F1200395E50121DD
:10D7E000119108912B91FFF70FBB109DB146169F29
:10D7F000AA46DDF81880089E02E001F0BBFD8346D2
:10D8000041465846FFF734F901350A2200235946AC
:10D8100000F1300C0AF807C001372046BE42ECDCAC
:10D82000DDF830A04E460027CDF82CC05946012225
:10D83000204601F09DFC0699834601F029FA002854
:10D840000FDD109900E01D4615F8012C6B1E392ADA
:10D8500040F08C808B42F6D11099312301360B7049
:10D860009AE503D10B9810F0010FEAD12B461D4623
:10D8700013F8012D302AFAD08EE55946159A204624
:10D8800001F0BCFD834628E505F00F0342F2A872C3
:10D89000C0F20102DDE9060102EBC303D3E9002374
:10D8A00002F0E6FC2D1108BF4FF00208CDE90C0193
:10D8B0003FF4FDAA42F68007DDE90C234FF0020891
:10D8C000C0F2010715F0010F1046194607D0D7E93D
:10D8D000002308F1010802F0CBFC02460B46083792
:10D8E0006D10EFD1CDE90C23FFF7E1BA1599179A26
:10D8F0005B1AC918D21815911792A0E5594620460F
:10D9000001F07CFD8346E8E41999002947D003F52E
:10D910008663159F03330F9D97E50132D2B29DE4D4
:10D92000DDF868B0DDF870A01D9E0C9CFFF7D3BB3E
:10D930000F99002308980D1A87E5B9F1000F0F9D84
:10D940000C9E0FDD59460122204601F011FC06997C
:10D95000834601F09DF9002847DD0B99392931D024
:10D9600001310B910B9A05F8012B15E501321A7064
:10D9700012E50C9A2046516801F0E0FA0C9B03F185
:10D980000C011A690232920005460C30FBF7C8FC04
:10D9900020462946012201F0EBFB824601E61F9B4F
:10D9A000159F0F9DC3F136034FE50F9D0C9E3DE77C
:10D9B0000B9B0F9D392B0C9E04D00B98431C05F834
:10D9C000013BE9E4392305F8013B10993CE70B984A
:10D9D00033460F9D39280C9EF4D0002B01DD013019
:10D9E0000B900B9905F8011BD6E4BBD10B9810F0F6
:10D9F000010FB7D0B1E700230C9920460A2201F0AD
:10DA0000B9FC119B08930C90A0E408990E298CBFD7
:10DA1000002707F00107FFF7FAB93FF481AC1C3388
:10DA200079E40127FFF78AB90B692DE9F0410C462B
:10DA30008046002B71D010B18369002B78D042F260
:10DA4000FC63C0F201039C4208BFD8F8044010D028
:10DA500042F21C73C0F201039C4208BFD8F8084090
:10DA600007D042F23C73C0F201039C4208BFD8F8D1
:10DA70000C40A3891AB212F0080F35D1626843F442
:10DA80000063A381002A5EDDE66A002E45D09BB2CA
:10DA900013F4805218BF656D59D013F0040F4AD1AA
:10DAA00000234046216A2A46B047854238D1A189E1
:10DAB0004FF2FF732269C0F2000301EA0303002161
:10DAC000616013F4805F616BA381226018BF65659C
:10DAD00019B304F14403994202D0404600F098F98A
:10DAE00000206063BDE8F0812669B6B12568266034
:10DAF000AD1B12F0030F0CBF63690023A3600AE0A3
:10DB000032462B46A76A4046216AB8470028C0EB38
:10DB10000505064404DD002DF2DC0020BDE8F0819F
:10DB2000A3894FF0FF3043F04003A381BDE8F081AB
:10DB300000F0EAF883E76268636BAD1A002BAFD0A0
:10DB4000236CED1AACE7226C002A9DDCE5E701238B
:10DB50004046216AB047B0F1FF3F054602D0A38995
:10DB6000E66A9AE7D8F800301D2BD6D0A38943F097
:10DB70004003A381BDE8F081014628B140F2400393
:10DB8000C1F2000318684FE742F25C734DF6292199
:10DB9000C0F20103C0F20001186800F0B3BB00BF7F
:10DBA000704700BF704700BF704700BF704700BF9D
:10DBB000002070470020704740F240034DF6B53119
:10DBC000C1F20003C0F20001186800F0C5BB00BF3D
:10DBD00040F240034DF6B131C1F20003C0F2000142
:10DBE000186800F0B9BB00BF4FF63951C0F2000110
:10DBF00000F0B2BB42F25C73C0F201031868F3E7B5
:10DC000010B5044600235C30A1811946E281082248
:10DC100023606360A360636623616361A361FBF7B4
:10DC200047FC4FF6CD104FF691114FF669124FF6A3
:10DC30006113C0F20000C0F20001C0F20002C0F2A5
:10DC400000036062A162E2622363246210BD00BF30
:10DC500070B568250E4605FB01F505F10C0100F0D5
:10DC600059FC044648B100F10C03002146602A46E5
:10DC700018462160A360FBF71BFC204670BD00BF67
:10DC800042F25C73C0F2010370B51D680646AB69D1
:10DC9000002B2AD0D8356B68AC68013B03D520E057
:10DCA0006834013B1DD4B4F90C20002AF8D10025BA
:10DCB0004FF0FF33656604F15C00E38129464FF0C5
:10DCC00001032560A3810822A56065602561656167
:10DCD000A561FBF7EDFBE5646563A563A5642046DC
:10DCE00070BD286828B10546D5E7284600F00CF835
:10DCF000D0E730460421FFF7ABFF28600028F2D1BF
:10DD00000C2304463360EAE770B58669044606B121
:10DD100070BD4DF6E9330125C0F20003C0F8D860AC
:10DD20008362C0F8DC60C0F8E0608561FFF7A8FF9F
:10DD300060602046FFF7A4FFA0602046FFF7A0FF29
:10DD4000324604212346E0606068FFF759FF2A4607
:10DD5000A06809212346FFF753FF2346E0681221FC
:10DD60000222BDE870404BE7F8B540F24414C1F21E
:10DD700000040F46054600F035FFA3685E6826F0F4
:10DD8000030606F57E630F33DF1B3F0B013F3F03A6
:10DD9000B7F5805F07DB0021284601F0CDFDA368C1
:10DDA000F318834204D0284600F01EFF0020F8BD7F
:10DDB0007942284601F0C0FDB0F1FF3F10D0A268C3
:10DDC00043F26C03C1F20003F61B46F0010628463D
:10DDD00056601A68D71B1F6000F006FF0120F8BDCF
:10DDE0000021284601F0A8FDA368C21A0F2ADADD37
:10DDF00040F24C5443F26C01C1F20004C1F2000144
:10DE000042F001022468001B08605A60CBE700BFA3
:10DE10002DE9F04105460C46002900F0888000F00D
:10DE2000E1FEA4F1080240F244105668C1F200007D
:10DE300026F00103D0F808C0D1188C454F6827F0B0
:10DE4000030700F0958016F001064F605FD00026B2
:10DE5000CC19646814F0010F06D1DB19002E7AD0BA
:10DE60008C68C9688C60E16043F00101D350516057
:10DE7000002E47D1B3F5007F5BD3590A04299EBF1A
:10DE80004FEA931C0CF1380C4FEACC0428D9142922
:10DE90009CBF01F15B0C4FEACC0421D954299EBFF1
:10DEA0004FEA133C0CF16E0C4FEACC0418D9B1F5D3
:10DEB000AA7F9EBF4FEAD33C0CF1770C4FEACC040B
:10DEC0000ED940F2545C614595BF4FEA934C4FF434
:10DED0007C740CF17C0C4FF07E0C98BF4FEACC04A4
:10DEE0000419A168A14203D164E089688C4204D07E
:10DEF000486820F003008342F7D3CB68D360916079
:10DF0000CA609A602846BDE8F04100F06DBE54F842
:10DF1000084C00F1080C121B1B199468644547D08B
:10DF2000D2F80CC0CCF80840C4F80CC090E7BDE8AB
:10DF3000F081DB084FF0010C466800EBC3019B1039
:10DF40000CFA03F3D1608C6846EA030343609460E3
:10DF5000E2608A60D6E78C681C4FBC4281D1D35006
:10DF600043F00103E260A26053609460D460C9E7AB
:10DF7000FB1816F0010F07D154F8081C521A5B1851
:10DF8000D4689168A160CC6040F250518260C1F2C7
:10DF9000000143F0010050600A689342B2D343F29B
:10DFA00068032846C1F200031968FFF7DDFEA9E700
:10DFB00001264DE7012644684FEAAC0C0B4606FAF1
:10DFC0000CFC44EA0C04446098E700BF4C010010CC
:10DFD0002DE9F04F936885B090460C460390002BD6
:10DFE00064D088891FFA80FA1AF0080F00F0A08028
:10DFF0000B69002B00F09C801AF0020BD8F800503F
:10E000001CBF4FF0000A574636D11AF0010A1DBF57
:10E01000DC46D9465F46564652D126B380B2A76841
:10E0200010F4007F00F08F80BE42BB4680F0A780D6
:10E0300020683746B3465A46514600F077FDA2683D
:10E040002368B146D71BA76037465B442360D8F8E6
:10E050000830C9EB0606CA44DF1BC8F808702FB3A6
:10E06000A089002EDAD1D5F800A06E680835D4E773
:10E07000D5F800A06F680835B7F5806F34BF3B4610
:10E080004FF4806352460398002FF1D0A66A216AAC
:10E09000B04700288244C0EB070740F3EC80D8F873
:10E0A0000830181AC8F808000028E5D1002005B08B
:10E0B000BDE8F08FD5F800904FF0000C6F68083580
:10E0C000002FF7D0BCF1000F00F0B5806369BB45AD
:10E0D00034BFDA46BA46A668206822699E19904283
:10E0E00094BF00220122B245D4BF002202F00102F7
:10E0F000002A40F0AE809A45C0F28280A66A4A4665
:10E10000CDF804C00398216AB047DDF804C0061EAC
:10E1100040F3B180BBEB060B00F08680D8F80830E6
:10E12000B144BF1B9E1BC8F80860002EC8D1BDE7D4
:10E1300003982146FEF718FC002840F0D480A089FF
:10E140001FFA80FA58E72068B9462369984294BFBD
:10E1500000230123B7422CBF002303F00103002B4F
:10E1600040F09D8063699E42C0F08C80A76A524651
:10E170000398216AB847071E7DDDB94667E710F4AA
:10E18000906F08BF20683FF456AF62692169236829
:10E1900002EB42095B1A09EBD97903F1010CB44493
:10E1A0004FEA6909E1454A463CBFE1464A4610F458
:10E1B000806F00F0838011460398029300F0AAF963
:10E1C000029B002800F099801A4621690293019071
:10E1D000FBF7A6F8A289029BDDF804C022F4906246
:10E1E00042F08002A281C3EB09020CEB0300374628
:10E1F000B346A260C4F810C02060C4F814901AE7B7
:10E20000524649465646CDF804C000F08FFCA2683D
:10E210002368BBEB060BCAEB0202DDF804C05344D3
:10E22000A26023607FF47AAF03982146FFF7FCFBDE
:10E2300008BBDC4672E748460A213A4600F03CFC3F
:10E2400000284BD000F1010B4FF0010CC9EB0B0B78
:10E250003CE749463246CDF804C000F067FC23682D
:10E26000214603989B192360FFF7DEFBDDF804C00D
:10E2700000283FF44FAFA3894FF0FF3043F0400335
:10E28000A38114E73246514600F050FCA26823688F
:10E290003746921BB1469B19A2602360D7E65146D0
:10E2A0003A4600F043FC236803982146DB192360BB
:10E2B000FFF7BAFB00283FF4CAAEDCE703980293ED
:10E2C00001F040F9029B844600288CD12169039813
:10E2D000FFF79EFD03990C230B60CCE707F1010BC0
:10E2E0004FF0010CF2E603990922A3894FF0FF30A9
:10E2F00043F040030A60A381D9E6039A0C2313601C
:10E30000B9E700BF2DE9F84507468A46FFF748FC04
:10E3100017F1D80608BFB04618D04FF0000875684E
:10E32000B468013D0FD4B4F90C304BB1B4F90E30E0
:10E3300021463846B3F1FF3F02D0D04748EA0008F3
:10E340006834013DEFD53668002EE8D1FFF72AFC8E
:10E350004046BDE8F88500BF2DE9F04106468846F5
:10E36000FFF71EFCD83608BF374615D00027756862
:10E37000B468013D0DD4B4F90C303BB1B4F90E30A2
:10E380002046B3F1FF3F01D0C04707436834013D49
:10E39000F1D53668002EEAD1FFF704FC3846BDE817
:10E3A000F08100BF42F26473C0F201031868704745
:10E3B000004870476827010000487047682701003F
:10E3C00070B505460E46144672B142F260711046B1
:10E3D000C0F2010101F00CFB58B942F260702C62EE
:10E3E000C0F20100EE6170BD42F26070C0F2010047
:10E3F00070BD42F298612046C0F2010101F0F8FAC6
:10E400000028EAD0002070BD40F240030A46C1F265
:10E41000000301461868D3E78B89F0B50C469AB221
:10E4200091B012F0020F054641D1B1F90E1000294A
:10E4300018DB01AA01F088FC002811DB029B03F421
:10E440007043B3F5005F14BF00270127B3F5004FF9
:10E4500040D0A3894FF4806643F40063A3810BE0AE
:10E46000A3899AB212F0800F43F400630CBF4FF4FB
:10E47000806640260027A3812846314600F04AF8EE
:10E4800070B1A1894DF6E932C0F20002206141F07D
:10E4900080016661AA62A18120607FB911B0F0BDE0
:10E4A000A38913F4007FF9D143F00203A38104F19F
:10E4B00047032361236001236361EFE72846B4F932
:10E4C0000E1001F057FC0028E8D0A38943F00103A7
:10E4D000A381E3E74FF66913E26AC0F200039A42B0
:10E4E000B7D1A2894FF480631E46236542EA030335
:10E4F000A381C1E740F240030146C1F2000318685E
:10E50000FFF786BC40F240030146C1F200031868E1
:10E5100000F000B82DE9F04F01F10B04162C83B088
:10E5200006462FD8002310248C422CBF194643F0F6
:10E530000101002930D1304600F054FBB4F5FC7FD6
:10E540002ED24FEAD40E40F24415C1F2000505EB7D
:10E55000CE02D368934200F006825A6803F10805A0
:10E56000D968304622F0030C9A6863445C688A607C
:10E5700044F00104D1605C6000F036FB284603B033
:10E58000BDE8F08F24F00704E30F8C422CBF19463E
:10E5900043F001010029CED00C2300253360EDE7C4
:10E5A0005FEA542E04BF4FEAD40E4FEACE0040F08B
:10E5B000908040F24415C1F200052818C3689842C3
:10E5C00006D10DE0002A80F26F81DB68984207D007
:10E5D000596821F003010A1B0F2AF3DD0EF1FF3EFB
:10E5E0000EF1010E40F24417C1F2000707F10801D5
:10E5F0008B68994208BF7A6826D05A6822F0030CCB
:10E60000C4EB0C020F2A00F39481002AC9608960D0
:10E6100080F29980BCF5007F80F065814FEADC0CC8
:10E620004FF0010A7A6807EBCC004FEAAC0C0AFA0B
:10E630000CFCD860D0F808804CEA02027A60C3F87B
:10E640000880C8F80C3083604FF0010C4FEAAE032D
:10E650000CFA03FC944500F2828012EA0C0F08D1F8
:10E660002EF0030E4FEA4C0C0EF1040E12EA0C0FC2
:10E67000F8D007EBCE09F246C846D8F80C309845DA
:10E6800007D168E1002A80F27881DB68984500F0C4
:10E690006281586820F00300021B0F2AF2DD1D463C
:10E6A0001F19D3F80CC044F0010E55F8084F30463E
:10E6B000BA5042F00102C3F804E0CCF80840C4F8B4
:10E6C0000CC08F60CF607A60B960F96000F08CFA9E
:10E6D00054E7BEF1040F9EBF4FEA941E0EF1380EB0
:10E6E0004FEACE007FF665AFBEF1140F9CBF0EF16E
:10E6F0005B0E4FEACE007FF65CAFBEF1540F9EBFBB
:10E700004FEA143E0EF16E0E4FEACE007FF651AF87
:10E71000BEF5AA7F9EBF4FEAD43E0EF1770E4FEAB8
:10E72000CE007FF646AF40F254539E4595BF4FEA68
:10E73000944E4FF47C700EF17C0E4FF07E0E98BF1D
:10E740004FEACE0035E703EB0C0203F10805304633
:10E75000536843F00103536000F046FA0EE7D7F820
:10E760000880D8F8043023F00309C4EB09024C45B3
:10E7700094BF002301230F2AD8BF43F00103002BCD
:10E7800000F0A18043F2680BD5F80824C1F2000B19
:10E79000DBF8003010331B19B2F1FF3F06D003F550
:10E7A0007E631F3323F47E6323F01F031946304634
:10E7B000019301F0C1F8019BB0F1FF3F824600F0E8
:10E7C000F48008EB0901814200F2EC80DBF80420C0
:10E7D0009A185145CBF8042000F04581D5F808542B
:10E7E00040F24410C1F20000B5F1FF3F08BFC0F88D
:10E7F00008A403D05244511ACBF804101AF00705AC
:10E80000304617BFC5F108054FF48055AA4405F5F9
:10E81000805553441B051B0DED1A294601F08CF859
:10E82000B0F1FF3F00F02C81CAEB0001491941F023
:10E830000101DBF8042043F26803C7F808A0C1F225
:10E840000003AA18B845CBF80420CAF8041017D062
:10E85000B9F10F0F40F2DF80A9F10C01052521F07D
:10E86000070108EB01000F2985604560D8F8040016
:10E8700000F0010041EA0000C8F8040000F2AC809A
:10E88000D04643F26803DBF82C10C1F200038A4241
:10E89000DBF8301088BFDA6243F26803C1F200038C
:10E8A0008A4288BF1A6382E05C189A68D968304649
:10E8B000666803F108058A6046F00103D160636071
:10E8C00000F092F95AE608EB040342F0010244F02A
:10E8D00001043046C8F8044008F108055A60BB60DE
:10E8E00000F082F94AE64FEA5C22042A54D9142A3D
:10E8F00000F289805B324FEAC208A84440F2441714
:10E90000C1F20007D8F80800404503D16FE08068E5
:10E91000804504D0426822F003029445F7D3D0F832
:10E920000CC0C3F80CC098607A68C360CCF808309B
:10E930008AE61F19304644F00104CF605C6003F1A1
:10E940000805BA5042F001028F607A60B960F96040
:10E9500000F04AF912E60AF1010A1AF0030F5FD03B
:10E9600003F1080889E603F10802D3689A4208BF58
:10E970000EF1020E3FF436AEEFE51D461918DA68C7
:10E98000304655F8083F4C68936044F00104DA6063
:10E990004C6000F029F9F1E54FEA9C1238324FEA59
:10E9A000C208AAE7B8453FF411AFD7F80880D8F8F5
:10E9B000042022F00302944294BF00230123121B7F
:10E9C0000F2AD8BF43F00103002B3FF47CAF304641
:10E9D000002500F009F9D1E508F10801304601935E
:10E9E000FFF716FA019BD7F808805A6849E74FF0FD
:10E9F000010AD7F80480921084460AFA02F248EA23
:10EA000002027A608DE7542A24D84FEA1C326E3213
:10EA10004FEAC20871E70123D046CAF80430C6E7BE
:10EA20004A461EF0030F13460EF1FF3E33D053F853
:10EA300008299A42F5D07B684FEA4C0C9C453FF67A
:10EA40008EAEBCF1000F3FF48AAE1CEA030F27D054
:10EA5000D6460EE6B2F5AA7F15D84FEADC327732F9
:10EA60004FEAC20849E70805000D00287FF4B6AE5A
:10EA7000D7F808804B4443F00103C8F8043000E79E
:10EA800001210025D5E640F2545082420DD94FF4C1
:10EA90007C787E2231E77B6823EA0C037B60CBE73E
:10EAA0004FEA4C0C0AF1040ACFE74FEA9C427C3251
:10EAB0004FEAC20821E700BF10F0030FC9B210B43B
:10EAC00010D0002A2FD003788B422AD0013A05E0DB
:10EAD000002A28D00378013A8B4222D0013010F06E
:10EAE000030FF5D1032A11D941EA012444EA044471
:10EAF000036884EA0303A3F1013C2CEA030313F047
:10EB0000803F03D1043A0430032AF1D85AB1037884
:10EB10008B4206D0013A32B110F8013F013A8B42E4
:10EB2000F9D110BC70470020FBE700BF88428C463B
:10EB300070B4054614460ED98B1898420BD242B1D8
:10EB4000C2EB030C0146531E1CF80320CA54013BC0
:10EB5000FAD270BC70470F2A09D8002CF9D00023D4
:10EB60001CF80320EA540133A342F9D1F1E741EA4A
:10EB7000000313F0030FF0D194460C4603462568BA
:10EB8000ACF1100C1D6065685D60A5689D60E5686E
:10EB90001034DD601033BCF10F0FF0D8103A4FEA9B
:10EBA000121C0CF10105CCEB0C7C2D0102EB0C16B8
:10EBB00001EB050C4519032E3446CED900235CF831
:10EBC0000320EA500433F21A032AF8D8043EB308AB
:10EBD0005A1CC3EB83739200944406EB8304AD1874
:10EBE000BBE700BF704700BF704700BF020C034681
:10EBF0001204B2B1002013F07F4F01D108301B0284
:10EC000013F0704F01D104301B0113F0404F01D1BC
:10EC100002309B00002B03DB13F0804F04D0013047
:10EC2000704703041020E6E720207047036802467F
:10EC300013F0070009D013F0010F21D113F0020FD8
:10EC400022D19B0802201360704799B209B91B0CAE
:10EC5000102013F0FF0F01D108301B0A13F00F0F23
:10EC600001D104301B0913F0030F01D102309B08BE
:10EC700013F0010F02D15B0804D00130136070471C
:10EC800000207047202070475B0801201360704708
:10EC900003460A69006910B4801A11D1043203F1E5
:10ECA000140C92009B1889180431043353F8044C57
:10ECB000043B51F8042C0439944203D19C45F5D30C
:10ECC00010BC704738BF4FF0FF30F9D30120F7E791
:10ECD00040F20003C7F6F07301EA0303A3F1507397
:10ECE000002B02DD1946002070475B421B15132BD9
:10ECF0000EDD143B1E2B03DD012300211846704757
:10ED00000122C3F11F03002112FA03F318467047D2
:10ED10004FF40022002052FA03F170472DE9F04130
:10ED2000046900F114060F46043450F8245000EB37
:10ED30008404A0462846FFF759FF0A28C0F12003A3
:10ED40003B6014DCA642C0F10B0337D254F8041C1C
:10ED5000D94025FA03FC15304CF07E53854043F42E
:10ED6000E00341EA050210461946BDE8F081A642DB
:10ED700020D300210B3802BF45F07E530A4643F4EE
:10ED8000E003F0D0B442C0F1200319D954F8044C88
:10ED9000DC40854021FA03FC45F07E5511FA00F075
:10EDA00045F4E00544EA000245EA0C031046194622
:10EDB000BDE8F08154F8041C043CDBE70021C8E7FF
:10EDC0000024E6E72DE9F04383B00E4601A907468B
:10EDD000FFF7A4FF0D46044669463046FFF79EFF45
:10EDE000DDF804C0A946A0460B4602463169164626
:10EDF00038691F46401A0099C1EB0C0101EB401124
:10EE00000029C9BF05EB0159A3EB015724464D4624
:10EE1000DCBF12463B462046294601F053FB03B0B7
:10EE2000BDE8F083172810B504460EDD40F200015E
:10EE30000020C3F6F07140F200030022C4F2240364
:10EE400001F016FA013CF6D110BD42F2A873C0F2EF
:10EE5000010303EBC003D3E9000110BD13690139BD
:10EE600002F1140C10B402EB83024C111432013481
:10EE7000944500EB84040FD200235CF80310C150CA
:10EE8000043303EB0C018A42F7D86FEA0C0C62449E
:10EE900022F0030204328018844204D9002340F88F
:10EEA000043B8442FBD810BC704700BF02694B1181
:10EEB0009A4210DB0EDD11F01F010BD01A4600EB59
:10EEC00083035B6923FA01FC0CFA01F1994202D039
:10EED000012070471A46043200F1140100EB82034E
:10EEE00003F1040C61450BD250F82220002AEFD127
:10EEF000994205D253F8042D002AE9D19942F9D359
:10EF00000020704730B5456A83B0044655B139B129
:10EF1000636A4A68DB6853F82200086043F82210ED
:10EF200003B030BD10200191FFF7ECFA0199606247
:10EF3000C560456085600560E9E700BF70B5446A5B
:10EF400006460D4664B1E268A2B152F82530EBB135
:10EF5000196842F825100022DA601A61184670BD5F
:10EF60001020FFF7CFFA002304467062C3604360AD
:10EF70008360036010223046042100F03DFE736A76
:10EF8000E060DA68002AE0D11346E7E70124304662
:10EF90002146AC40621D920000F02EFE0346002880
:10EFA000DCD045608460D6E72DE9F04583B00121CF
:10EFB0001D4614460A9F0B9EFFF7C0FF25F0004236
:10EFC00025F07F4323F4700315465FEA125A00933D
:10EFD0001CBF43F4801300938046002C23D002A86A
:10EFE00040F8044DFFF722FE0346002837D101996F
:10EFF000009AC8F81410002A14BF02240124C8F88B
:10F000001820C8F81040BAF1000F1BD0AAF5866A84
:10F01000C3F13502AAF1030A53443B603260404613
:10F0200003B0BDE8F0856846FFF700FE01231C46EB
:10F03000C8F81030009BC8F8143000F12003BAF172
:10F04000000FE3D108EB8402A3F58663023B3B602B
:10F050001069FFF7CBFDC0EB44103060DFE7009A8A
:10F06000C0F1200112FA01F1C24001980143C8F831
:10F0700014100092BFE700BF2DE9F84F13690F6924
:10F080000C461546FF1A002F4FD06ADB002701F10E
:10F0900014066168FFF752FFD5F81080D4F810C04D
:10F0A00005F11401002205EB880504EB8C0405F141
:10F0B0001408143400F11403C76051F8047B56F8A7
:10F0C000045BBB461FFA87FA3F0C1FFA85F9C7EBB2
:10F0D0001547CAEB090A524407EB224792B242EAAB
:10F0E000074243F8042B3A148845E6D8A6420ED2CC
:10F0F00056F8041B8DB2090C521901EB224192B251
:10F1000042EA014243F8042B0A14B442F0D853F8FF
:10F11000042C32B953F8082C0CF1FF3C043B002AB4
:10F12000F8D0C0F810C0BDE8F88F043301F1140620
:10F130009B00D218CB180433043253F804CC043BA0
:10F1400052F8041C043A8C450AD19E42F5D30021A2
:10F15000FFF7F4FE0123036100234361BDE8F88F4C
:10F1600097D223462C4601271D4604F1140690E74A
:10F170002DE9F8450D698B68561101350C46AD191E
:10F1800090469D428246496803DD5B0001319D4205
:10F19000FBDC5046FFF7D2FE002E074600F11402BA
:10F1A0000ADD0023194642F823100133B342FAD195
:10F1B00007EB830303F11402206904F1140304EB49
:10F1C0008000143018F01F081BD0C8F1200E002159
:10F1D0001E6806FA08FC41EA0C0142F8041B53F8C9
:10F1E000041B984221FA0EF1F2D8116001B10135E9
:10F1F0005046013D21463D61FFF784FE3846BDE89B
:10F20000F88553F8081042F8081008F1040808EBD4
:10F2100003018842ECD953F8081042F8081008F1AD
:10F22000040808EB03018842EBD8E1E72DE9F04F31
:10F23000D1F8108017690D46164687B0B845B5BF9E
:10F2400015463B460B464746B4BF1E469846AB683C
:10F2500008EB070469689C42C8BF0131FFF76EFEE6
:10F2600000EB840300F1140B143303909B450493CB
:10F2700006D204995B46002243F8042B9942FBD83E
:10F2800006EB880806F1140908F1140805EB870C51
:10F290001435C145CDF804800CF1140C02954BD205
:10F2A0004FF0000A059459F80A400AEB0B08A0B287
:10F2B000D8B1029A4346002452F8045B1968AFB2F1
:10F2C0002D0C8EB2090C00FB076600FB05113619E8
:10F2D00001EB1641B6B20C0C944546EA014643F8E0
:10F2E000046BE9D81C6059F80A40240C1CD05BF868
:10F2F0000A204146029B002510461E8897B206FB55
:10F30000045505EB104547EA05470F6051F8040F17
:10F3100053F8042B86B2120C02FB046202EB154276
:10F32000150C9C45E9D80A600AF1040A019A0AEB17
:10F3300009039A42B7D8059C002C0BDD049A52F8B9
:10F34000043C3BB9134603E053F8082C043B0AB9CC
:10F35000013CF9D1039B18461C6107B0BDE8F08F52
:10F3600010B50C460121FFF7E9FD0122446102615D
:10F3700010BD00BF2DE9F0450D46002106462C6961
:10F3800083B005F11408084658F8017001301FFADF
:10F3900087FA4FEA174C0AFB02330CFB02FC0CEB1A
:10F3A000134C9BB203EB0C4348F801300431844208
:10F3B0004FEA1C43E8DC3BB1AA68944208DA05EB4B
:10F3C000840201342C615361284603B0BDE8F08506
:10F3D0006968304601930131FFF7B0FD2A6905F1F4
:10F3E0000C010232920007460C30F9F799FF2946CA
:10F3F00030463D46FFF786FD019BE0E72DE9F041F1
:10F40000154612F00302044688462CD1AD101ED0DA
:10F41000666A002E34D0B768002F3BD015F0010F7C
:10F4200008D16D1013D03E68A6B13046074615F0DE
:10F43000010FF6D041463A462046FFF7F7FE414617
:10F4400006462046FFF75EFD6D10B046EBD1404604
:10F45000BDE8F08139463A462046FFF7E7FE3860BE
:10F4600007460660E3E742F2A87C0023C0F2010CE5
:10F470000CEB8202D2F8C420FFF77CFF8046C5E780
:10F480001020FFF73FF8002306466062C360436028
:10F4900083600360204640F27121FFF761FF002383
:10F4A000B06007460360B9E72DE9F8451E4648F607
:10F4B000396306F1080CC3F6E30388460546174690
:10F4C00083FB0C134FEAEC7CCCEB630CBCF1010F1B
:10F4D00035DD00210122520001319445FBDC284634
:10F4E000FFF72CFD089B43610123092F036122DDF7
:10F4F00008F1090A092418F8043001460A220134E7
:10F50000303B2846FFF736FFA742F4DC0AEB07083A
:10F51000A8F10808BE420CDD002418F804300146AA
:10F5200001340A22303B2846FFF724FFE3199E42AC
:10F53000F3DCBDE8F88508F10A080927EAE70021AD
:10F54000CDE700BF2DE9F04F914683B007460E4648
:10F55000002900F03A81A1F1080809F10B04FFF736
:10F5600041FB162CD8F804100B4600F2A0801022A4
:10F57000002514464C4538BF45F00105002D40F0EC
:10F580002A8121F0030A9245A2BF4046554608F160
:10F59000080875DA40F2441308EB0A00C1F20003D0
:10F5A000D3F808E0864500F01A81D0F804C02CF0AA
:10F5B000010B8344DBF804B01BF0010F7CD0AC4698
:10F5C000284611F0010F40F09B8056F8081CC1EB53
:10F5D000080BDBF8045025F00305002800F0DD805F
:10F5E000704500F01F8105EB0A030CEB0305954203
:10F5F000B8BF1D46C0F2D28081685B46C068AAF1E0
:10F600000402242A8160C86053F8081FDBF80C004C
:10F610008160C86000F2D080132A9C4621D931460F
:10F620000BF1100C51F8040BCBF8080070680E1D9C
:10F630001B2ACBF80C0014D94868311D0BF1180CAB
:10F64000CBF8100070680E1D242ACBF8140008D1E6
:10F650004A680BF1200CCBF8182072680836CBF8FA
:10F660001C20314698466246584651F8043B42F801
:10F67000043B7368CCF804304B685360DBF804300B
:10F68000C4EB050CBCF10F0F26D8421903F001039F
:10F6900043EA05054560536843F00103536038466B
:10F6A0004546FFF7A1FA284603B0BDE8F08F24F0E5
:10F6B00007042246E50F5DE72CF0030C0CEB0A056E
:10F6C0009542FFF67EAF82680B46C168404608F15E
:10F6D00008088A60D160D3E7011903F0010301EB48
:10F6E0000C0243EA04044CF0010344604B603846CA
:10F6F0005368083143F001035360FEF789FBCEE7FE
:10F7000049463846FEF706FF0546002841D0D8F89E
:10F710000430A0F1080223F0010141448A4200F0C4
:10F72000D780AAF104023146242A78D8132A034646
:10F7300021D9344654F8043B211D40F8043B031DF5
:10F74000D6F804C01B2AC5F804C014D9D4F804E0C4
:10F750001C1D01F1040CC0F804E048680CF1040120
:10F760005860231D242A06D1DCF8042062604A6810
:10F7700008315A60083308461A4650F8044B42F8DC
:10F78000044B496859604368536031463846FEF778
:10F790003FFB3846FFF728FA85E755449542AFDB33
:10F7A0005B46DBF80C00AAF1040253F8081F242A78
:10F7B0008160C8607FF630AF184631469846FFF743
:10F7C000B5F95846DBF804305AE7114603B0BDE8F6
:10F7D000F04FFEF79FBE0C2300253B6063E7DEF889
:10F7E000045004F1100B25F0030C0CEB0A005845F3
:10F7F000B8BF7046FFF6E5AE08EB0402011B41F00E
:10F8000001019A6051603846D8F80410354601F07D
:10F8100001031C43C8F80440FFF7E6F943E7FFF78C
:10F8200085F9B2E7554404F11001AC448C45B5DBD1
:10F830005D46DBF80C00AAF1040255F8081F242AE3
:10F840008160C8604CD8132A284624D931460BF170
:10F85000100051F804EBCBF808E0D6F804E00E1DD8
:10F860001B2ACBF80CE016D9D1F804E0311D0BF1BE
:10F870001800CBF810E0D6F804E00E1D242ACBF8CF
:10F8800014E008D14A680BF12000CBF81820726808
:10F890000836CBF81C203146024651F804EB42F8FA
:10F8A00004EB76684660496851600BEB0402C4EBD8
:10F8B0000C0141F001019A6051603846DBF80410F8
:10F8C00001F001031C43CBF80440FFF78DF9EAE691
:10F8D0005568404608F1080825F003055544CFE671
:10F8E000314628460093CDF804C0FFF71FF9DDF834
:10F8F00004C0009BD9E700BF0246404240EA020331
:10F9000021F0004141EAD373C3F1FE4303F57003D4
:10F91000584240EA0303D81701307047024640427C
:10F92000104321F0004141EAD070C0F1FE4000F5E3
:10F930007000C00F704700BF38B545F2BC74C1F20B
:10F940000004054608460023236000F0C9FFB0F11B
:10F95000FF3F00D038BD2368002BFBD02B6038BDA3
:10F96000B1F90E1000F076B910B50C46B1F90E10D1
:10F9700000F014FAA389B0F1FF3F15BF606523F4CE
:10F98000805343F48053A38118BFA38110BD00BFEF
:10F990002DE9F0411D468B890C461646074613F4A7
:10F9A000807F06D00223B1F90E10002200F0F6F994
:10F9B000A38923F480533846A3813246B4F90E104C
:10F9C0002B46BDE8F04100F001B900BF10B50C4670
:10F9D000B1F90E1000F0F8F9002803DB636D1B1875
:10F9E000636510BDA38923F48053A38110BD00BFBC
:10F9F00080EA010212F0030F3AD110F0030220F066
:10FA0000030021F0030150F804CB08BF51F8043B78
:10FA10000DD082F003024FEAC2026FF07F4323FA57
:10FA200002F251F8043B4CEA020C43EA020300BF25
:10FA3000ACF101329C4501BF22EA0C0212F0803F7A
:10FA400050F804CB51F8043BF2D04FEA0C604FEA77
:10FA50001C2C012828BFB0EB036F08BF1B0AF4D091
:10FA600003F0FF034FEA1060A0EB0300704700BFF4
:10FA700010F0030F0AD010F8012B11F8013B012AF6
:10FA800028BF9A42F4D0A2EB030070474DF8045D02
:10FA90004DF8044D4FF0010242EA022242EA0242CE
:10FAA00001F0030C21F0030150F8044B51F8045B02
:10FAB000BCF1020F26D04BD824F07F4CBCEB152FA5
:10FAC000A4EB020323EA04030DD113EAC21308BF17
:10FAD00051F8045B0AD18CEA040CBCEB056F0CD125
:10FAE00050F8044BE8E74FEA15255CE033F07F431C
:10FAF00052D10D784FEA146C55E04FEA146C05F0C2
:10FB0000FF0550E04FEA044CA4EB02034FEA1C4C03
:10FB100023EA0403BCEB154F17D113EAC21308BF45
:10FB200051F8045B07D18CEA040CBCEB054F08D1FB
:10FB300050F8044BE6E71B042ED10D884FEA144C15
:10FB400031E04FEA05454FEA144C4FEA15452AE0EB
:10FB500004F0FF0CBCEB156FA4EB020323EA0403D3
:10FB60000DD113EAC21308BF51F8045B0AD18CEA25
:10FB7000040CBCEB052F0AD150F8044BE8E74FEA20
:10FB8000156510E014F0FF0F06D051F8045B4FEA42
:10FB9000142C25F07F4506E04FF000005DF8044B83
:10FBA0005DF8045B70470CF0FF0205F0FF000128D0
:10FBB00028BF904204BF4FEA1C2C2D0AF3D0A2EBC1
:10FBC00000005DF8044B5DF8045B704738B545F202
:10FBD000BC74C1F200040546084611461A460023CB
:10FBE000236000F074FEB0F1FF3F00D038BD236801
:10FBF000002BFBD02B6038BD38B501FB02F1FEF7BE
:10FC000089FC0446F8B150F8042C22F00302043AAF
:10FC1000242A1AD8132A03460FD9002140F8041BBE
:10FC2000031D1B2A616008D91D1D416059602B1DF1
:10FC3000242A02BF6960596008331A46002142F83D
:10FC4000041B59605160204638BD0021F9F730FC93
:10FC5000204638BD38B545F2BC74C1F200040546F3
:10FC600008460023236000F00BFEB0F1FF3F00D0F8
:10FC700038BD2368002BFBD02B6038BD70B505461E
:10FC80000C4600294BD0FDF78BFF15B1AB69002B5B
:10FC900048D042F2FC63C0F201039C4208BF6C688A
:10FCA0000ED042F21C73C0F201039C4208BFAC6844
:10FCB00006D042F23C73C0F201039C4208BFEC68DC
:10FCC000B4F90C603EB328462146FDF7ADFE236B28
:10FCD00006463BB12846216A984736EA200628BFE7
:10FCE0004FF0FF36A38913F0800F1FD1616B41B134
:10FCF00004F14403994202D02846FEF789F8002314
:10FD00006363A16C21B12846FEF782F80023A36447
:10FD10004FF00003A381FDF745FF304670BD0E464E
:10FD2000304670BD2846FDF7EFFFB2E7284621694F
:10FD3000FEF76EF8DAE700BF40F240030146C1F279
:10FD4000000318689AE700BF38B545F2BC74C1F2E9
:10FD500000040546084611460023236000F098FD84
:10FD6000B0F1FF3F00D038BD2368002BFBD02B60E3
:10FD700038BD00BF38B545F2BC74C1F20004054679
:10FD800008460023236000F08BFDB0F1FF3F00D058
:10FD900038BD2368002BFBD02B6038BD38B545F249
:10FDA000BC74C1F200040546084611461A460023F9
:10FDB000236000F07CFDB0F1FF3F00D038BD236828
:10FDC000002BFBD02B6038BD38B545F2BC74C1F2B6
:10FDD00000040546084611461A460023236000F039
:10FDE0006EFDB0F1FF3F00D038BD2368002BFBD083
:10FDF0002B6038BD70B5044688B104F148025368E1
:10FE00005D1E07D4023302EB830656F8043D984783
:10FE1000013DFAD5A36A0BB12046984770BD40F268
:10FE20004003C1F200031C68E7E700BF70B50C4651
:10FE30000968054609B1FFF7F9FF28462146BDE8E4
:10FE40007040FDF7E5BF00BF40F24003C1F2000380
:10FE500070B51B680546984246D0436A1946BBB147
:10FE6000DA68AAB10026915941B10C682846FDF71D
:10FE7000CFFF2146002CF8D16B6ADA6804363C2E9D
:10FE800001D0DA68EFE711462846FDF7C1FF696A3D
:10FE9000096811B12846FDF7BBFF696911B1284611
:10FEA000FDF7B6FF696A11B12846FDF7B1FFA96BEE
:10FEB00011B12846FDF7ACFFE96B11B12846FDF7FB
:10FEC000A7FF296C11B12846FDF7A2FFAB6CD3F850
:10FED000881011B12846FDF79BFF696B11B12846C8
:10FEE000FDF796FFAB6903B970BDAB6A284698472A
:10FEF000D5F8D8100029F7D02846BDE8704095E71E
:10FF000081F0004102E000BF83F0004330B54FEACA
:10FF100041044FEA430594EA050F08BF90EA020F37
:10FF20001FBF54EA000C55EA020C7FEA645C7FEACA
:10FF3000655C00F0E2804FEA5454D4EB5555B8BFED
:10FF40006D420CDD2C4480EA020281EA030382EA5E
:10FF5000000083EA010180EA020281EA0303362DF0
:10FF600088BF30BD11F0004F4FEA01314FF4801CC3
:10FF70004CEA113102D0404261EB410113F0004FD5
:10FF80004FEA03334CEA133302D0524263EB43038C
:10FF900094EA050F00F0A780A4F10104D5F1200E2A
:10FFA0000DDB02FA0EFC22FA05F2801841F1000185
:10FFB00003FA0EF2801843FA05F359410EE0A5F159
:10FFC00020050EF1200E012A03FA0EFC28BF4CF08A
:10FFD000020C43FA05F3C01851EBE37101F0004540
:10FFE00007D54FF0000EDCF1000C7EEB00006EEB4D
:10FFF0000101B1F5801F1BD3B1F5001F0CD34908D7
:020000021000EC
:100000005FEA30004FEA3C0C04F101044FEA44522D
:1000100012F5800F80F09A80BCF1004F08BF5FEAB4
:10002000500C50F1000041EB045141EA050130BD94
:100030005FEA4C0C404141EB010111F4801FA4F137
:100040000104E9D191F0000F04BF01460020B1FA8C
:1000500081F308BF2033A3F10B03B3F120020CDAC4
:100060000C3208DD02F1140CC2F10C0201FA0CF0A2
:1000700021FA02F10CE002F11402D8BFC2F1200C07
:1000800001FA02F120FA0CFCDCBF41EA0C019040BD
:10009000E41AA2BF01EB0451294330BD6FEA040406
:1000A0001F3C1CDA0C340EDC04F11404C4F12002F1
:1000B00020FA04F001FA02F340EA030021FA04F303
:1000C00045EA030130BDC4F10C04C4F1200220FA5A
:1000D00002F001FA04F340EA0300294630BD21FA98
:1000E00004F0294630BD94F0000F83F4801306BF5E
:1000F00081F480110134013D4EE77FEA645C18BF52
:100100007FEA655C29D094EA050F08BF90EA020FE8
:1001100005D054EA000C04BF1946104630BD91EAE0
:10012000030F1EBF0021002030BD5FEA545C05D1E3
:100130004000494128BF41F0004130BD14F5800422
:100140003CBF01F5801130BD01F0004545F0FE4196
:1001500041F470014FF0000030BD7FEA645C1ABFCB
:10016000194610467FEA655C1CBF0B46024650EA02
:10017000013406BF52EA033591EA030F41F400212E
:1001800030BD00BF90F0000F04BF0021704730B5B4
:100190004FF4806404F132044FF000054FF0000189
:1001A00050E700BF90F0000F04BF0021704730B54A
:1001B0004FF4806404F1320410F0004548BF40421F
:1001C0004FF000013EE700BF42004FEAE2014FEA74
:1001D00031014FEA02701FBF12F07F4393F07F4F4F
:1001E00081F06051704792F0000F14BF93F07F4F81
:1001F000704730B54FF4607401F0004521F00041C4
:1002000020E700BF50EA010208BF704730B54FF049
:1002100000050AE050EA010208BF704730B511F04E
:10022000004502D5404261EB41014FF4806404F186
:1002300032045FEA915C3FF4DCAE4FF003025FEA08
:10024000DC0C18BF03325FEADC0C18BF033202EB90
:10025000DC02C2F1200300FA03FC20FA02F001FAEA
:1002600003FE40EA0E0021FA02F11444C1E600BF89
:1002700070B54FF0FF0C4CF4E06C1CEA11541DBF3C
:100280001CEA135594EA0C0F95EA0C0F00F0DEF807
:100290002C4481EA030621EA4C5123EA4C5350EAEC
:1002A000013518BF52EA033541F4801143F480133D
:1002B00038D0A0FB02CE4FF00005E1FB02E506F0CE
:1002C0000042E0FB03E54FF00006E1FB03569CF023
:1002D000000F18BF4EF0010EA4F1FF04B6F5007F29
:1002E00064F5407404D25FEA4E0E6D4146EB06069B
:1002F00042EAC62141EA55514FEAC52040EA5E5024
:100300004FEACE2EB4F1FD0C88BFBCF5E06F1ED8CD
:10031000BEF1004F08BF5FEA500E50F1000041EB04
:10032000045170BD06F0004646EA010140EA0200B1
:1003300081EA0301B4EB5C04C2BFD4EB0C0541EAD3
:10034000045170BD41F480114FF0000E013C00F3E8
:10035000AB8014F1360FDEBF002001F0004170BD0C
:10036000C4F10004203C35DA0C341BDC04F1140425
:10037000C4F1200500FA05F320FA04F001FA05F2B1
:1003800040EA020001F0004221F0004110EBD3707E
:1003900021FA04F642EB06015EEA430E08BF20EAAA
:1003A000D37070BDC4F10C04C4F1200500FA04F34D
:1003B00020FA05F001FA04F240EA020001F00041DF
:1003C00010EBD37041F100015EEA430E08BF20EA52
:1003D000D37070BDC4F1200500FA05F24EEA020E9A
:1003E00020FA04F301FA05F243EA020321FA04F0C9
:1003F00001F0004121FA04F220EA020000EBD37080
:100400005EEA430E08BF20EAD37070BD94F0000F7F
:100410000FD101F00046400041EB010111F4801FB3
:1004200008BF013CF7D041EA060195F0000F18BF64
:10043000704703F00046520043EB030313F4801FA0
:1004400008BF013DF7D043EA0603704794EA0C0F5A
:100450000CEA135518BF95EA0C0F0CD050EA410670
:1004600018BF52EA4306D1D181EA030101F00041ED
:100470004FF0000070BD50EA410606BF1046194615
:1004800052EA430619D094EA0C0F02D150EA013621
:1004900013D195EA0C0F05D152EA03361CBF104662
:1004A00019460AD181EA030101F0004141F0FE4101
:1004B00041F470014FF0000070BD41F0FE4141F485
:1004C000780170BD70B54FF0FF0C4CF4E06C1CEA85
:1004D00011541DBF1CEA135594EA0C0F95EA0C0F3A
:1004E00000F0A7F8A4EB050481EA030E52EA0335F5
:1004F0004FEA013100F088804FEA03334FF0805516
:1005000045EA131343EA12634FEA022245EA111542
:1005100045EA10654FEA00260EF000419D4208BFF3
:10052000964244F1FD0404F5407402D25B084FEAA0
:100530003202B61A65EB03055B084FEA32024FF44C
:1005400080104FF4002CB6EB020E75EB030E22BFA9
:10055000B61A754640EA0C005B084FEA3202B6EB69
:10056000020E75EB030E22BFB61A754640EA5C0018
:100570005B084FEA3202B6EB020E75EB030E22BFA8
:10058000B61A754640EA9C005B084FEA3202B6EBA9
:10059000020E75EB030E22BFB61A754640EADC0068
:1005A00055EA060E18D04FEA051545EA16754FEACA
:1005B00006164FEAC30343EA52734FEAC2025FEAE8
:1005C0001C1CC0D111F4801F0BD141EA00014FF077
:1005D00000004FF0004CB6E711F4801F04BF014348
:1005E0000020B4F1FD0C88BFBCF5E06F3FF6AFAE64
:1005F000B5EB030C04BFB6EB020C5FEA500C50F1F4
:10060000000041EB045170BD0EF0004E4EEA113176
:1006100014EB5C04C2BFD4EB0C0541EA045170BD7D
:1006200041F480114FF0000E013C90E645EA060EC1
:100630008DE60CEA135594EA0C0F08BF95EA0C0FEF
:100640003FF43BAF94EA0C0F0AD150EA01347FF437
:1006500034AF95EA0C0F7FF425AF104619462CE70E
:1006600095EA0C0F06D152EA03353FF4FDAE104671
:10067000194622E750EA410618BF52EA43067FF4C2
:10068000C5AE50EA41047FF40DAF52EA43057FF452
:10069000EBAE12E74FF0FF3C06E000BF4FF0010C5D
:1006A00002E000BF4FF0010C4DF804CD4FEA410CC1
:1006B0007FEA6C5C4FEA430C18BF7FEA6C5C1BD08E
:1006C00001B050EA410C0CBF52EA430C91EA030F0F
:1006D00002BF90EA020F0020704710F1000F91EA6C
:1006E000030F58BF994208BF90422CBFD8176FEA3A
:1006F000E37040F0010070474FEA410C7FEA6C5C08
:1007000002D150EA013C07D14FEA430C7FEA6C5C0E
:10071000D6D152EA033CD3D05DF8040B704700BF3A
:100720008446104662468C461946634600E000BF88
:1007300001B5FFF7B7FF002848BF10F1000F01BD5A
:100740004DF808EDFFF7F4FF0CBF012000205DF825
:1007500008FB00BF4DF808EDFFF7EAFF34BF0120AA
:1007600000205DF808FB00BF4DF808EDFFF7E0FF43
:1007700094BF012000205DF808FB00BF4DF808ED94
:10078000FFF7CEFF94BF012000205DF808FB00BFFB
:100790004DF808EDFFF7C4FF34BF012000205DF8DD
:1007A00008FB00BF4FEA410212F5001215D211D525
:1007B0006FF47873B3EB625212D94FEAC12343F05E
:1007C000004343EA505311F0004F23FA02F018BFE0
:1007D000404270474FF00000704750EA013005D1A9
:1007E00011F0004008BF6FF0004070474FF000006C
:1007F000704700BF08B500F0A3F8074800B10068D3
:10080000064901B109680022EFF77AFF044B0BB1EA
:10081000AFF30080FEE700BF000000000000000012
:100820000000000080B51448144B21E05C68996812
:10083000DD688C420CD0002205E0A6180832D6E90B
:10084000008941E902898C460831AA42F5D101E0CC
:1008500004EB050C1C696146002204E00832002606
:10086000002741E902670831A242F7D11433013869
:100870000028DBD1FFF7BEFF01000000F0280100D7
:1008800008B500F057F8092303604FF0FF3008BDAA
:1008900008B500F04FF8092303604FF0FF3008BDA2
:1008A00008B500F047F809230360002008BD08B52B
:1008B00000F040F8092303604FF0FF3008BD08B591
:1008C00000F038F8092303604FF0FF3008BD08B589
:1008D00000F030F8092303604FF0FF3008BD00003E
:1008E00008B50E4B1A680E4B1B6818184AB1121A3D
:1008F000002A06DA00F01EF80C2303604FF0FF30E8
:1009000008BDADEB0302002A03DBADEB0002FF2ABA
:10091000F0DD034A1060184608BD00BF58050010FE
:100920005405001001498D46014908470080001018
:100930002508010040F24003C1F200031868704727
:1009400070B542F6DC0642F6DC05C0F20106C0F2E4
:100950000105761BB61006D0002455F8243001346A
:100960009847A642F9D842F6DC0542F6E006C0F206
:100970000105C0F20106761B01F0AAFFB61006D0F1
:10098000002455F8243001349847A642F9D870BDA8
:10099000754950206C6F67206D6573736167653AA8
:1009A000200000000000000048656C6C6F204E586D
:1009B000502053656D69636F6E647563746F7273F5
:1009C0000000000075495020706F7274696E6720D6
:1009D0006F6E204C5043313778780000496E69744F
:1009E00020436C6F636B0000496E697420454D4174
:1009F000430000004572726F7220647572696E6701
:100A000020696E697469616C697A696E6720454D09
:100A100041432C2072657374617274206166746541
:100A2000722061207768696C65000000496E697406
:100A30002075495000000000536574206F776E20C8
:100A4000495020616464726573733A2025642E25D1
:100A5000642E25642E2564200A0D00005365742041
:100A6000526F7574657220495020616464726573B9
:100A7000733A2025642E25642E25642E2564200AD1
:100A80000D000000536574205375626E6574206D0F
:100A900061736B3A2025642E25642E25642E25640F
:100AA000200A0D00496E697420485454500000001B
:100AB000496E697420636F6D706C65746521000008
:100AC000496E697420454D4143206D6F64756C65B6
:100AD000000000004D414320616464723A202558B3
:100AE0002D25582D25582D25582D25582D25582094
:100AF0000A0D0000496E697420454D414320636F23
:100B00006D706C65746500000C0000A3210000008E
:100B100057616974656420666F72206E65776461E1
:100B200074610A00FFFFFFFF0000000069703A20B7
:100B3000696E76616C69642076657273696F6E2088
:100B40006F7220686561646572206C656E67746899
:100B50002E00000069703A207061636B6574207329
:100B6000686F72746572207468616E207265706F50
:100B70007274656420696E204950206865616465FF
:100B8000722E000069703A20667261676D656E743E
:100B90002064726F707065642E00000069703A20E6
:100BA00062616420636865636B73756D2E0000007D
:100BB00069703A206E65697468657220746370208C
:100BC0006E6F722069636D702E00000069636D7036
:100BD0003A206E6F742069636D70206563686F2EB4
:100BE000000000007463703A2062616420636865ED
:100BF000636B73756D2E00007463703A20666F75B9
:100C00006E64206E6F20756E7573656420636F6E01
:100C10006E656374696F6E732E0000007463703AC2
:100C200020676F742072657365742C2061626F7227
:100C300074696E6720636F6E6E656374696F6E2E84
:100C400000000000FFFFFFFFFFFF0000FFFFFFFFAE
:100C5000687474703A2F2F0032303020000000008A
:100C6000333031200000000033303220000000001B
:100C70004745542000000000485454502F312E3076
:100C800000000000485454502F312E310000000065
:100C9000636F6E74656E742D747970653A20000010
:100CA000746578742F68746D6C0000006C6F6361FC
:100CB00074696F6E3A200000686F73743A20000008
:100CC0000D0A00002F696E6465782E68746D6C00E3
:100CD0002F3430342E68746D6C00000052656665E8
:100CE0007265723A00000000485454502F312E3083
:100CF00020323030204F4B0D0A5365727665723AC0
:100D0000207549502F312E3020687474703A2F2F7F
:100D10007777772E736963732E73652F7E616461B5
:100D20006D2F7569702F0D0A436F6E6E6563746960
:100D30006F6E3A20636C6F73650D0A00485454500F
:100D40002F312E3020343034204E6F7420666F7572
:100D50006E640D0A5365727665723A207549502F9C
:100D6000312E3020687474703A2F2F7777772E7376
:100D70006963732E73652F7E6164616D2F75697071
:100D80002F0D0A436F6E6E656374696F6E3A206350
:100D90006C6F73650D0A0000436F6E74656E742D81
:100DA000747970653A20746578742F706C61696E1F
:100DB0000D0A0D0A00000000436F6E74656E742DFD
:100DC000747970653A20746578742F68746D6C0D51
:100DD0000A0D0A00436F6E74656E742D7479706528
:100DE0003A20746578742F6373730D0A0D0A00003E
:100DF000436F6E74656E742D747970653A207465F6
:100E000078742F746578740D0A0D0A00436F6E7440
:100E1000656E742D747970653A20696D6167652F10
:100E2000706E670D0A0D0A00436F6E74656E742D47
:100E3000747970653A20696D6167652F6769660D21
:100E40000A0D0A00436F6E74656E742D74797065B7
:100E50003A20696D6167652F6A7065670D0A0D0A32
:100E600000000000436F6E74656E742D74797065B8
:100E70003A206170706C69636174696F6E2F6F6383
:100E80007465742D73747265616D0D0A0D0A00002E
:100E90002E68746D6C0000002E7368746D6C000019
:100EA0002E68746D000000002E6373730000000054
:100EB0002E706E67000000002E676966000000005B
:100EC0002E6A7067000000002E7478740000000025
:100ED0002E7478740000000066696C652D7374616F
:100EE000747300007463702D636F6E6E6563746954
:100EF0006F6E73006E65742D7374617473000000FF
:100F0000253575003C74723E3C74643E25643C2F6C
:100F100074643E3C74643E25752E25752E25752E11
:100F200025753A25753C2F74643E3C74643E2573E8
:100F30003C2F74643E3C74643E25753C2F74643EC3
:100F40003C74643E25753C2F74643E3C74643E25BD
:100F5000632025633C2F74643E3C2F74723E0D0A5F
:100F6000000000002535750A00000000D80E0100C1
:100F70004D3A0000E40E0100DD3B0000F40E0100DC
:100F8000D93C0000434C4F534544000053594E2D6B
:100F9000524356440000000053594E2D53454E54C1
:100FA0000000000045535441424C49534845440019
:100FB00046494E2D574149542D31000046494E2D8A
:100FC000574149542D320000434C4F53494E47007E
:100FD00054494D452D574149540000004C4153544C
:100FE0002D41434B000000002F70726F63657373D7
:100FF00065732E7368746D6C0025213A202F686527
:10100000616465722E68746D6C0A3C68313E537978
:101010007374656D2070726F6365737365733C2FB5
:1010200068313E3C62723E3C7461626C6520776957
:101030006474683D2231303025223E0A3C74723E91
:101040003C74683E49443C2F74683E3C74683E4E94
:10105000616D653C2F74683E3C74683E5072696FE8
:10106000726974793C2F74683E3C74683E506F6CB2
:101070006C2068616E646C65723C2F74683E3C74D1
:10108000683E4576656E742068616E646C65723C7E
:101090002F74683E3C74683E50726F637374617461
:1010A000653C2F74683E3C2F74723E0A25212070E7
:1010B000726F6365737365730A25213A202F666F1B
:1010C0006F7465722E68746D6C0000002F343034BC
:1010D0002E68746D6C003C68746D6C3E0A20203C78
:1010E000626F6479206267636F6C6F723D2277680C
:1010F000697465223E0A202020203C63656E746579
:10110000723E0A2020202020203C68313E343034BA
:10111000202D2066696C65206E6F7420666F756E79
:10112000643C2F68313E0A2020202020203C683378
:101130003E476F203C6120687265663D222F223E4B
:10114000686572653C2F613E20696E7374656164E9
:101150002E3C2F68333E0A202020203C2F63656EF2
:101160007465723E0A20203C2F626F64793E0A3C0F
:101170002F68746D6C3E00002F66696C65732E736A
:1011800068746D6C0025213A202F68656164657272
:101190002E68746D6C0A3C68313E46696C6520733C
:1011A0007461746973746963733C2F68313E0A3CDF
:1011B00063656E7465723E0A3C7461626C6520778B
:1011C000696474683D22333030223E0A3C74723EBA
:1011D0003C74643E3C6120687265663D222F696EF6
:1011E0006465782E68746D6C223E2F696E64657834
:1011F0002E68746D6C3C2F613E3C2F74643E0A3C3B
:1012000074643E25212066696C652D737461747366
:10121000202F696E6465782E68746D6C0A3C2F749B
:10122000643E3C74643E3C696D67207372633D228A
:101230002F666164652E706E672220686569676835
:10124000743D31302077696474683D2521206669DA
:101250006C652D7374617473202F696E6465782ECC
:1012600068746D6C0A3E203C2F74643E3C2F74728F
:101270003E0A3C74723E3C74643E3C612068726578
:10128000663D222F66696C65732E7368746D6C22DF
:101290003E2F66696C65732E7368746D6C3C2F61AC
:1012A0003E3C2F74643E0A3C74643E2521206669EE
:1012B0006C652D7374617473202F66696C65732E71
:1012C0007368746D6C0A3C2F74643E3C74643E3CDD
:1012D000696D67207372633D222F666164652E70AD
:1012E0006E6722206865696768743D3130207769D0
:1012F0006474683D25212066696C652D7374617482
:1013000073202F66696C65732E7368746D6C0A3E6A
:10131000203C2F74643E3C2F74723E0A3C74723E33
:101320003C74643E3C6120687265663D222F7463A4
:10133000702E7368746D6C223E2F7463702E736808
:10134000746D6C3C2F613E3C2F74643E0A3C7464A7
:101350003E25212066696C652D7374617473202F9E
:101360007463702E7368746D6C0A3C2F74643E3C19
:1013700074643E3C696D67207372633D222F666121
:1013800064652E706E6722206865696768743D31F8
:10139000302077696474683D25212066696C652D6D
:1013A0007374617473202F7463702E7368746D6C22
:1013B0000A3E203C2F74643E3C2F74723E0A3C74FB
:1013C000723E3C74643E3C6120687265663D222F2B
:1013D00073746174732E7368746D6C223E2F737412
:1013E0006174732E7368746D6C3C2F613E3C2F7476
:1013F000643E0A3C74643E25212066696C652D7349
:1014000074617473202F73746174732E7368746DB8
:101410006C0A3C2F74643E3C74643E3C696D6720EA
:101420007372633D222F666164652E706E672220A1
:101430006865696768743D31302077696474683D18
:1014400025212066696C652D7374617473202F7378
:10145000746174732E7368746D6C0A3E203C2F7433
:10146000643E3C2F74723E0A3C74723E3C74643E8F
:101470003C6120687265663D222F7374796C652E1D
:10148000637373223E2F7374796C652E6373733CA0
:101490002F613E3C2F74643E0A3C74643E2521203B
:1014A00066696C652D7374617473202F7374796C25
:1014B000652E6373730A3C2F74643E3C74643E3C37
:1014C000696D67207372633D222F666164652E70BB
:1014D0006E6722206865696768743D3130207769DE
:1014E0006474683D25212066696C652D7374617490
:1014F00073202F7374796C652E6373730A3E203CDE
:101500002F74643E3C2F74723E0A3C74723E3C74ED
:10151000643E3C6120687265663D222F3430342E73
:1015200068746D6C223E2F3430342E68746D6C3CC0
:101530002F613E3C2F74643E0A3C74643E2521209A
:1015400066696C652D7374617473202F3430342E8A
:1015500068746D6C0A3C2F74643E3C74643E3C6954
:101560006D67207372633D222F666164652E706E15
:101570006722206865696768743D31302077696447
:1015800074683D25212066696C652D7374617473E0
:10159000202F3430342E68746D6C0A3E203C2F743A
:1015A000643E3C2F74723E0A3C74723E3C74643E4E
:1015B0003C6120687265663D222F666164652E700D
:1015C0006E67223E2F666164652E706E673C2F61E8
:1015D0003E3C2F74643E0A3C74643E2521206669BB
:1015E0006C652D7374617473202F666164652E7051
:1015F0006E670A3C2F74643E3C74643E3C696D67C0
:10160000207372633D222F666164652E706E6722BF
:10161000206865696768743D313020776964746853
:101620003D25212066696C652D7374617473202FCC
:10163000666164652E706E670A3E203C2F74643EBE
:101640003C2F74723E0A3C2F7461626C653E0A3C0A
:101650002F63656E7465723E0A25213A202F666FEE
:101660006F7465722E68746D6C0A00002F666F6F60
:101670007465722E68746D6C0020203C2F626F645C
:10168000793E0A3C2F68746D6C3E00002F686561DE
:101690006465722E68746D6C003C21444F4354594C
:1016A00050452048544D4C205055424C494320222F
:1016B0002D2F2F5733432F2F4454442048544D4C43
:1016C00020342E3031205472616E736974696F6EEC
:1016D000616C2F2F454E222022687474703A2F2F90
:1016E0007777772E77332E6F72672F54522F687467
:1016F0006D6C342F6C6F6F73652E647464223E0AB8
:101700003C68746D6C3E0A20203C686561643E0A4A
:10171000202020203C7469746C653E57656C636FB3
:101720006D6520746F207468652075495020776559
:101730006220736572766572213C2F7469746C65E2
:101740003E0A202020203C6C696E6B2072656C3D47
:10175000227374796C65736865657422207479707E
:10176000653D22746578742F6373732220687265F7
:10177000663D227374796C652E637373223E20205C
:101780000A20203C2F686561643E0A20203C626F7D
:101790006479206267636F6C6F723D2223666666B0
:1017A0006565632220746578743D22626C61636BA9
:1017B000223E0A0A20203C64697620636C617373C0
:1017C0003D226D656E75223E0A20203C64697620BC
:1017D000636C6173733D226D656E75626F78223E36
:1017E0003C6120687265663D222F223E46726F6E14
:1017F0007420706167653C2F613E3C2F6469763EC2
:101800000A20203C64697620636C6173733D226D0D
:10181000656E75626F78223E3C6120687265663D38
:101820002266696C65732E7368746D6C223E46691E
:101830006C6520737461746973746963733C2F61A0
:101840003E3C2F6469763E0A20203C646976206322
:101850006C6173733D226D656E75626F78223E3CDC
:101860006120687265663D2273746174732E7368BB
:10187000746D6C223E4E6574776F726B2073746169
:10188000746973746963733C2F613E3C2F6469769D
:101890003E0A20203C64697620636C6173733D22AC
:1018A0006D656E75626F78223E3C61206872656678
:1018B0003D227463702E7368746D6C223E4E6574A5
:1018C000776F726B0A2020636F6E6E656374696F49
:1018D0006E733C2F613E3C2F6469763E0A20203CAB
:1018E00062723E0A20203C2F6469763E0A20200A5C
:1018F00020203C64697620636C6173733D22636FC2
:101900006E74656E74626C6F636B223E0A00000039
:101910002F696E6465782E68746D6C003C21444FAD
:1019200043545950452048544D4C205055424C4941
:101930004320222D2F2F5733432F2F445444204828
:10194000544D4C20342E3031205472616E736974C2
:10195000696F6E616C2F2F454E222022687474705F
:101960003A2F2F7777772E77332E6F72672F545257
:101970002F68746D6C342F6C6F6F73652E64746494
:10198000223E0A3C68746D6C3E0A20203C6865610A
:10199000643E0A202020203C7469746C653E5765C3
:1019A0006C636F6D6520746F207468652075495095
:1019B0002077656220736572766572213C2F7469A9
:1019C000746C653E0A202020203C6C696E6B20728E
:1019D000656C3D227374796C65736865657422204B
:1019E000747970653D22746578742F637373222057
:1019F000687265663D227374796C652E6373732219
:101A00003E20200A20203C2F686561643E0A202089
:101A10003C626F6479206267636F6C6F723D222352
:101A20006666666565632220746578743D22626C23
:101A300061636B223E0A0A20203C64697620636C55
:101A40006173733D226D656E75223E0A20203C64F1
:101A5000697620636C6173733D226D656E75626F8C
:101A600078223E3C6120687265663D222F223E4608
:101A7000726F6E7420706167653C2F613E3C2F640D
:101A800069763E0A20203C64697620636C6173733A
:101A90003D226D656E75626F78223E3C61206872F2
:101AA00065663D2266696C65732E7368746D6C2281
:101AB0003E46696C652073746174697374696373FD
:101AC0003C2F613E3C2F6469763E0A20203C6469CD
:101AD0007620636C6173733D226D656E75626F78FD
:101AE000223E3C6120687265663D227374617473A6
:101AF0002E7368746D6C223E4E6574776F726B2026
:101B0000737461746973746963733C2F613E3C2F15
:101B10006469763E0A20203C64697620636C6173B8
:101B2000733D226D656E75626F78223E3C61206860
:101B30007265663D227463702E7368746D6C223E0C
:101B40004E6574776F726B0A2020636F6E6E6563EB
:101B500074696F6E733C2F613E3C2F6469763E0A58
:101B600020203C62723E0A20203C2F6469763E0AA7
:101B70000A20203C64697620636C6173733D2263A4
:101B80006F6E74656E74626C6F636B223E0A202008
:101B90003C703E0A2020546865736520776562209A
:101BA0007061676573206172652073657276656424
:101BB000206279206120736D616C6C2077656220F2
:101BC0007365727665722072756E6E696E67206FCE
:101BD0006E20746F70206F660A2020746865203C48
:101BE0006120687265663D22687474703A2F2F77A1
:101BF00077772E736963732E73652F7E6164616DD1
:101C00002F7569702F223E75495020656D6265649D
